:040000050000FDC139
:020000040000FA
:1000000028430020398F000001CA011001CA0110E5
:1000100001CA011001CA011001CA011001CA011070
:1000200001CA011001CA011001CA011001CA011060
:0C00300001CA011001CA01103FCA0110F2
:100100003C0000000000000000000000340100007E
:1001100000000000000000000100000000000000DE
:1001200000000000000000000000000001000000CE
:100130000000000008000000000000003400000083
:100140000000000000000000680100000000000046
:10015000000000000100000000000000010000009D
:100160000000000000000000080000000000000087
:1001700030000000000000000000000098010000B6
:10018000040000000000000001000000FFFFFFFF6E
:10019000FF00000001000000080000000000000057
:1001A0002C0000000000000000000000C40100005E
:1001B000040000000000000001000000FFFFFFFF3E
:1001C000FFFFFFFF080000000000000034050000F2
:1001D000E401000099A1011095A70110A5C201102A
:1001E00009B2011045B80110000000000000000035
:1001F0002F000000280000000000000000000000A8
:10020000140200000000000000000000FFFFFFFFDC
:1002100000000000080000000000000030050000A1
:100220003002000069C201106DC101101FC201102F
:1002300095BA011000000000000000002D00000031
:10024000300500005402000075C20110A9B601106B
:100250009DBF011049B60110000000000000000021
:100260002E0000002400000000000000000000003C
:1002700080020000000000000000000000000000FC
:100280000800000000000000240000000000000042
:1002900000000000A40200000000000000000000B8
:1002A0000000000008000000000000002400000022
:1002B0000000000000000000C80200000000000074
:1002C0000100000000000000080000000000000025
:1002D000000000002C0B00200400000000000000C3
:1002E000000000002000000070010000300000004D
:1002F0001C0200004C0B0020040000000000000065
:10030000000000000C000000300400001800000095
:1003100040020000540B0020040000000000000018
:100320000000000024000000480400001800000045
:1003300000000000940B00200400000000000000FA
:100340000000000010000000A00100002C000000D0
:10035000CC0100009C0B0020040000000000000005
:1003600000000000200000006402000024000000E3
:10037000FFFFFFFFBC0B0020040000000000000096
:100380000000000028000000880200002400000097
:10039000FFFFFFFFE40B002004000000000000004E
:1003A00000000000580000003C0100003400000084
:1003B000FFFFFFFFEC0B0020040000000000000026
:1003C00000000000100000006004000018000000A1
:1003D000FFFFFFFFF40B00200400000000000000FE
:1003E000000000001C000000AC020000240000001F
:1003F000FFFFFFFFFC0B00200400000000000000D6
:100400000000000038000000F40100002800000097
:10041000FFFFFFFF640C002004000000000000004C
:100420000000000054000000000100003C0000003B
:100430001800000000000000000000004004000060
:10044000080000000000000018000000000000008C
:100450000000000058040000080000000000000038
:100460001800000000000000000000007004000000
:10047000080000000000000001000000A48F000040
:100484000100000000000E0000000F003200000018
:1004940001000000340B00200002000000000000F6
:1004A40001CA011000000000000000000800000064
:1004B400000023005C0B002001000000A40B0020BE
:1004C4000800000000000000000000000000000020
:1004D400000000000000000001000000040C0020E7
:1004E40006000000010000006C0C00200000000069
:0C04F400000000000002000000000000FA
:0F0502002900010025002D002E002F000100010F
:1005140004000000788F00000000000000000000CC
:10052400000001000000030087C40110380500002A
:10053400380500000000000090000000900000005A
:1005440000000000A40B0020492E00002000000041
:10055400508F0000208D00000DC30110FB1D000012
:10056400FD1D000099C801109BC801100000000087
:10057400E62A0000888C0000A08C0000708C00002B
:090584000800090001000000015B
:10059000000000000000000000000000000000005B
:1005A000E1190000011A0000051900002B1A0000D3
:1005B0004D190000231900007F190000571A000090
:1005C000C12D0000D12F0000D52F00000800000031
:1005D0002400000018000000280000002000000097
:1005E0003C0000000C00000034000000DFF800F0C8
:1005F00049C10110DFF800F019C20110DFF800F066
:1006000041AC0110DFF800F0CDA00110DFF800F0E0
:1006100085C10110DFF800F0C1C20110DFF800F061
:10062000E3BF0110DFF800F0C1C10110DFF800F0F6
:1006300009B70110DFF800F03DC10110DFF800F04C
:1006400029AF0110DFF800F0CDC10110DFF800F094
:1006500085B00110DFF800F0DDB20110DFF800F026
:1006600079B50110DFF800F0D5C00110DFF800F017
:10067000E1B5011020B1082328220021FFF7E2BFD5
:10068000704720B1082330220021FFF7D3BF704705
:1006900038B500F091FF25680DB129682160FFF79A
:1006A000A9FF284632BD70B504460D4626680020D5
:1006B00028601EB9FFF79AFF25600DE0FFF796FF4F
:1006C00000E0366831680029FBD1AE4203D1FFF764
:1006D00091FF002070BD3560FFF78CFF012070BDD9
:1006E0000022DFF8541C01EB4211CB7F1B0605D51D
:1006F000B1F91C30834201D108467047521C082AC8
:10070000EFDB0020704770B50646FFF76FFFDFF89C
:10071000545C0446A87E01001AD0401EA876C0B2E0
:10072000B0B9082100F026FC96B1A86B703001F03A
:100730007CF800F010FE301AB0FBF1F1022938BF4E
:100740000121EC352846FFF765FF2846FFF766FFD5
:10075000204600F065BE10B50446207B00F00F0077
:1007600002280FD100F012FDA168081ADFF8F41B6F
:10077000896BC968800801F57A71814238BFB0F190
:10078000405F00D3002010BD38B5DFF84C0ADFF819
:100790004C2A0168DFF87C4C02EA0105E94301605C
:1007A000A90608D54068800605D54FF4005104F12C
:1007B0004C0001F064F815F4602F08D0206905F4AE
:1007C000602108432061002104F19C00D0E131BD8B
:1007D00070B5FFF70BFFDFF83C4C0646206910F4BC
:1007E000602F27D02069C5012D0EE80748BF0025DE
:1007F00006D4A80748BF012502D4680748BF0225D0
:10080000681D40B200F040FF2069012105F111028E
:100810009140884320613046FFF7ECFE04EB8500F1
:100820004668300009D0206800224FF00063691D3F
:10083000B04702E03046FFF7DDFE206930B104F139
:100840009C00BDE87040002101F019B870BD70B582
:1008500001F0E0FBDFF80C5BDFF8BC4BAB6A024653
:1008600090071DD4D3E90401104007D0EB629969C9
:10087000084398614FF4804100F07CFBA86A00288F
:1008800047D16E6A002E44D0F068A96B884224D00C
:1008900005F14C00BDE870404FF4805100F0EFBF0F
:1008A0000BB9A86AEAE70020A862D3E904019E69AF
:1008B000024042F0020232439A61626982436261FD
:1008C000E26822EA0100E060194605F13000FFF716
:1008D000EAFE022100F04EFBE3E7B068FFF73BFFC2
:1008E000A86408B1A86CD8E0D6E9040162690243A3
:1008F0006261E26841EA0200E0600020E061B06805
:100900002060E0690028FCD005F12400FFF7C0FE5C
:10091000AE6270BD0020F6E6F8B506461446376EA6
:100920001D4607B1B847A00708D4D6E916012040F4
:1009300029400022914208BF904207D0C6E91A45DB
:1009400006F13800BDE8F240FFF758BEF1BDFEE702
:1009500080B500F084FFDFF8BC2A0146906BD26BB3
:10096000BDE80840104710B5DFF8A84A0FF2311172
:10097000E06B884202D101F0A9FB206404F14C0035
:10098000BDE81040042100F07ABF80B501F042FBC1
:10099000DFF8881A084207D0BDE804404FF0005144
:1009A000DFF8100C00F06BBF01BD70B5040073D010
:1009B000A168202001E04968401E79B1C2B26AB145
:1009C0000A8840F603039A421CBF40F604039A4289
:1009D000F1D1E0681822203001F094FBA0690021D9
:1009E000A1616168D9B140F00202E07F002300F00C
:1009F0000700012807D0022809D0042804BF0022DC
:100A00004FF0805306E000224FF0005302E0002236
:100A10004FF08043B4F91C10E0686568A847FFF701
:100A2000E5FDDFF840590646E88E401CC0F30B0098
:100A3000E8860020296BC87705F13000FFF728FE13
:100A40003046FFF7D7FDB5F93610E06800F1B8027F
:100A5000B2F90030994204BF297E00291CD1917857
:100A600009B9016811B90020907016E0AA6B1268EC
:100A700012F1010F10D0DFF8F42B1268B1FBF2F184
:100A8000022938BF01217030FFF7C4FDE068BDE8DE
:100A900070407030FFF7C2BD70BDBDE8704032E6F7
:100AA00038B50D46A807DFF8BC4816D5206BFFF710
:100AB0007CFF206B25F0020510B145F0020109E032
:100AC000680702D4606A002851D004F1EC0000F0FD
:100AD000ACFE042104F14C004AE0680747D5606A87
:100AE00008B1C068A063A06BDFF8E42A41680B7806
:100AF0001360126809788A421CBF8569002D05D0F1
:100B000000224FF000736FF0FF01A847022001F0B0
:100B10005DFC112001F06FFC01206077A06BE17E8D
:100B2000007C084204BF0E2001F065FCA06BDFF8DA
:100B3000E81840688268002A04BFC068002804D012
:100B40000020C861DFF8D80A086040F2FF70DFF8C3
:100B5000D42A106000208861DFF8C00848610FF2D5
:100B60001900E0631920BDE83240FFF773BD31BDC5
:100B7000BDE8344000F083BE2DE9FF478046880081
:100B800040F1B580DFF8DC57A86B40684068010091
:100B900018BF8047A86BDFF88098406881680029FB
:100BA00004BFC168002914D0D9F81C100029FBD05B
:100BB0000021C9F81C108068010018BF8047A86B8D
:100BC0004068C068010018BF8047DFF8B40A01F030
:100BD00029FA0020C9F81C0040F60A0ADFF8A40A26
:100BE000DFF8E07AC9F8000008F10804012001F0FC
:100BF00061FA0FF25110E863A7F800A00020788096
:100C0000002100F0B0F900F0A7F9206806467180D5
:100C1000E97E09B1617A99B1018840F602029142F8
:100C200005D1318A4FF60F421140318204E0318BF9
:100C30004FF60F42114031830021617201F028FA12
:100C40002068694601F016FA684601F022FA00E0D1
:100C50000646706800281CBF01885145F8D17760AE
:100C600040F60301707B00F0F0007073686A8068E2
:100C7000008888421CBF40F60401884202D100204F
:100C8000286417E0208BA8B100206083E06108F1A0
:100C90002C00017801F0F0010170417801F0F001C1
:100CA00041F00101417008F120007860787B00F08C
:100CB000F0007873D9F81C000028FBD00020C9F898
:100CC0001C00012001F056FE012808D0707B00F0C6
:100CD000F00040F0010070730FF21900E8634FF666
:100CE000FF322068018A11400182C9F80000BDE886
:100CF000FF870000DFF8D009014200D170470120D2
:100D000010B501F037FE0128DFF8584608D10FF280
:100D10003500DFF80417E063DFF8A809086010BDAC
:100D2000DFF8481909683220B0FBF1F1022938BF19
:100D30000121EC342046FFF76DFC2046BDE8104051
:100D4000FFF76CBC2DE9FE4306460C466004DFF855
:100D5000145619D5FFF74AFCEE6AB769B9070ED4E5
:100D60006EB10021B161FFF745FC706848B1B6F97A
:100D70001C10F06876683A460023B04701E0FFF7A0
:100D800039FC24F48044E1E0A0070AD5286BFFF782
:100D90000CFE286B002824F0020401D044F0020469
:100DA000D4E0A00005F1800840F60909DFF81479C5
:100DB00071D5B068018840F60202914205D1028ADD
:100DC0002D2161F30912028204E0028B2D2161F3CF
:100DD00009120283286CB8B1042001F0CBFD98B150
:100DE00001F074F9296C814228BF401E401A718AB3
:100DF00011EB1030F06040F2D761A0F2EE20884293
:100E000024BF40F6C410F060D6F818C0BCF1000F43
:100E10001CBFDFF8BC188C450DD0787B0F21084231
:100E200004BF708C484506D100224FF000736FF468
:100E300080713046E0470022DFF89818404600F005
:100E400031FD287F50B10220ADF80000684601F066
:100E5000E9F8BDF80800A88200202877012068760C
:100E6000A87E401CA87600206877686A18B119200F
:100E700000F01BFD01E044F00204D6F81480B8F144
:100E8000000F05D000224FF0806300213046C0479C
:100E900024F000545AE095F8200024F0080628B108
:100EA000200703D5002085F820003CE020073CD532
:100EB000002068760120A877002001F0FBF80FF2EF
:100EC000BD00DFF81418DFF86047E86300224046F1
:100ED00000F0E8FC297FE87E81F00101084202D1A0
:100EE0000120E8760FE0A86CB8B101F0EFF8296CAA
:100EF0006A6C401A02EB10306864A96CB0EBC11F39
:100F00000BD300206864A7F8009000F025F80020BB
:100F1000788000F028F8276003E04FF0005100F0DF
:100F200029F800202864344610E0A0040ED5AE6AEB
:100F3000002E1CBF7068002806D0B6F91C10F0689F
:100F4000766800222023B04724F4005414B12146CF
:100F500000F010F8BDE8F783787B00F0F00040F077
:100F6000010078737047387B00F0F0003873002080
:100F70007860704705F14C0000F081BC70B5054603
:100F80000E46B007DFF8DC430BD5206BFFF70DFDF5
:100F9000206B08B1022129E0B0002DD54FF000519F
:100FA00024E0B00028D501F04AF8DFF83007DFF878
:100FB0003067E063307818B905F13800FFF71EFBA1
:100FC000DFF8601600200860022001F095F911207A
:100FD00001F0A6F9287C10B90E2001F0A1F900203B
:100FE000E083B07840B10020B070042104F14C00DF
:100FF000BDE8704000F043BC70BD30B58DB001F06D
:10100000FCF8DFF8E006DFF8E0460168DFF854534B
:1010100041F00201016001A8FFF72CFBA078DFF886
:10102000CC160790002301AA05F14C00FFF70EFB38
:1010300001A8FFF726FB0020ADF81C0001AB2078CB
:10104000DFF89426099019210020009005F1800016
:10105000FFF7F4FA01A8FFF70DFBE078DFF8901630
:101060000790002301AA05F19C00FFF7EFFA01A801
:10107000FFF707FB0120ADF81C0001AB6078DFF83B
:10108000742609901A210020009005F1D000FFF786
:10109000D5FA00230022DFF8601605F1EC00FFF717
:1010A000DDFADFF83806E8630DB04FF6FF70A8826E
:1010B000012028770020E875E8766877E88385F8CE
:1010C0002000286430BD2DE9F041DFF814660446A5
:1010D00030788EB00F4690461D4618B9FFF78DFF49
:1010E00001203070002F1CBF6760B8F1000F4BD09B
:1010F000C4F80880FFF77AFA7178002942D10121FB
:101100007170FFF777FA35B909A80FF2246114223C
:1011100000F0F8FF09AD286820606868E060287C6E
:101120002074A868606101206074688A6082E86841
:10113000010018BFA061A02104F1200001F0D0FC43
:101140000823242200216846FFF76CFA01208DF85D
:1011500018006A46002104F13800FFF767FA0823F7
:10116000242200216846FFF751FA06946B460022BC
:10117000DFF8881504F17000FFF770FA20460EB012
:10118000BDE8F081FFF736FA0020F8E738B5FFF741
:101190002DFA7449497E31B1DFF868150C68FFF704
:1011A00029FA204632BDFFF725FA00F08FFF10F52F
:1011B0000030DFF8542541F10001A2FB0045DFF8C3
:1011C0000C0502FB015501690020221845EB0103C3
:1011D000184632BD000000000810044020000E0038
:1011E0002DE9F84F04460E4692469B46FFF7FEF95E
:1011F0005C4D8046B5F93400B5F93610401AC0F39D
:101200000B0008286FF0010944DAA88E401CC0F3D7
:101210000B00A886B5F93400ADF80000002046495F
:1012200001EB4017F97F090604D5401CC0B208281D
:10123000F5DB002704F1700000F0F7FABE6087F8D4
:101240001EA0C7F804B02021BDF80000B883FC60E0
:10125000DDE90A23DFF8B40410401940C7E90401AE
:10126000B8340020F87740F6FF76686A00283946DF
:1012700005F1240006D0FFF716FA30B100F05EF851
:1012800040464BE0FFF70FFA40B9A88E3018C0F384
:101290000B00A88600F070F948464AE000F04EF8CE
:1012A000E87F697E084208D0012085F820000020F0
:1012B000E8772877A87E401CA87600F05DF9A86A38
:1012C000002834D1687E18B1192000F0EEFA2EE023
:1012D000687F60BBFFF78AF90446A87F20B1DFF87A
:1012E00000140120887018E0B868FFF734FAA86489
:1012F000B8B100F030F8AA6C121AB2FBF1F2022A6F
:1013000023BFAA6C101AB0FBF1F10121EC3528467D
:10131000FFF780F92846FFF781F92046FFF76AF9C1
:1013200005E02046FFF766F90421FFF723FEBDF92B
:101330000000BDE8F28F0000180E0020BDF800008C
:101340002080F87F40F08000F877A07810B100206E
:10135000A07028777047A86BDFF81013C068096881
:1013600070470000982100202DE9F04106460F4605
:1013700014461D46FFF776F980463846FFF7B0F968
:10138000070003D14046FFF771F90AE0F87F072113
:10139000084209D04046FFF769F90721F87F084263
:1013A000FCD10220002116E07968DFF86403814255
:1013B00002D0796831667860C6E916454046FFF785
:1013C00055F94FF0FF3106F13800FFF71BF9002007
:1013D0003066D6E91A01BDE8F081DCB5DDE90667C3
:1013E0000446CDE90067180008BFDFF82433204623
:1013F000FFF7F6FE002803D500204FF00041DCBDCA
:101400000146204602B0BDE8D04002224FF0E04342
:10141000AAE70000982100200010044002000040CC
:10142000BDE87040FFF7E6B801E042F002022DE9A6
:10143000F843DFF8CC42606A0090894603271546DE
:10144000FFF7D4F819F1010F05F0010680460AD123
:10145000A06A002819BFA06AB0F91C90E08E00F1C4
:1014600001090020E0750FFA89F0FFF739F9010052
:1014700070D0A06A814205F0020525D1280003D072
:10148000606A0090002060620122C87FB240104371
:10149000C877FFF7E7F80746002E14BFDFF874029D
:1014A000DFF8740200F0BEFD00F066F825B906E032
:1014B00000F055F800F05BF800980028F8D13846A5
:1014C000FFF7D4F8832747E0009A8A4204F1EC0042
:1014D00016D100F0AAF9280012BF0020606A006847
:1014E000606200F049F8009800F039F800F03FF829
:1014F000009818B32800F6D120E0009A12680092F4
:10150000009AEAB112688A42F7D100F08EF9009889
:1015100000681DB1009A0021116004E00168009A82
:10152000116000210160009003E000F018F800F065
:101530001EF800980028F8D100F01EF8832701E07B
:1015400000F01AF8607F38B9022104F14C0000F075
:1015500096F901E000F010F83846BDE8F283C07F4C
:10156000009940F00400C8776846FFF791B801463B
:1015700004F13000FFF797B84046FFF73BB838B5A5
:1015800000F01AF805465E48407E68B1204600F03B
:1015900049FD044600F04AF804F0FF00012801D19B
:1015A000812032BD022032BD00F040F8012032BD62
:1015B00000000000E42100200446FFF717B80A46A7
:1015C0004F49896B884201D00320704709E0000031
:1015D000D02108400A464A49896B884201D003203D
:1015E000704700211046CAE770B545498A6B9042A2
:1015F0006FF07F0411D1487E78B1FEF7F7FF054602
:10160000464800F00FFD064600F010F806F0FF0017
:10161000012802D13002001670BD204670BD0000C6
:101620005100070600000460001004402846FEF741
:10163000E1BF70B50E461546FEF7D8FF832430494A
:101640001EB1022E0DD005D30EE08A6A3AB1896A26
:10165000898B02E00A7F12B9898A298005E08024FB
:1016600003E0497E297000E003245BE09C8F0000CA
:1016700080B50846FFF734F800B1806802BD00006D
:101680000100070601010E0438B5FFF795FF1C495C
:10169000CA7D520702D58B7D9C420FD001228B8AD6
:1016A00002FA04F52B438B820C341D4B1D68A240BB
:1016B00025EA02021A601A6802B90A76BDE83240C9
:1016C000FEF798BFA822002004000020A8220020D6
:1016D0004F0900004F0800008B090000A10A00001C
:1016E0009F260020002009409C890000510900002D
:1016F000D1070000890700006709000015090000F4
:10170000982100200430044000093D00F1EFFF9FC4
:101710001909000001000204010001040100030492
:101720000C100440FEF766FF204670BD000000006C
:10173000FFFFFFFFC4090000000000004F09000088
:1017400001001A01DFF800F021B30110DFF800F00A
:1017500095C00110DFF800F00DA80110DFF800F0CF
:10176000BDBE0110FEE7DFF80001007D70476DE0AF
:1017700038B5FFF7FCFFDFF8F8500446A8680021F1
:10178000FFF7E4FF6969081AA969814238BF0020A0
:1017900084F3118832BD2DE9F041FFF7E8FFDFF84F
:1017A000D0500446A8680121FFF7D0FF0121A9838A
:1017B0000021E9836E6929682A68871B801A711ADB
:1017C000884204D20020A88384F311882BE084F39C
:1017D0001188002406E0A61931460120FFF7BAFF60
:1017E0003F1B0446A742F6D2FFF7C1FF8046E88BB5
:1017F000012804D131460020FFF7ACFF0446A96957
:1018000014F1010F08BF084603D0E01B814238BF26
:1018100008468119FFF7A2FF012028840020A88331
:101820002E6088F31188BDE8F08100218182DFF805
:101830003C10C0684969884204D1DFF85C00006848
:10184000FEF7ECBE7047808A70477047DFF84C1097
:101850000968EFF3118081F311887047F6E7DFF82C
:101860004000806870470000A4010020780100203B
:1018700078010020616280F311882046704738B5F6
:1018800004460D46FFF7EAFF616A2943FFF7F2FFBE
:10189000BDE83240FFF756BFA08F0000988F0000D0
:1018A000C8010020816042607047102804D3DFF82F
:1018B0000C101038C1F8000F7047000000E000E085
:1018C00001F012B9FFF7C2BFDFF89811C20744BF99
:1018D00001220A60820744BF4FF480720A60400709
:1018E00044BF4FF4803008607047DFF87C21C307A5
:1018F00048BF1160830748BF5160400748BF9160EF
:101900007047000010B504460020D4E90A2347F6CA
:10191000906101F095F90123994228BF4FF0FF3003
:1019200010BD10B50C4600F0C7FB011D201AB0F128
:10193000004F05D8081BB0F1004F38BF8C4200D2D1
:101940000C462146BDE810400120CEE72DE9F041CC
:1019500080460A46D8E90A01D8E90C45A0FB02678F
:1019600001FB0277A6196F41340C002244EA0741BB
:101970004046FFF7D6FFC8E90E67BDE8F081F8B52D
:101980000646FFF79FFF0446DFF8E050DFF8E070FF
:101990000120E861FFF798FFF96A096A1420884777
:1019A0003069B0F5802F34BF0421010C0120FFF70E
:1019B0009CFF3A681268232100209047DFF8B4109A
:1019C00001200860DFF8B400016821F4E02141F44F
:1019D000803101600120286084F31188F1BD00008E
:1019E00000F074BB10B5DFF89000446800F006F812
:1019F0006069A169BDE8104008470000012063E765
:101A0000F8B504460D4600F061FBD4E90A6732469A
:101A10003B4601F015F93DB1A6FB002306FB01335F
:101A200007FB0033C4E90C23F2BD10B5DFF83C001E
:101A3000DFF86440002101600121C161216020685C
:101A4000FFF7DCFFDFF860100968096A1420884797
:101A5000206810BD000080B500F038FB000C40EAA3
:101A6000014002BD04200940182009400000244321
:101A70008401001080022443E4010020002009407A
:101A8000DFF8EC14096821B10A898242FAD10846CC
:101A900070470020704700002C200940DFF8D80470
:101AA000C088704700000000B001001000F008F886
:101AB0000EBD00BF08B582B00023009302ABF5E76E
:101AC00077B58DB01C461498ADF8180000250F9816
:101AD00028B92CE10EAA0DA800F070F96D1C00F0D9
:101AE00032F9080000F01D812529F3D100F02BF90F
:101AF0002D2905D10120ADF8060000F024F902E0FF
:101B00000020ADF80600302904D10120049000F037
:101B10001AF901E000200490002000904FF0FF30FF
:101B200002900A202A2918D12168216051F8042B3B
:101B30002160009200F0FDF8009A002A11D50122E0
:101B4000ADF80620009A524200920AE0009A00FB8B
:101B500002113039009100F0ECF8A1F130020A2AAC
:101B6000F4D32E291AD1002100F0F2F82A290F927D
:101B700010D100F0F9F80291002944BF0020029032
:101B800000F0E1F80AE0029A00FB0211303900F09F
:101B9000DFF80F92A1F130020A2AF4D3049808B1B9
:101BA000009804906C2918BF4C2905D10120ADF88C
:101BB000040000F0C8F802E00020ADF8040008A816
:101BC00007900CA805900020642918BF692903908C
:101BD0000DD1BDF818000028FFD000F0BFF86FF05D
:101BE00009030298049A8242B8BF049019E00A23BC
:101BF00075291FBF1023782908236F2903D1BDF849
:101C0000180038B906E0702913D1049320682060C9
:101C1000016814E000F0A2F8049A02988242B8BF6A
:101C20000490049A059800F0A5F807900599081A01
:101C30002FE0632919D12068206001680FE0001DA2
:101C4000206010230598082200F094F8401E0790A9
:101C500040200799087005980799401A19E0001D5F
:101C6000206007980170012013E0732913D100F060
:101C70007BF8079111B90FF244300790079801F0F3
:101C800057F80390029810F1010F1ED00399884273
:101C90001BDA039019E00F98401E0F900E9802284F
:101CA00013D3029810F1010F02D00E99884201D38C
:101CB0000E9800E0401CDFF8C462366802906B4664
:101CC00022460FA90DA8B047451900980399401A5C
:101CD0000090BDF8060038B902E000F030F86D1C45
:101CE0000098401E0090F8D50398411E039150B112
:101CF0000798401C07900EAA10F8011D0DA800F0CF
:101D00005DF86D1CF0E7BDF8060000283FF4E7AE73
:101D10000098401E00903FF5E2AE00F010F86D1CF8
:101D2000F6E70D9810B10D9900200870284610B004
:101D300070BD0F990F9A0978521C0F9270470EAA26
:101D400020210DA83AE00F9810F8011B0F90704762
:101D500002910F990F9A0978521C704720682060F1
:101D60000168001D206070472068206050F8041B47
:101D700020607047F0B500240025002B44BF5B4273
:101D8000002902D54942521E2D25B1FBF3F60FF270
:101D9000342703FB1611641C795C00F8011D3146E1
:101DA0000029F2D19442BEBF302100F8011D641C0D
:101DB000F8DB290018BF00F8015DF0BD10B50C4636
:101DC000116802290BD3491E1160016819B14A1C20
:101DD00002600C7010BD01F001F900B100E010BD0F
:101DE0002046BDE8104001F0F7B86549096808478A
:101DF00064480068004701207047FEE7704770475D
:101E000010B50446606808B9012010BD0B460146B4
:101E1000206852A200F0BCF8A1684118A160616876
:101E20000129A4BF081A6060002010BD2DE9F0410F
:101E300004468846A088164600F021F80746F11BA4
:101E4000002E01D40A2904DB236845A200F083F8A0
:101E5000C719A08980B1F51BA468002E05D42046BF
:101E600000F066FF401D854206DB23460FF2681234
:101E7000294600F070F8C7193846BDE8F0813EB534
:101E80000D463A49098814468142034628BF0FF29D
:101E9000501210D237490988814207D3FFF7F0FD6D
:101EA00021464268284600F073F83EBD2D49098856
:101EB00031B90FF238122146284600F069F83EBDCC
:101EC000314B1B680095002C48BF47F6FF7400217A
:101ED000029101946A462D49984702983EBD2DE92A
:101EE000F843170048BF47F6FF77044688460026A8
:101EF00074B32088010004D03A464146FFF7BFFF83
:101F00000646B91B012922DB208820B116A24046D3
:101F100000F03EF88619A068C8B1656875B128461A
:101F200000F006FFA7EB0609401D814506DB2B46A6
:101F30000FF2CC02494600F00EF88619B91B12299F
:101F400005DBA3680FF2C00200F005F886193046E1
:101F5000BDE8F283000040461AE00000257300004F
:101F6000257000008A0500003A2000005A21000078
:101F7000FC0D0020B6200000F0010020B08F000012
:101F8000A88F0000AC8F0000B48F0000011E00007D
:101F900008B478B504001ABF2668002E00260D4646
:101FA00005AB3046FFF786FD854238BF681E16B187
:101FB00021680144216072BC5DF808FB286E756CD5
:101FC0006C290000303132333435363738396162AC
:101FD0006364656600000000282725732729000038
:101FE0007B6D6F64756C652325647D007B6D6F640C
:101FF000756C652D726F70653A25787D0000000064
:10200000222573222C2000006C696E652025643A1D
:102010002000000021490868C2430A600A680242A1
:10202000FAD170471E490A68002AFCD1CA610860CB
:10203000C8690028FCD00020C8614868704719486A
:1020400001686FF00202114041F400710160032148
:102050001548816041F2300141610121C160502188
:1020600041610121C1604FF4CA6141610121C16038
:10207000016070470D4802680A6082684A60C26861
:102080008A60406B20F0784040F08050C860704714
:10209000704701461022064800F024B81010044092
:1020A0000010044000000460004104404C13005044
:1020B000180000217047FF7F0948016842680368E3
:1020C0009942FAD1100C40EA0140704710B5044A19
:1020D000136850681468A3421946F9D110BD000076
:1020E0000820094062B38B0708D0521E11F8013B4B
:1020F00000F8013B00F024808B07F6D1830740F005
:10210000208000BF103A07D330B4B1E83810103A3D
:10211000A0E83810F9D230BC530724BFB1E808104A
:10212000A0E8081044BF51F8043B40F8043BD20734
:1021300024BF31F8022B20F8022B44BF0B78037028
:102140007047083A07D3B1E80810083A40F8043B52
:1021500040F804CBF7D25307E4E70040DFF800F083
:10216000F5C00110DFF800F049BA011020B10823D2
:1021700024220021FEF74ABA704780B50120009062
:1021800009234FF400720021DFF8080700F07BFFFD
:1021900001BD80B5002301223421DFF8F80600F0EC
:1021A00085FF00B10120C0B202BDDFF8EC068068F7
:1021B0007047DFF8E416401890F8ED0070470022F1
:1021C000022904D1012806D140F2EE2203E00128C1
:1021D00008BF4FF47A7210467047DFF8BC06D0F89B
:1021E000DC007047DFF8B00690F8E61021B1D0F8B7
:1021F0000C01010018BF004770472DE9F041DFF8DE
:10220000988608F1E1058AB0A879002861D10120FB
:10221000A871DFF88866DFF88876307B68717068AF
:10222000C8F80C0101A8FFF7A1FF00200690ADF847
:102230001400079001AB00220FF2F54108F10C00E9
:10224000FEF70CFA01AB00220FF2A15108F13000A9
:10225000FEF704FA01AB00220FF2D94108F1540055
:10226000FEF7FCF9B16801208847DFF838060078EE
:102270007868C0F38154707B20B1032C02D1012017
:10228000287003E0032C18BF022C16D1022000F0A6
:102290009DF8032CDFF810160CBF4FF47A7042F251
:1022A00010700968B0FBF1F108F15400FEF7B2F9C3
:1022B00008F15400FEF7B2F905E0012C03D100F05B
:1022C00063FAFFF75AFF386840075CBF002000F050
:1022D0007DF80AB0BDE8F08110B508B1140001D155
:1022E000022010BD8160C26003610146DFF8A805CD
:1022F00000F0F6FE002010BD10B50446FEF776F99A
:10230000DFF89415621892F8E8305B1E82F8E83026
:10231000DBB223B98A680123A3409A438A6066E04E
:102320002DE9F0410546FEF761F98046DFF86815B2
:10233000681890F8ED20521E80F8ED20D2B2002AE5
:102340003FD10FF2A050DFF8644500EB85052E78F1
:102350006F88300615D52168096A38468847216894
:10236000896A384688472168096B38468847DFF80C
:10237000401501200860DFF83C0500688007FAD5A9
:1023800012E0700606D501EB87010020D1F800119C
:10239000884709E021688969384688472168496B80
:1023A000384688470228F9D106F03F003F2818BF79
:1023B000FFF7B6FF687800F03F003F2818BFFFF72F
:1023C000AFFF4046BDE8F041FEF714B910B5044632
:1023D000FEF70CF9DFF8C0148A680123A3401A4302
:1023E0008A60611891F8E820521C81F8E820BDE865
:1023F0001040FEF7FFB8F8B50646FEF7F7F80446BA
:10240000DFF89454701990F8ED104A1C002980F8F8
:10241000ED2039D10FF2CC4000EB8607387800F080
:102420003F003F2818BFFFF7E6FF787800F03F0035
:102430003F2818BFFFF7DFFF7E883878DFF86C741D
:1024400001060ED53968C969304688473968496A36
:10245000304688473968C96A3046884700F019F81D
:1024600012E0400606D505EB86010120D1F80011E7
:10247000884709E039684969304688473968496BB7
:10248000304688470128F9D12046BDE8F240FEF7E2
:10249000B1B8DFF81C1401200860DFF818040068E8
:1024A0008007FAD570472DE9F04F002483B04FF034
:1024B000000A0128D04618BF012664D1DFF8D8935E
:1024C000D9F8DC0001285DD10220C9F8DC00FFF753
:1024D00045FE0090012000F062F9060054D1FEF79D
:1024E000C1F8DFF8D81301900C60012000F042FA27
:1024F000012804D1002000F0A7F94FF0010ADFF80D
:10250000C013DFF8B4030C6000681120FFF751FE20
:1025100008B14FF001081020FFF74BFE08B148F05A
:1025200002080F20FFF745FE08B148F004080B2011
:10253000FFF73FFEDFF8746320B13168096B4FF499
:10254000806088470A20FFF734FE20B13168096BAC
:102550004FF481608847DFF85813DFF86873DFF8BD
:1025600068B30120086048F0200031688969884715
:10257000DFF858130120086099F80800C00707D554
:10258000012416E0042673E00120C9F8DC006CE0A9
:10259000584600F0C7FD0546042DF9D0012D04D1A1
:1025A000326A526803215846904738688008800094
:1025B0003860002000F0C2FDBF4800683068806BC2
:1025C000804754B9012D04D1326A5268012158461E
:1025D0009047386840F0030038600120B84908602F
:1025E00040463168496988470B20FFF7E2FD20B17A
:1025F0003168C96A4FF4806088470A20FFF7D9FD27
:1026000020B13168C96A4FF481608847A849012028
:1026100008600020AD4908600320C9F8DC0031687B
:10262000496B404688470128F9D1042000F0B7F8EB
:10263000A24901200860A0480068A54800688006FB
:10264000FBD5BAF1000F1CBF012000F0FDF800F02F
:10265000C1FE082000F0A3F806460120C9F8DC00FE
:102660000198FEF703F800F039FE0098FFF77AFDB5
:102670003046BDE8FE8F38B50446FDF7B7FF054686
:102680002146854800F040FD28464BE030B5002447
:1026900001288BB004D021D303281DD018D31DE00E
:1026A00001A8FFF763FD7C4D8A490694ADF81440FC
:1026B000079401AB012205F17800FDF7CFFF0094EC
:1026C0000023854A2C2105F19C00FDF7B7FF05E0AA
:1026D00000F09CFE044601E000F03EFF20460BB0F7
:1026E00030BD00F054B938B5FDF780FF05466A48A3
:1026F00090F8E000012410B1FFF74BFD0446284696
:10270000FDF778FF204632BD38B5FDF76FFF624D0B
:10271000044695F8E00020B100F080F9002085F82B
:10272000E0002046BDE83240FDF764BF0000000035
:102730007047000010B582B0042000F01BF9022899
:1027400018BF032807D100F01FF8FFF716FDBDE8FA
:1027500016400220D0E56148534900684E4CC0F352
:10276000815003280CBF4FF47A7041F28830096819
:10277000B0FBF1F104F15400FDF74CFF04F15400FB
:10278000BDE81640FDF74ABF032000901C234FF020
:10279000405200213F4800F076BC0020704770B5E1
:1027A00004463D4E304600F091FC002598B9304675
:1027B00000F092FC0646B068204207D03269F36808
:1027C0000021204698470546012D05D0304600F0EF
:1027D00085FC0600EFD1284670BD414901280CBF99
:1027E00040F2FF70002008600020704770B5FDF7D0
:1027F000FDFE294E294D044696F8E00028B100F070
:102800000DF968B1002086F8E0000220AD68A84705
:1028100006461020FFF7C3FF8EB10320A8470EE045
:10282000214909683220B0FBF1F101B9012106F11B
:102830003000FDF7EFFE06F13000FDF7EFFE204619
:10284000BDE87040FDF7D6BE38B501281ED100F0B6
:1028500091F801281CD000F0D7F80F4C1249012044
:1028600084F8E00032200968B0FBF1F505B90125D4
:1028700004F13000FEF7D9FF294604F13000FDF7DE
:10288000C9FE04F13000FDF7C9FE01E000F0E8F8F0
:10289000002032BD00A00C40EC0C0020F4880000A9
:1028A000B03F0050A32600209C8F0000B80100100C
:1028B00028200860282008402C2009400C400940AE
:1028C00000022243242208400040034080010443C8
:1028D000141009409536000065340000B43F0050E4
:1028E000000004608F3F00008F3F01008F3F020017
:1028F0008F3F0300903F00018F3F0101903F000296
:10290000903F00038F3F01048F3F00058F120804A2
:102910008F3F00048F3F0006513F00007F3F0100C2
:102920003F3F04003F3F02003F3F01007F3F020066
:1029300070B50446E00782B00D46624E05D5A8B2D8
:1029400000900023012200F011F8A00705D5A8B2DD
:1029500000900123022200F009F8600705D5ADB20E
:10296000009502230C2200F001F873BD00213046CF
:1029700000F089BB0146042907BF1D234FF0C04268
:102980001C234FF080524F48342100F08FBB38B5E4
:102990000546FFF791FB4C4CA168401A4FF47A7141
:1029A000484305EB104500F04BFF2169401A48BF32
:1029B000404240F6B9318D4207D2062805DAA068B8
:1029C000E168814201D322685AB940494A68D20776
:1029D0004FF4FA6017D4086800F0FF007D214843E7
:1029E00008E0081A3A494843000C00EB9000904276
:1029F00038BF1046C82801D2C82032BDB0F57A6F62
:102A000088BF4FF47A6032BD80B501210320FFF703
:102A10008FFFFFF751FB2C49886001BD80B5012075
:102A2000FFF7A8FF012819D00023012234212548EF
:102A300000F03CFB98B100F026F8FFF73DFB22497F
:102A40008B680A68C860A2EB9202C01A204B5843F8
:102A5000000C0860904238BF10460860012002BD9B
:102A600010B500210320FFF763FF0120FFF782FF6D
:102A700008B100F008F8144CFFF71EFB606000F08E
:102A8000DFFE206110BD1348006800F0EDBE10B5F8
:102A900011490A6811490968140424161B38444373
:102AA000E41004EB2244120600FB00F312160906A0
:102AB0005A435843091604EBA222484302EBA040B4
:102AC00010BD000000A00C4080260020AC3F00504C
:102AD00040420F008000001090130050A4100050DE
:102AE000002200F0DDBE000010B54048046814F17B
:102AF000010F08BF002400F055FF3D490020086089
:102B000001203C4908603C49086001F01BF93B4842
:102B1000006820B13A480068204600F01CF83949A6
:102B2000394A00200860394801686FF31B4111439E
:102B3000016037480168C1F30131012906D10168FC
:102B4000344A114041F400320260016032480068AA
:102B50000028FBD110BD70B5054630480121016049
:102B60002F4909680029FBD02E4C2F4AC021216033
:102B700053682E499B075DBF13681B0C43F0F0039D
:102B800072230B70002101639668304600F014FF39
:102B90003146284600F043FF2548816D89B240F256
:102BA0000F22914213D201680068C1F30361C0F3A0
:102BB000034001B1491E072805D006280EBF072093
:102BC000801C00F00F0041EA00101A4908703046DE
:102BD00000F094FF18490968C9680220884740201E
:102BE000206001201549086070BD00001C130050D2
:102BF000840460425C600C40082204438001284346
:102C0000000120438C210840000039014820034086
:102C100004000940FFFFFCFC0C0068421010094052
:102C20009402224300600C40AC3F005056620840C2
:102C3000BC12005002600840A001001094046042E1
:102C40001B4213D1094236D12AB18446B0FBF2F0BF
:102C500002FB10C2704701F0E5B8FCD3002200234C
:102C600070470B000200002100207047904271EB7A
:102C7000030CF6D370B5B1FA81F4B3FA83F52C1BCB
:102C8000A340C4F1200532FA05F63343A2405FF0B9
:102C90000046E64002E05B085FEA3202841A71EB0C
:102CA000030524BF204629467641F4D302000B00D9
:102CB0003000002170BD012ACFD970B5140C20D08E
:102CC000B1FA81F4B2FA82F5C4F120046419B4F1C6
:102CD0002006D6D3B2405FF00044F440002502E065
:102CE00052085FEA3303C61A71EB020E24BF304666
:102CF000714664416D41F3D302000B0020002900AE
:102D000070BD0C46B1FBF2F102FB11452D0445EA02
:102D10001045B5FBF2F402FB145580B240EA0545BC
:102D2000B5FBF2F002FB105240EA044070BD000017
:102D300000F10103810704D010F8011B89B181075C
:102D4000FAD10268B2F10131914311F0803F04BF22
:102D500050F8042FF6E710F8011B11B110F8011B11
:102D6000FBE7C01A70470000DFF800F00DC3011048
:102D7000DFF800F081C60110DFF800F095B7011010
:102D8000DFF800F08DC20110DFF800F03DC2011045
:102D9000DFF800F009C30110DFF800F045C00110B2
:102DA000DFF800F0D1C70110DFF800F067BE0110B6
:102DB000DFF800F011C80110DFF800F021C80110A1
:102DC0000C381F283ED8DFE800F0103D3D3D3D3D6A
:102DD0003D3D3D3D3D3D3D153D3D3D1A3D3D1F24A5
:102DE0003D3D3D293D3D3D2E3338DFF8F40100687F
:102DF00000687047DFF8E801006840687047DFF856
:102E0000E001006880687047DFF8D4010068C0689E
:102E10007047DFF8CC01006800697047DFF8C00137
:102E2000006840697047DFF8B80100688069704742
:102E3000DFF8AC010068C0697047DFF8A4010068E2
:102E4000006A70470020704700B589B009216846C4
:102E5000FFF78AFF09B000BD00B581B0FEF730FD75
:102E6000DFF88001DFF880110068884218BF00F0A9
:102E70009BF8DFF87801B0F5B26F03D001B05DF8D0
:102E800004EB92E001B000BD2DE9F04184B01D4695
:102E90000B6880461446002226681F78002003F144
:102EA000010C242FC1F800C038D15F780CF1010368
:102EB0004C2F0B6006D156F8040BAA684146FEF76A
:102EC000B5FF25E0462F0DD156F8041B0191414670
:102ED00056F8040BADF8002002906846AA68FEF789
:102EE000FEFF15E0532F19D156F8040BE861266058
:102EF0002346288B0090EA69A968D8F80000FEF7FD
:102F0000DFFDD8F8001011B10144C8F800102668A0
:102F10000021E96001222968091A2960662F08D179
:102F2000298B002911BF361DF11D21F0070101F188
:102F300008061AB9E9690F700121E960266004B03A
:102F4000BDE8F0814FF0FF309060704700B581B070
:102F5000FEF7A4FD012818BFFEF704FC0FF21D00C8
:102F6000FFF706FFFFF708FFFFF70AFFFFF70CFF69
:102F700001B05DF804EBFFF70BBF000000B581B0B6
:102F8000FDF770FBFFF7EAF801B05DF804EB0320F2
:102F9000FFF702BF10B504460320FFF7FDFE2046F1
:102FA000BDE81040FFF7FCBEFEE7FEE700B581B0CC
:102FB000FFF7FAFEDFF83800C06801B05DF804EBF7
:102FC000FEF7C0BBDFF82C10DFF82C0088617047DB
:102FD000FFF7EEBEFFF7F0BEFEF707BFFEF708BF34
:102FE000F001002098CA01107047282090050000C9
:102FF00078010020440100200004000070B5044660
:103000000D46164600F0E2F9401E8041C00F1A49F5
:103010000A68002AFCD0012E02D0022E02D003E062
:10302000257002E0258000E0256001220A6000286A
:103030001CBFBDE8704000F0CDB970BD38B5044686
:103040000D4600F0C3F9401E8041C00F0A490A68CE
:10305000002AFCD0012D02D0022D02D003E02478FA
:1030600002E0248800E0246801220A6008B100F030
:10307000B1F9204632BD000000800C400B461146DD
:1030800004221818BAE710B500EB4100102B1446C3
:1030900000F5007002D3103B001D240C02999940EA
:1030A00041EA0441BDE810400422A7E738B51D46B7
:1030B0000818102D144602D3103D801C240C022148
:1030C000FFF7BCFF204080B2E84032BD0068002816
:1030D0000CBF0120002070470068704700687047EF
:1030E00038B504460D4600F09EFE00212960616857
:1030F00069606168002914BF0D6025606560FFE7A5
:10310000BDE8324000F091BE0B684A68002B0CBF4E
:1031100042605A604A680968002A0CBF0160116069
:1031200070470000006801074CBF042000F0030056
:10313000704700001628A8BF203870472DE9F84FC7
:1031400006469348934C0068934D800704D50820A9
:10315000A87192482060BFE000F072FB8046904862
:10316000006800900027001700F101090098800214
:1031700008D4C8F13E00C0100928A8BF0820814526
:10318000B8BF814687480068C0F30460FFF7D2FFEC
:10319000824685480068C0F30440FFF7CBFF09EB87
:1031A0000A011629A8BF152104DA6FF0090291421D
:1031B000B8BF114601F01F027C4B42F4F8521A804E
:1031C0007B4A126812F0030F18BF0127520748BF4D
:1031D00047F002070EB147F0040795F90720A8EB66
:1031E0000202052A02DAAA7997425DD0A8F10F0CF3
:1031F0000026BCF1000FB64607F0010207F00403F9
:10320000DFF8B09123D40CEB0C1C4FEA2C2EBEF14E
:10321000080F28BF4FF0070E7646072E28BF062658
:1032200009EB860A59F82660DAF804A0AAEB060A28
:103230000AF0FF0613B1CAF3072B5E445FEA877BEF
:1032400044BFCAF3074B5E440AB106EB1A6659F84D
:103250002E9009F0FF0A13B1C9F307239A44BB0764
:1032600044BFC9F307439A440AB10AEB196A401AEA
:10327000ACEB0E220099AF71724380320128B8BFC7
:103280000120342301F0FF0158430AEB1222484386
:10329000B0FBF2F0B0F5803F28BF4FF6FF7008F3A7
:1032A0000708A88085F8078043480068A988286037
:1032B00000201F2904D21F21A98004E04908401CD6
:1032C000B1F5007FFAD20F39090940EAC1003B4944
:1032D0000843206000206060BDE8F18F10B53848D9
:1032E000006884B21CB300F0ABFA2B4991F90720B7
:1032F000904205DA6FF07F029042B8BF1046C87165
:103300008888844201D28C8010BD2B4A12680B68D9
:10331000D21A921C202A28BF1F22231A5208D340F7
:103320001818B0F5803F28BF4FF6FF70888010BD99
:103330002448026802B9704710B5234B996801F020
:103340004060B0F1406F21D011480468A4071DD43B
:103350005C68A4071AD404681B68C3F303531C33C6
:103360001B0114F0050F06D09A420FD26FF0050131
:103370002140016010BD934208D20A0158BF44F0B9
:103380000104490158BF44F00404046010BD00006A
:10339000000009403010094094260020FDFDA400E3
:1033A000B43F0050B81200503C1100506E6208400B
:1033B000242208409C1300500820094000E7A48004
:1033C0003410094028500940AC3F0050EFF3108002
:1033D00072B67047EFF3108062B67047DFF800F006
:1033E00099C8011010B50C18FFF7F0FF401E80417E
:1033F000C00FDFF8F0130A68002AFCD0246801220D
:103400000A6008B1FFF7E6FF204610BD38B5DFF8C7
:10341000D843DFF8D8132078897B002508430AD0E9
:10342000FDF7E4F8A178002906BF0121A17001256C
:10343000FDF7E0F80DB1002032BD0220FEF7C6FF17
:103440000E20FEF7D8FFDFF8A803016809B10120BC
:1034500032BDDFF8A023402111600121C1610020AD
:10346000607032BD70B5DFF88C0382B0002101605E
:103470004821C160DFF8800300F1D804A17A002957
:1034800068D00129DFF8742329D110684BF2F521A7
:103490004843050ADFF868030068C0F3814001284B
:1034A00006D100F0CDF9FFF7F2FA684305EB90552D
:1034B000607B10B10020607305E0D2480068000214
:1034C00015EB10204508D0480560290C416001210A
:1034D0008160C648807B00283AD0052039E0022967
:1034E00009D11568284600F0FDF8A5F2FF50032821
:1034F0002ED308202DE003292CD1116800F1B80546
:10350000A1F5C0612868E961002848BF4042002950
:1035100048BF49428842A8BF002018DA6868BB4EFD
:1035200080B2009008234FF47F4230213046FFF7ED
:10353000AAFDA86800F072F904213046FFF7A3FD48
:10354000A86900F071F93046FFF79DFD0120207059
:103550000B202073BDE873402DE9F041A64CDFF845
:10356000AC82AB4FAB4EA34804F1E10582B0E978E1
:103570004A1E0B2A00F28080DFE802F00622334662
:103580005B33465B3346636EA349096809682020B4
:1035900088470F20F860072341F61D5038614FF42B
:1035A000C0720220009000F070F807234FF4C07240
:1035B00000214046FFF77AFD01203060022044E000
:1035C0000120F861287800281DBF00203061032009
:1035D0000620E87003203860002070607068800763
:1035E00034D4E878032804D1022000F04BF80420FA
:1035F00007E0002000F046F8E87806280CBF072016
:103600000A20E87001201AE0042903D12021B961C1
:10361000012105E00122BA610A290CBF0321022120
:103620006970002139600821C160016001203860A3
:1036300026E005290CBF06200920E87000207060F4
:1036400004E00020306070600C20E87004F1780025
:10365000BDE8F641FCF7E2BF0021016001206449AA
:1036600008600E20FEF75CFE0220FEF745FE0120FA
:10367000E8700020A87003E0BDE8F341FFF7AEBE9C
:10368000BDE8F38100900523602200214046FFF74A
:10369000FABC000080B558495E4891F8E410891ED4
:1036A0000A291AD8DFE801F0060A0E190A0E190ACB
:1036B0000E19120001688907FCD510E041688907DE
:1036C000FCD40CE041688907FCD508E00168890753
:1036D000FCD441688907FCD401E0FFF77FFEBDE818
:1036E000014039E7F8B50746484C30212046FFF73E
:1036F00079FE414E06F1B805C0F307206860042149
:103700002046FFF76FFEC0F38440A86020212046CA
:10371000FFF768FEC0F38120A861B7F5C06028609C
:1037200002D186F8D800F1BD296996F8D8202AB9C7
:103730006A68A968EA60E861AA696A61E8690028BC
:103740004CBF6FF00102022200EB40001018421043
:1037500000EB927001EBA0006968E960012810DAC3
:103760006A69032A04D1153001281DDA01201BE003
:103770000B300128B8BF0120491E48BF0021E96075
:1037800007E01F2812DB6A692AB915381F28A8BF6D
:103790001E20032109E00B381F28A8BF1E20491C4A
:1037A0004029A8BF3F21E960002169612861082301
:1037B000E86880B200904FF47F42302100F03CF87E
:1037C0000120009011234FF4003200F034F82869F2
:1037D00000F024F800F02FF8686900F025F800F0F8
:1037E0002BF8F1BD00800C40CD0D0020F4880000C6
:1037F00004800C402C500C40EC0C002008400C4085
:10380000B43F0050102009403C600C4000A00C4028
:1038100000400C4034600C40A001001080B20090C9
:1038200012234FF4F802704780B200900A234FF43D
:1038300040622021704704212046FFF724BC00008D
:103840000748084A81681278006852B2A0F54070B3
:10385000C9035043C913A1EB2010803000127047F8
:10386000285009400C13005070B50446FFF7AEFD18
:10387000451EAD41ED0F074E30680028FCD0A04733
:1038800001203060002D1CBFBDE87040FFF7A2BDD5
:1038900070BD000000800C4062F30F2262F31F42F3
:1038A00000B500BF130096469446103928BFA0E823
:1038B0000C50FAD85FEA417C28BF0CC048BF40F8E2
:1038C000042BC90728BF20F8022B48BF00F8012BA2
:1038D00000BD000030480068000C00F0070005281B
:1038E00028BF4FF0FF3070472C490A68C2F30F32EF
:1038F0004BF69A139A424FF0FF3006D10868000F3A
:103900000B280CBF0420002070474BF6BE118A42E2
:1039100001D1012070474BF641318A4201D1032089
:1039200070474BF620318A4208BF022070470000E2
:103930001A48F8B50068050F1948006800F0FF063E
:10394000802E28BF0026FFF7CFFF04284FF0FF345A
:1039500006F10A071DD8DFE800F003121A1A1B004F
:10396000012D12D0032D06D0072D06D0082D08BF3B
:1039700006F116040DE014240BE0152409E025B12E
:10398000022D08BF06F1140403E00A2401E005B982
:103990003C4660B2F2BD0000941200501813005073
:1039A000A010005080B5FFF79FFF20B9FFF7C0FFC0
:1039B000162800DB01BDFEE7DFF8E8130968C1F354
:1039C00004611629A8BF203901EB2071491C162972
:1039D000A8BF152104DA6FF009029142B8BF114661
:1039E00001F01F01DFF8C02341F4F8511180DFF826
:1039F000BC13096889074FBF40F040600021DFF821
:103A0000B0231160DFF8AC13C0F3C06282F0010292
:103A1000C0F380600A6080F001008860704770B574
:103A2000054682B0084600F0EEF80246DFF888430B
:103A3000182100F060F800F012F980B20090002325
:103A400040F2FF322C212046FFF71DFBDFF86C63AC
:103A5000F068C0F30D021C2100F04DF8706800F012
:103A6000FC32142100F047F83068DFF85413DFF817
:103A7000546301EA0002102100F03DF8284600F0EE
:103A8000F8F802460C2100F036F8284600F01CF940
:103A9000400040F020003072284600F01EF940F04F
:103AA00010003072284600F021F90246282100F06B
:103AB00022F8284600F0FFF8400040F06000F07265
:103AC000284600F02DF9C00040F0800030702846F4
:103AD00000F02FF98000BC4940F47C400880284663
:103AE00000F011F90246082100F005F8B7494FF43B
:103AF0008000086073BD2046FFF7C0BAF8B5810C9E
:103B000001F003010129B24CB04D02D002292AD0A4
:103B100026E0216A8A0323D44FF480422A606FF0A2
:103B20008F06AC4AD2F8023033404E0A06F08006C7
:103B30003343C1F303363343C2F80230C1F30326E3
:103B4000D2F801301B0946EA0313C2F801306FF0C6
:103B5000E7061368334001F0E7011943116002E002
:103B60004FF0004129609C4E9C4AB16809075CBF38
:103B70004021A9624FF400712964800D216AC90CAB
:103B800001F0030141F0300110F00300117003D087
:103B9000022826D008D326E001210420FEF7C8FE23
:103BA0008F4800F0F0F822E00120FEF7E3FE074620
:103BB00039460420FEF7BCFE0420FEF7DBFEB842C7
:103BC000FAD1366826F07F4000F0DDF8854B1B689F
:103BD0001B684FF060220721300E98474FF4806039
:103BE0002860032100E002210420FEF7A1FE2068E6
:103BF0007D4900F03F00087047F618007B490880B7
:103C00007B480068F1BD7B490968C1F38362830387
:103C1000C1F38F2120D4000400164FF6FF7307E094
:103C2000490804D11946520804BF01220121401C51
:103C30000028F5D401280FDB490041F00101B1F55E
:103C4000803F21BF0121520042F00102102A24BF0F
:103C50000F221946401EEDE741EA024070476548D1
:103C6000016800680002C1F3870100F44070084356
:103C7000704730B5604C61490A686568ED07C2F36A
:103C80000351C2F303430AD42468250501EB2571CF
:103C9000240481F3040103EB247383F304031B0462
:103CA00043EA015193B21943222824BF02F0804015
:103CB0000143084630BD0021202803D35048006846
:103CC000C0F30151084670470121222803D34D4813
:103CD0000068C0F30071084670470121222803D311
:103CE00048480068C0F3407108467047002120280A
:103CF00007D343480068C10C01F44071C0F38450FD
:103D000001430846704720283F4907D33C483F4AB3
:103D10000068810A02EA003040EA81510846704793
:103D20000021222803D337480068C0F3C061084649
:103D300070470021222803D332480068C0F3455160
:103D400008467047324800680028FBD13148324AA3
:103D5000416812688908890041F0005141F004016E
:103D6000520748BF41F001010BD4026812F0030F63
:103D700007D041F003024260026802F00302032A06
:103D8000FAD141607047254982B20A60C0F307400A
:103D9000486001208860224800680028FBD000208D
:103DA00088607047B81200506E62084000000940F9
:103DB00094042A430000204300A00C4070130050DC
:103DC000FFFFFC0041A10C40DCA10C4040A00C40D6
:103DD0006C1300500A600840A83F005008A10C4036
:103DE000BD378600B40100100BB00C4070B00C4021
:103DF0002C20094050130050AC3F00507813005065
:103E0000981300508C13005000803F4000F03F009A
:103E10000C00684200400340B03F00503C600C4042
:103E200084088C437047FCF7E1BBFCF7E3BB000060
:103E3000DFF800F0D9C10110DFF800F0ADB50110D6
:103E4000DFF800F019AE0110DFF800F0E5C1011055
:103E5000DFF800F085C20110DFF800F081C2011028
:103E6000DFF800F055C10110DFF800F043C2011087
:103E7000DFF800F079AB0110DFF800F0D9B60110DF
:103E8000DFF800F0EDB3011020B108232C2200214F
:103E900000F012BD704720B108233C220021FFF73B
:103EA000C7BF704780B5FEF759F9ADF80000FCF7C1
:103EB0009DFBADF80200009802BD01B5BDF80200FF
:103EC000FCF798FBBDF80000BDE80240FEF74AB9D8
:103ED00038B5DFF8A008DFF8A018DFF8A0488008A0
:103EE0008000091A2161E060034602E0002523F802
:103EF000025B0D18AB42F9D38B0800EB8303002261
:103F000023F8042CE82202804FF6FC721140EC39B1
:103F1000A0F8E810E8306060002000F004F8A0602D
:103F2000E068606031BDF8B500240025061D16F07C
:103F300003001CBF311D0E1AFFF7B4FFDFF83C2849
:103F4000B6B21060112EB4BF576897683A88130450
:103F500003D582F4004200251AE02B0014D02388F8
:103F600039880B4423809BB2B34211D327461A46AB
:103F7000B7B1921B92B2042AA7BFBA5346F40041CC
:103F8000398841F4004109E0B242F1DA01253C46AA
:103F900017443A88002ADAD1002701E027F8041BE9
:103FA000FFF78BFF3846F2BD10B50446FFF77AFFE6
:103FB000DFF8C817086034F8042CC2F30E0224F8A6
:103FC000042C221F4B689A4238BF4A60BDE810405B
:103FD00073E738B50446FFF765FF00210C23DFF8CF
:103FE000A0274B43D518AA6C4AB1944204D1FFF7DD
:103FF00064FF05F1480032BD491C0329EED3FFF7E9
:104000005CFF002032BD70B50546FFF74BFF04464C
:1040100000200C22DFF8681742438E18B16C49B9B2
:1040200000203065B5640022FFF706FFF06418B980
:1040300000F04CFC8D4205D12046FFF73EFF06F113
:10404000480070BD401C0328E3D32046FFF735FF2E
:10405000002070BD38B50446FFF724FF0025DFF8C7
:1040600020170C226A438A5A130008D0944203D1C5
:10407000FFF723FFE8B232BD6D1C062DF1D3FFF729
:104080001CFFFF2032BD10B504462088FFF7E2FF79
:10409000FF2800D16BE10C22DFF8E41650430844FE
:1040A0008168080002D16FF0010010BD2046BDE814
:1040B0001040084702460FF23870104710B5002034
:1040C0000C21DFF8BC26002401FB00F31344401C44
:1040D00003289C641C65F7D30020002301FB00F437
:1040E000401C13530628F9D3082010800FF2E96012
:1040F0009060BDE81040EBE670B590B0FEF72EF88A
:1041000004466846FFF7C7FE05200690002240F2ED
:10411000B630089069464FF6C1500490DFF8640647
:104120000590DFF86406FFF78BFE050006D0FFF769
:10413000B9FE06462846FFF766FF08B900F0C6FB41
:104140003046FFF7BAFE2046FEF70CF810B070BDFF
:10415000F8B500F0E6F8FFF756FF05006FF002062D
:1041600016D0FFF79FFEA28800210C27DFF810363B
:104170004F433B441F883FB91A805D60A2689A6034
:10418000217369682161C4E2BA4203D1FFF795FE49
:104190003046F2BD491C0629E7D300F097FB00BF6B
:1041A00038B500F0BEF8FFF72EFF050016D0FFF778
:1041B00079FE00210C23DFF8C8254B431A441388ED
:1041C0004BB94FF6F873138055600023936021714B
:1041D0006968A16013E7491C0629EBD300F076FB60
:1041E00000BF10B5044660680C3080B2FFF79BFE3C
:1041F00000B91AE06168018100210160FF2181722C
:104200000C30A060002010BD80B540680C3811E073
:1042100080B288E610B50446606880B2FFF783FE7E
:10422000A06000B901E0002010BD6FF0030010BDD8
:1042300080B54068FFF7B8FE002002BD38B50446DF
:104240000D46FFF72FFE002145F80C1C216811B91F
:10425000256006E0114651F80C2C002AFAD141F8ED
:104260000C5CBDE8324028E62DE9F04104466FF0D1
:104270000206E068A0F10C05A0790628BCBF2079F1
:1042800006280BDAFFF70EFEA179DFF8F4840C277D
:1042900079434144496819B9FFF70FFE304617E0EA
:1042A000FFF70BFE20792871A0796871207AA87138
:1042B000A079E1687843404440680830FFF7BEFFCA
:1042C000A0797843404440684068FCF797F90020A3
:1042D000BDE8F08170B500F024F8FFF77AFE060023
:1042E00002D16FF0040070BDFFF7DCFDB16800255E
:1042F00041B10D46A5F10C010A68B26000220A60C6
:10430000FF228A72FFF7D9FD2800A56001D10220A3
:1043100070BDA5F10C00017921714079A0710020D8
:1043200070BD0446FFF790BD06280ADA0C23DFF8BB
:1043300050245843105A02001CBF4FF6F8729042A6
:1043400002D14FF0FF307047088000207047811D78
:104350000079E9E710B50446E088FFF77BFEFF2807
:1043600000D104E0A0712046BDE810407CE74FF08A
:10437000FF3010BD3EB50446FFF7ACFF050017D176
:1043800020796946FFF7D0FF78B10820ADF8040026
:104390000320ADF80600DFF8F413A06889680290E6
:1043A00001A888476FF005003EBDBDF80000A08061
:1043B00028463EBD10B5DFF8D82312680C464FF4EE
:1043C0007A71A1FB00010023FEF73AFC0023994219
:1043D0004FF0004201D8904202D36FF0020010BDAE
:1043E0002060002010BD38B5FFF79BFFFFF7F1FDFF
:1043F0000546FDF7B8F9002818BF012800D015B907
:104400006FF0040032BD606840B9009000996868A0
:10441000FCF7F8F8401E8041C00F32BD10F1010FCB
:1044200008BF4FF0FF30F0D06946FFF7C3FF002808
:10443000ECD032BD80B54068FCF7E0F8002002BD4A
:1044400000F044FA00BF80B54068FFF701FD00208E
:1044500002BD80B54068FFF7FFFC002002BD80B5BB
:10446000FFF7FEFCFFF700FD002002BD80B5FDF761
:1044700075FEFCF7BBF8002002BD10B58CB00446F9
:104480006846FFF701FDE02000F013F808B900F0DE
:104490001DFA0BE010B58CB004466846FFF7F4FC3B
:1044A000E06800F006F808B900F010FA00200CB03F
:1044B00010BD08900023A16860686A46FFF7D8BC69
:1044C00010B50446FFF7D8FC6060002010BD01461F
:1044D000886849680847F0B507468BB0BC68AB4DA3
:1044E0006CBB0C20FFF71FFD04006FF003061ED00D
:1044F00008232422002101A8FCF788F80020ADF849
:1045000014000690079400237968A24801AAFFF7D7
:10451000B7FC206068B90820ADF800000C20ADF8A9
:1045200002006846A96888472046FFF73DFD3046EF
:1045300018E0F86860603869A060BC600AE028682C
:10454000804706462068FDF770F93869A06030465C
:104550006968884779682068FCF75CF82068FCF790
:104560005DF800200BB0F0BD10B5044682B0606865
:104570006946FFF71FFF20B9009860602046FFF7EB
:10458000AAFF16BD80B5406810B96FF0020002BDE9
:104590000068FDF74AF9002002BD7D4909684160C5
:1045A0000020704750B50446794802686FF0004615
:1045B000A6FB020100234FF47A72FEF741FB0023B1
:1045C00099424FF0004201D8904200D330466060DB
:1045D000002050BD2DE9F04186B00646FFF734FCBF
:1045E000FFF7F7FC0446002002900025FDF7BBF81A
:1045F000002818BF012800D014B96FF0040063E050
:10460000706820B110F1010F03D14FF0FF3000901E
:1046100004E06946FFF7CEFE070054D1FFF72CFCFB
:104620000099012701EB000800E000900099606804
:10463000FBF7E8FF78B303A8FFF74CFE07001AD199
:104640009DF8100001A9FFF76FFE80B9059A9DF84B
:104650001210BDF80400B368984740B1BDF80400DB
:10466000B0819DF81200B0730598306113E0059990
:1046700002A8FFF7E3FD009801276D1C10F1010F60
:1046800018BF0028D2D0FFF7F7FBB8EB000002D02C
:1046900000998142C9D2029EFFF704FC56B131460F
:1046A00000E0114651F80C2C002AFAD1A26841F81A
:1046B0000C2CA660FFF701FC002D03E06068FBF7FF
:1046C0009DFF6D1EFAD1384606B0BDE8F081F8B501
:1046D000FFF727FE0546FDF746F8002818BF01281A
:1046E0006FF0040613D0FFF7DDFB0021244A0C23F2
:1046F0004B43D75A4FB113445B681B68AB4201D19F
:10470000217106E0491C0629F1D3FFF7D6FB30469C
:10471000F2BDFFF7D2FB0020F2BDF8B50446FDF76D
:1047200022F8002818BF012802D16FF00400F2BD62
:10473000FFF78AFB0546FFF7B5FB0021104A0C2363
:104740004B43D65A37000ED0A788BE4208D1D118A5
:1047500049680968A9420CBF01210021A160D8E77E
:10476000491C0629EBD3FFF7A8FB4FF0FF30F2BD41
:1047700000000000A8260020283F0020641E002022
:10478000F81D0020C0070020B5400000AC07002045
:104790009C8F0000CF44000070B504463C20FFF71A
:1047A000C2FB05006FF0030611D0FFF774FB207AFF
:1047B000A8610022608928622946E0682861606853
:1047C000FFF73EFB04462846FFF7EEFB0CB93046E8
:1047D00070BD002070BD000041882D2902D36FF00C
:1047E000010070470FF2140252F821100847000030
:1047F00087400000A53E0000BB3E00005141000084
:10480000A1410000E3410000094200001542000000
:104810003142000069420000D542000055430000CB
:1048200075430000E74300003544000041440000A8
:1048300047440000534400005F4400006D44000002
:104840007B440000C1440000694500009B45000016
:10485000A54500004F430000CF850000A38600005F
:10486000D5450000CF460000D74400008545000034
:104870003D86000075860000898600001B47000009
:10488000D5860000ED86000099470000000000007A
:1048900000000000E3860000FB8600009544000055
:1048A0000000000000000000000000000000000008
:1048B000DFF800F0F1C5011001B90149FFF7F8BFB9
:1048C000A0010000DFF800F0ED8C01100120FFF7DF
:1048D000F9BF0000DFF800F025B101102DE9F04E1E
:1048E000DFF8BC799246002640F2013B0C46BA78CC
:1048F0007B7997F804C097F80190B0EB0B0540F670
:104900007B4132D06D1E38D06D1E3DD0AD1E41D0E2
:104910006D1E00F07A806D1E00F07D806D1E00F02F
:1049200087806D1E00F094806D1E00F099806D1ED2
:1049300000F09E806D1E00F0A5806D1E00F0AA8024
:10494000ED1E00F0AF806D1E00F0B4806D1E00F013
:10495000B9806D1E00F0BE806D1E00F0C3806D1F1B
:1049600000F0CB80AD1E2DD0E1E0102C40F0DD80BA
:104970001022514607F1A40081E0102C69D11022C9
:10498000514607F1B4007AE0042C62D1DAF8000055
:10499000F862D7E0012C5CD1012B34D09AF80000EA
:1049A0003871BCF1000F06D00028F2D1022A19D0CC
:1049B000052AEED116E00028EBD0012A1FD0042AE8
:1049C0001BD11CE0012C44D1BCF1010F1BD09AF883
:1049D0000000787153B1002807D1032A1CBF072AB1
:1049E000052A02D1484600F0D8FEABE00028FCD0F2
:1049F000012A1CBF042A062A01D0052A02D101205F
:104A000000F047FC9EE012269CE0022C21D1BAF86F
:104A10000000F88396E0202C0BDA07F1CC0600F0BA
:104A200094F800F09AF8BC713346224601210BE05D
:104A3000202C7ADA07F1EC0600F087F800F08DF808
:104A4000FC71334622460021484600F088FE76E09D
:104A5000012C6AD19AF80000052866DA387271E0F4
:104A6000012C62D19AF8000004285EDA787269E0BD
:104A7000062C5AD14FF48670062251463844FDF771
:104A800031FB5FE0012C50D19AF8000008284CDA85
:104A9000B87257E0012C48D19AF80000042844DA93
:104AA000F8724FE0012C40D19AF8000006283CDA59
:104AB000387447E000F04DF837D1821F8A4234D273
:104AC00078823FE000F045F82FD1821F8A422CD235
:104AD000B88237E000F03DF827D1B0F5FA7F24DA4C
:104AE000F8822FE000F035F81FD1A0F10A0140F65E
:104AF0007742914219D2388324E0012C04BF9AF8FE
:104B00000000012811D107F1800001F004F950B92B
:104B100007F1100100F070FB060013D107F15C00F3
:104B200001F000F90EE016260CE018260AE028280D
:104B300007DA022C05D1BAF8001000F041FE064653
:104B400000E002263046BDE8F08E1F21304601F01D
:104B50005DB9BAF80000022C704722465146304633
:104B6000FDF7C0BA38B500244FF440730D46C21AA1
:104B7000DFF82C1736D0521E36D0521E37D0521EB8
:104B800038D0521E39D0521E3AD0521E3CD0521E3E
:104B90003CD0521E3DD0521E3ED0521E3ED0521E20
:104BA0003ED0521E40D0521E40D0521E40D0921EC7
:104BB00040D0521E40D0521E40D0521E40D0521EF5
:104BC00040D0521E40D0521E46D0521E46D0521ED9
:104BD00046D0921E48D0521E14D0521E42D0521EB1
:104BE00044D046E0C87842E01022A43130E01022E0
:104BF000B4312DE0C86A286042E00622C43127E0C3
:104C0000087934E0487932E0C88B36E08A79CC31D3
:104C10001EE0CA79EC311BE0087A28E0487A26E0E9
:104C200006224FF4867012E0887A20E0C87A1EE0EF
:104C3000088C22E0087C20E0488A1EE0888A1CE07C
:104C4000C88A1AE0088B18E006224FF48A700144E3
:104C50002846FDF747FA13E0488C0EE0888C0CE0FC
:104C6000C88C0AE0087B02E0887800E0487B287066
:104C700006E0282803DA00F0BAFD288000E00224CC
:104C8000204632BD1CB5DFF81846A17881B900B1C5
:104C9000206304F12C00019004F1B400009004F1B1
:104CA000A403E1786078002200F010FD002016BD1A
:104CB000112016BDDFF8E8058178062918BF0729FD
:104CC00004D1018C4078132200F02ABD12207047D5
:104CD00000B58FB008233C2200216846FFF7A8F8F2
:104CE000DFF8C00500F15001079100234FF4DC719B
:104CF00008916A46032106910FF2D101FFF7EAFD00
:104D00000FB000BD70B584B000F019F90120DFF8D4
:104D10009815DFF88C4509680FF29155ADF802003F
:104D20000026684688479DF8040060700298A062DB
:104D30000020A0704FF6FF70208400F076FD2070F8
:104D4000002301200190002200200090294604F158
:104D5000380000F0A5FF022000F02FF804F15C00FD
:104D600000F09EFF042000F028F804F1800000F01D
:104D700097FF0420E07004F1A4020020002100232A
:104D800000252BC204F1B405103A4BC5E062207235
:104D90006072E1720720A0721021022000F016FF5D
:104DA000103D2A461021032000F010FF04F12C02D0
:104DB0000421042000F00AFF7FBD019000230020A1
:104DC000009000222946704700000000FEB5FFF762
:104DD00099FFDFF8CC54DFF8D04405F1800700F0EC
:104DE000AEF80A20ADF802004FF0FF30019068469F
:104DF0002168884700284BD100F0A1F80920ADF8C0
:104E000002006846216888479DF80610029E002827
:104E10003ED1BDF80400102804BF687881422DD12E
:104E200030884FF6FF71884209D17088400425D53B
:104E300005F12C020421042000F0DDFE1EE0307894
:104E4000A22805D0D02804BF304600F07CF815E039
:104E50007079132812D13089012804BFA87B022859
:104E600005D1384600F05EFFFFF724FF06E005207D
:104E700000F0BDFC0146384600F038FF46B100F0B6
:104E80005EF80320ADF80200019668462168884765
:104E9000A88BC10730D54FF6FE710840A883297949
:104EA0006879014328D018B103208DF800000DE087
:104EB000287A8DF800000622687A8DF801004FF4F8
:104EC000867029180DF10200FDF70CF9A87A8DF80B
:104ED00008006946E87A8DF80900687800F03BFC24
:104EE00000281FBF0820A870286B002804D0016884
:104EF00008001CBF08208847A88B810708D54FF6FB
:104F0000FD710840A88305F11001002000F074F93C
:104F1000A88B41070AD54FF6FB710840A883A87BF0
:104F2000012804D0022808BFFFF7C4FE57E700900D
:104F30002B8BEA8AA98A688A00F093F94FE7082048
:104F4000ADF800007047FEB5D54DA9784FF48A73CF
:104F50000446EE18A2786879130005F1800715D091
:104F6000022A3CD0032A18BF042A5CD0052A00F08C
:104F70007F80062A00F0AC80072A00F0CD800F2A3F
:104F800000F0E580112A00F0E780F7BD60780100AD
:104F90001AD105F1A4021021022000F02CFE05F127
:104FA000B4021021032000F026FE0622E11C05F1C8
:104FB000C400FDF797F80120A87005F1CC03AA7989
:104FC0006878012100F0CBFB08B10820A870286B9D
:104FD00020B1016808001CBFA8788847F7BD627837
:104FE000EAB9E27842B1EA79687805F1EC03002188
:104FF00000F0B5FB607012E0022918BF07290ED03F
:10500000062902D101280AD101E0032907D005F1C0
:10501000380000F080FE10B9012000F03AF9607805
:105020000028DBD0D1E763780BBB2B79032A08D1AA
:10503000062908BF0720C9D0002B0CBF032002207F
:10504000C4E7E98B0A0006D018430AD005F13800FE
:1050500000F04CFE05E0012B07BF00202871002066
:105060006871A878072814BF04200620AEE7ACE7D3
:105070006078010026D10622211D3046FDF732F866
:10508000608928840620A870E0896884208AA88422
:10509000608AE884E0782873287C012818BF0228F9
:1050A00009D11F2000F0A3FB4FF47A71414305F1B1
:1050B0005C0000F01BFE6289E0780423211D00F0F3
:1050C0000DFA84E73128D2D10020287104207DE731
:1050D000A08800F01AFA0621FFF738FD0020688446
:1050E000A884E884A079687305F15C0000F01AFEDA
:1050F000384600F017FE4FF6FF702884687908B133
:10510000032063E7A07908280CBF05200420A870BD
:10511000012000F0BEF85AE7384600F003FE607840
:10512000002813D1E08868842089A8846089E884F5
:1051300005F15C0000F0EFFD002807D16B6B002B40
:1051400004D0EA8CA98C688C1B689847F7BDA088AE
:10515000052100F027FBF7BDA088ADF80000287CF2
:10516000052803D100208DF80A0041E001208DF8C8
:105170000A0005F15C0000F0D5FD287C012818BF6D
:1051800004281AD1688AE188814228BF0846ADF810
:105190000200A98A2089884238BF0846ADF8040079
:1051A000E98A6089884238BF0846ADF80600298B35
:1051B000A08988421AD2084618E0032818BF02289E
:1051C0000AD1688AADF80200A88AADF80400E88A1E
:1051D000ADF80600288B09E0E088ADF802002089D0
:1051E000ADF804006089ADF80600A089ADF80800AC
:1051F000684600F091FAF7BDFEB50F46284D7A8853
:105200000446688C904224BFB988814207D3A88C99
:10521000F988884202BFE88C398988421ED005206F
:1052200000F0E5FA0646288CADF800007888ADF865
:105230000200B888ADF80400F888ADF80600388997
:10524000ADF80800684600F062FA070007D1AC73B9
:10525000314605F1800000F049FD00E0182738468E
:10526000FEBD3EB50E4CA578062D01D014203EBDE6
:10527000ADF80200ADF80410ADF80620ADF8083026
:1052800004F15C0000F04EFD06986946FFF7B4FF9C
:105290003EBD03498A8B10438883886AFBF7AEB909
:1052A000F0070020801E0020B4070020F1E7000076
:1052B000E0B50821ADF800100190022100F00FF8D0
:1052C00008B100200EBD02980EBD00B583B00821C4
:1052D000ADF800100190032100F001F807BDADF812
:1052E00002106846DFF87413096808471FB5ADF867
:1052F00006108DF804000824DFF860138DF80820EC
:105300000393ADF80040ADF802406846096888474D
:1053100004B010BD30B585B0144608220291ADF836
:1053200000201922DFF8341309680190ADF802203B
:105330001D466846884714B1BDF80C10218015B190
:105340009DF80E102970089A0499116005B030BDBF
:1053500000B583B00820ADF800001A2000F015F861
:1053600010B99DF804000EBDFF200EBD00B583B03E
:10537000ADF800008DF80610002000F006F810B916
:105380009DF807000EBDFF200EBDDFF8D0120968A2
:10539000ADF802006846084750B110F1040F01D182
:1053A0000420704710F1030F01D102207047012043
:1053B00070478123037042EAC111002341F47C410C
:1053C000C370818070478223037081800023C37083
:1053D000827170473EB504460820ADF800000D46C6
:1053E0002020ADF802001020DFF870120968ADF837
:1053F00004006846884720B9029810B16FF0040095
:105400003EBD00950023002221464FF0FF30FFF7FC
:1054100081FF3EBD10B582B01446CA78012A03D17F
:105420008A88DFF844351A8000F010F858B90090E7
:1054300069462046FFF7CEFF28B900984478FFF769
:1054400044FF204616BDFFF7A7FF16BD0B460222FC
:1054500010214BE738B51C461546FFF7F7FFC0B9DA
:10546000009069462846FFF7B5FF90B90098457847
:10547000280002BF0098C079A04205D10098816839
:1054800004982246FCF72EFE0098FFF71EFF2846E0
:1054900032BDFFF781FF32BDF8B500F084FA00F0AD
:1054A000C1F907000DD032462946FFF78CFF00F006
:1054B0004EF93872FFF74CFF3B4601B0BDE8F040B3
:1054C0005FE0F1BD10220121E6E738B500F00FFAE8
:1054D000050002D0042201214AE031BD2DE9F0414E
:1054E00000F064F907000FD0142200F019F83C72A4
:1054F000FD603E8287F81280FFF72AFF3946BDE83B
:10550000F041DFF8682485E725E038B500F02BF896
:10551000050004D0152200F003F82C812BE031BDEA
:10552000012150E70022042183E02DE9F04100F041
:105530003DF907000FD0022200F010F8BC60BD81D9
:10554000BE73C7F81080FFF703FF3946BDE8F0418E
:10555000DFF81C245EE70420BDE8F081042132E777
:105560001022022198E704460A20A1E602212AE738
:10557000FFF729FFAC60FFF7EBFE2B4601B0BDE85B
:10558000304002221021B1E6F8B500F0AAF9070078
:105590000AD01522FFF7EAFF00F045FB3946BDE8C7
:1055A000F840DFF8D02335E70420F2BD00220321C4
:1055B0003FE000B583B00FF2490301930623009347
:1055C000032300F04DF80EBD1078802802BF5088EC
:1055D00040F27F61884208D19088984202BF917959
:1055E0000098814201D1012070470020704710B51A
:1055F00082B00624FFE70094FFF7E6FF16BD000027
:105600000323F4E71078802802BF508840F27F61BE
:1056100088420CD19088032818BF042807D19079BC
:1056200001001CBF1028112801D101207047002063
:105630007047F8B500F057FA07000CD032462946FB
:10564000FFF7C1FEBC60FFF783FE3946BDE8F840B6
:10565000DFF82423DEE60420F2BD0000B4070020BA
:105660002DE9F04100F02BF807000AD0069A4146D8
:10567000FFF7A9FE3C817D8100F0D7FA079A00F080
:1056800075BA68E704460D460C2011E64246032130
:105690008FE670B582B000F086F9FFF759FE1B2146
:1056A0000091034632462946204600F02AF976BD8D
:1056B00010B582B01D24009400F023F916BD0446F5
:1056C0000D46164698461020FFF7F2BD2DE9F04131
:1056D00080460D4616461F461820FFF7E9FD0400D8
:1056E00014D0002200F069F800F068FA20726572A8
:1056F000A672E7600698206107986061FFF728FEB0
:105700002146BDE8F0410FF2153283E623E70FF2A0
:105710001133112200214AE10FF209331222F9E775
:10572000F8B500F0E8F807000FD00A2200F045F8BD
:1057300000F00DF838727D813E73FFF709FE39469F
:10574000BDE8F8400FF2E12264E60420F2BD2146F4
:105750005020FFF70BBE0FF2D523062238E12DE9CA
:10576000F04180460D4616461F461020FFF7A0FD6B
:10577000040011D0072200F020F800F01FFA207278
:105780006572A672E760FFF7E3FD2146BDE8F041D0
:105790000FF29D22FFF73EBEDDE60FF299230822AD
:1057A000002115E10FF291231022EBE004460D4693
:1057B000164698461420FFF77BBD0421FFF7F9BD7C
:1057C00070B5FFF75FFF06000BD03022FFF7F5FF43
:1057D00000F009F83146BDE870400FF26122FFF792
:1057E00019BE042070BD34817581FFF7B1BD30B59D
:1057F00083B004460020ADF8040000F013F8050063
:105800000DD03122FFF7D9FF2C81FFF7A1FD01A9AF
:10581000009102230FF229222946FFF71BFEBDF853
:1058200004003EBD0A20FFF743BD1CB500F077F928
:1058300004000AD01222FFF773FEFFF789FD00F083
:1058400005F80FF2012200F018F813E001A9009109
:10585000012370471CB500F062F904000AD0182239
:10586000FFF75EFEFFF774FDFFF7F0FF0FF2E512A2
:1058700000F003F89DF8040016BD2146FFF7EABDCD
:1058800070B500F014F806000BD01922FFF748FE9F
:1058900000F009F83146BDE870400FF2C112FFF781
:1058A000B9BD042070BD3481F560FFF751BD0446D9
:1058B0000D461020FFF7FCBCF8B500F012F8070009
:1058C0000DD03622FFF779FF3C817D8100F0ADF9E4
:1058D0003946BDE8F8400FF28D12FFF79BBD04205A
:1058E000F2BD04460D4616461020FFF7E1BC044603
:1058F0000C20FFF7DDBC04460D4616460E20FFF7D0
:10590000D7BC2DE9F041FFF751FF070011D0069AEF
:10591000FFF7BDFE3C813E74FD6000F04FF97874E6
:10592000FFF716FD3946BDE8F0410FF26D12FFF7A3
:1059300071BDFFF710BE38B51446104A15682A002D
:1059400006D0009302460B4621460120A84732BDEF
:10595000002032BD0A4A13681A0003D00A460146E5
:105960000120184770470000040E0020B95A0000BB
:10597000C95A0000BF5A000005560000781E0020DA
:105980007C1E00202DE9F04100F00DF898460C2017
:10599000FFF78EFC070004D000F016F83C81BD72C2
:1059A000E1E0FFF7D8BD04460D46164670472DE9E5
:1059B000F041FFF784FE070004D000F005F8BC605A
:1059C000FD60D0E0FFF7C7BD32460421FFF7F1BC10
:1059D0002DE9F041FFF773FE070006D0FFF7F4FF53
:1059E000FFF7B5FE3872FD60BDE0FFF7B4BD10787B
:1059F000802802BF508840F27F6188420CD1908895
:105A00004FF680710140B1F57E4F04BF00F07F007A
:105A1000984201D101207047002070470023E6E73B
:105A20001123E4E71223E2E70A23E0E70623DEE797
:105A30000723DCE70823DAE71023D8E73023D6E78B
:105A40003123D4E780B5122300930123FFF7BCFD77
:105A500002BD000080B51823F6E7000080B51923C9
:105A6000F2E700003623C2E71078802802BF508892
:105A700040F27F6188420DD190884FF680710140DD
:105A80004FF68052914204BF00F07F00984201D14E
:105A9000012070470020704770B5FFF784FF1D2379
:105AA000FFF7E2FF30B9324629462046BDE8704094
:105AB0001B23D9E7012070BD80B51423C4E780B54E
:105AC000152300930223C1E780B50223009304232A
:105AD000BCE70FF20D0142F22F000AE000000000C7
:105AE00042F22F0347E004460D4616460C20FFF70E
:105AF000DFBB70B504460D4600F014F806000CD06C
:105B000081203070B4800120F070FFF721FC2A461C
:105B10003146BDE87040FFF77DBC042070BD002019
:105B20008DF804000820FFF7C3BB2DE9F041FFF713
:105B30003AFF98460E20FFF7BBFB070009D000F0A4
:105B40000AF83D817E81A7F80C80FFF701FC069AD8
:105B50000CE0FFF700BD812038700120F870BC8098
:105B600070473D81FE60FFF7F3FB42463946BDE8D2
:105B7000F041FFF74FBC1078802802BF508840F2F8
:105B80007F61884204BF9088984201D1012070470C
:105B900000207047000038B50446154600F00FF8A5
:105BA0000FF221010091C2B22B4621464FF6184058
:105BB000FFF7BBFF32BD3C817D81BE814146502055
:105BC000FFF7D4BB4FF61843D5E70000F8B5FFF751
:105BD00088FE07000DD0012200F022F83C727D7291
:105BE00000F023F83946BDE8F8400FF27902FFF7DC
:105BF00011BC0420F2BDF8B5FFF773FE07000DD00D
:105C0000022200F00DF83C727D7200F00EF8394669
:105C1000BDE8F8400FF25102FFF7FCBB0420F2BDD3
:105C20000521FFF7C6BB3C81BD72FE60FFF790BB4C
:105C30001078802802BF508840F27F6188420DD1E1
:105C400090884FF6807101404FF68062914204BF08
:105C500000F07F00984201D101207047002070477A
:105C6000000000000123E3E70223E1E7DFF800F092
:105C7000F5B80110DFF800F02DBF0110DFF800F0DB
:105C800011BF011000B583B00821ADF800100190DC
:105C90000521ADF80210684654490968884707BDD8
:105CA000F0B589B004460D4616461F460823242247
:105CB00000216846FAF7AAFC0F984D49096806903A
:105CC0006B464FF47A70B0FBF1F101FB07F00590E1
:105CD00001FB06F20E98ADF8100029462046FAF7AF
:105CE000BDFC204609B0F0BDFAF798BC38B50446B3
:105CF0000D46FBF7A8FD10B12046FBF796FD00F01E
:105D000013F800FB05F12046FAF784FC2046BDE8B5
:105D10003240FAF783BC80B5FBF795FD00B1012056
:105D2000C0B202BDFBF781BD314909684FF47A70FA
:105D3000B0FBF1F0704710B504460021FFF796FF65
:105D4000204610BD70B584B004460820ADF80000B0
:105D50000D460420ADF802000C202449096801908A
:105D600016466846884758B9029949B18E60204660
:105D7000FFF780FF15B12846FAF740FC012003E049
:105D80003046FFF77FFF002004B070BD10B5044619
:105D9000FFF774FFA04204D08468FFF773FF20462A
:105DA00010BD002010BD30B585B0044668460FF226
:105DB00048011422FCF7A6F90E4830210170A21DFB
:105DC000782141700623811C12F8015D2D095B1EAC
:105DD0001DF8055001F8015B157805F00F051DF859
:105DE000055001F8015BEFD105B030BDB4070020CC
:105DF0009C8F000090250020303132333435363707
:105E0000383941424344454600000000002200F07A
:105E100001B80000401810F0030308D0C91A1FD3BE
:105E2000DB0748BF00F8012D28BF20F8022D130022
:105E300030B414461546103928BF20E93C00FAD882
:105E4000490728BF20E90C0048BF40F8042D89000D
:105E500028BF20F8022D48BF00F8012D30BC704744
:105E6000C91818BF00F8012DCB0728BF00F8012D75
:105E700070470000DFF800F061C20110DFF800F0A9
:105E8000E9C20110DFF800F0E1C20110DFF800F014
:105E9000F9BF01104068006800F204500068084033
:105EA00018BF0120C0B270474068006800F204507B
:105EB0000160704750F8041F21F002010160704733
:105EC00050F8142F01E050F8242F22EA010101605C
:105ED000704770B504460D46FAF788FB064695F8FC
:105EE000D80060B114F0704F03D114B10420FCF756
:105EF00003FA0220FCF700FA002085F8D8003046AB
:105F000027E070B54568846805F19C06706800F06C
:105F1000F8FB306800F022FE2068FFF7CBFF05F1A8
:105F20001C00FFF7A7FF05F13800FFF7A7FF207B54
:105F3000FCF7F6F9287818B905F16C00FFF7A2FF15
:105F400005F1C400FCF797FBFAF750FB002185F838
:105F5000D910BDE87040FAF74DBB2DE9F84346680B
:105F60008568DFF8CC8620294FF0FF3406F19C07C6
:105F700004D04DD3222913D00AD349E0307B012825
:105F800048D1387296F88D0048EA0001386834E04C
:105F90000020387296F88D0040F0004138682CE0FF
:105FA000307B92F80090012807BF49F0004141F48E
:105FB0000051DFF8800640EA09013868B9F1FF0FA7
:105FC0001ED000F07AFD28BB2868B0F1804F3868F9
:105FD0000CBF0B222322494600F036FE96F88D10A6
:105FE000386800F097FD307B86F88D9001280DD140
:105FF000387A58B1386848EA090100F0D3FD05E065
:1060000096F88D1000F086FD86F88D90002401E052
:106010006FF001042046BDE8F2832DE9F0434668A5
:1060200080680B880568DFF81046DFF810860FF2ED
:106030006C6906F18C02B5F1804F92F800C08D6852
:1060400003FA0CF30CBFC646A6469BB2A63655B162
:106050000FF2406757F82C70CEF808705D196D1E6E
:10606000CEF8045005E059F82C50CEF80850CEF880
:10607000046043F6F07C05680835CEF80050DEF881
:1060800008500F687F1E0CEA07173D43CEF80850F2
:106090000568B5F1804F4D680CBF08F1100410344D
:1060A00055B10FF2E85692F8009056F82960A660B4
:1060B0002B445B1E236006E0C3895383137859F891
:1060C0002330A3602660036808336360A36809680F
:1060D000491E0CEA01111943A16052695268016915
:1060E00043691268194342F8281F006850F8241FBA
:1060F00041F003010160BDE8F083F8B50546AC68E6
:1061000020686F6800F11C0100F12002096811602D
:1061100007F18806C90717D50121FFF7D1FE3068BE
:1061200018B12846BDE8F24052E12068FFF7C2FEF0
:1061300020680321FFF7C7FE2069616900F097F925
:106140002846BDE8F24033E06169B069FFF7A2FE7E
:1061500030B120680221FFF7B6FE616900F088F9CE
:106160002169B069FFF796FE60B120680121FFF751
:10617000AAFE216900F07CF907F13800BDE8F24081
:10618000FBF7E0BAF1BD70B5044600206568D5F8AC
:106190008860307429467068FFF79BFE0020C5F8C0
:1061A00088003146AA682046BDE870401047704715
:1061B0008068006800F10C0102E000F1080212683A
:1061C0000A685207F9D400F180020223136002E04A
:1061D00000F18C031B680B68DB07F9D50020106009
:1061E00070474068D83000214170017070472DE938
:1061F000F04180468EB0D8F80460D8F808700D469B
:10620000FAF7F4F996F8D91081BB012186F8D91074
:1062100006F18804FAF7EEF9002020602869306161
:1062200068697061287E3076287B307328783070FA
:106230006868706000202077686909288041C04341
:10624000C00F2071387BFCF7D6F8404600F032F9D9
:10625000F87E6071404600F055F958B9387BFCF77C
:106260005FF8FAF7C3F9002186F8D910FAF7C2F9F6
:10627000002052E008233022002101A8FAF7DAF9C1
:10628000CDF8188001AB7879DFF8B42309900020AD
:10629000009006F11C003979FAF7D0F9082328227A
:1062A000002101A8FAF7CEF9CDF814800023B868D0
:1062B000E449079001AA06F13800FAF7C7F93078E7
:1062C00088B908232422002101A8FAF7ABF901209C
:1062D0008DF81C0001AA002106F16C00FAF7A6F95E
:1062E0000FF2911000E0A868B06000F0E1F9A06141
:1062F000307B012808D160690FF2811100F067FC42
:10630000606908B1C0F8088043460FF25532042195
:1063100006F1C400FBF7E0FF40460EB0BDE8F08197
:106320002DE9F8430E46044630686568A7680028E2
:106330004CD0FAF75BF9D5F8881021B1FAF75AF981
:10634000032030743FE001213174C5F88860FAF70A
:1063500051F9D6F80480FAF749F9814695F8D80042
:1063600070B918F0704F05D1B8F1000F1CBF0420B0
:10637000FCF72CF80220FCF729F8012085F8D8005A
:106380004846FAF737F9386850F8041F41F002011F
:10639000016020463146FFF740FE386850F8141F70
:1063A00041F001010160287878B9696805F16C0055
:1063B000FAF728F948B9204600F00AF8002105F15B
:1063C0006C00FAF71FF9002000E00120BDE8F2831D
:1063D000F8B504466568A768FAF708F905F1880674
:1063E000316819B9BDE8F240FAF704B9FAF702F9D1
:1063F0003868FFF75FFD38680321FFF764FD3869EF
:10640000796900F034F838680121FFF759FD3968DF
:10641000012041F8200F2046FFF7CAFE306840688F
:106420002946FFF756FD3168087C04281CBF03206D
:1064300008743A697B6901201A439040B269526836
:10644000126842F82C0F38680A68B0F1804F0CBF10
:106450007A4879488068C0F30910101A401E086015
:10646000002030602046AA68BDE8F840104701438C
:10647000B06919E540686C30FAF7C0B8F8B5054660
:10648000AC68606800F18806707900F0A6FB0746EA
:106490007179284600F086FB654800EA07018142D1
:1064A00007D1306808B1042101742046BDE8F240EC
:1064B0008EE7F1BD30B585B0856844682868FFF780
:1064C000F9FC28680F21FFF7FBFC2968032041F83D
:1064D000200F02A8FFF7DAFC6069019020690090A4
:1064E000217B0FF2881050F821300FF28810217EA6
:1064F000554C246850F82120039928682468A04747
:1065000005B030BDF0B585B0446885684F492A7E36
:1065100004F10C063378012B10D142F000420092B6
:106520006A7E11430191A97E41F00041029194F8E5
:106530008D1041F0004141F4005119E00A430092EE
:106540003C4B6A7E42F0004242F480420192327B30
:10655000170018BF012A07BFAA7E1143A97E19435D
:106560000291032194F88D20FF2A03D043EA02010F
:1065700003910421FE224DF82120694604F1900088
:1065800000F05CFA0028C4F89C004FD00FF2DC0247
:10659000337852F823202968012A20D1B1F1804FA5
:1065A000297E0CBF0922212200F04EFB00F050F89A
:1065B0000CBF0A22222200F047FB2868A97E00F0C7
:1065C00049F80CBF0C22242200F03EFB286894F806
:1065D0008D10B0F1804F0CBF0B22232221E0B1F1CE
:1065E000804F297E0CBF0A22222200F02DFB00F0F2
:1065F0002FF80CBF0922212200F026FB2868A97E73
:1066000000F028F80CBF0C22242200F01DFB94F8A7
:106610008D10FF2909D02868B0F1804F0CBF0B22E4
:106620002322D4F89C0000F00FFB012005B0F0BD40
:10663000000006800004C0A00005002030040020F7
:10664000FB60000087610000C4010010000480A00E
:106650002868697EB0F1804FD4F89C007047000034
:1066600080B51046FFF726FF002002BD00000000A5
:106670000100000000000000020000000100000016
:10668000030000001000000020000000018000C096
:10669000018000D50180000C0180005D018000CCEC
:1066A000018000DD40680068012140F84C1F704700
:1066B000F0B52A4C656826688DB02879FBF79BFEFB
:1066C000F9F794FF07463078A8B908233022002153
:1066D00001A8F9F7AFFF069401ABA879204A099009
:1066E00000200090301D6979F9F7A8FF0120307073
:1066F000204600F024F83846F9F77CFF20460DB01C
:10670000F0BD70B544680568F9F770FF0646287853
:1067100080B12079FBF74DFD012808D121680020C8
:1067200041F8040F281DFFF7A5FB002028702079F1
:10673000FBF7F6FD3046BDE87040F9F75BBF4068F7
:106740000268002142F82C1F0068064900F1080287
:106750001160012140F8041F704700000C890000FF
:10676000A56600000004002070B5FBF778F8044629
:106770000026DFF8FC540DE024FA06F0C00708D527
:1067800005EB8600406820B1026811001CBF31464D
:106790009047761C2868F6B28642EDD370BDDFF8CC
:1067A000D4040168DFF8D0040160DFF8D004FBF7FF
:1067B00066B82DE9F0470E00F5B2044644BF86F0F6
:1067C000204686F4C046A80000F1804000F5012074
:1067D00004EA06030168DFF8A8743B4086EA010278
:1067E000A1431943224004F4E023120EB3F5E02F35
:1067F00002F0010202D1CA0105D411E014F4E02F25
:1068000008BF002A0CD001F4E022B2F5A02F04D07A
:10681000B2F5C02F04D1052200E0062262F3124136
:10682000DFF8607401603868E84000F0010805F1A5
:10683000804000F50839B00DB8F1000F00F0010AF2
:1068400003D1600248BF89F800A020020DD5F9F7F6
:10685000CDFE0122AA40396833024CBF1346002303
:10686000914319433960F9F7C5FEB8F1000F03D021
:10687000600248BF89F800A0BDE8F087002948BF42
:106880000021800000F1804000F5012001F03F016F
:106890000268920941EA82110160704710B5DFF881
:1068A000E803006800F07F04FDF71EF8012804D11A
:1068B000FDF710F8022808BF641C204610BD2DE922
:1068C000F04FA1B00546FBF798FCFDF70DF8002648
:1068D000012804D1FCF7FEFF022808BF0126DFF8DB
:1068E000AC03C168C1F3815101294FF0010A04D101
:1068F0000068000E0AFA00F00643DFF89403DFF8A0
:1069000070930078DFF88C73FFF7C8FF5FEA000B25
:10691000C9F800B004D0FF2259463846FCF7BCFF46
:106920004FF00008002405E00AFA00F07C5440EA29
:106930000808641C55F8240000F0FF01FE2909D066
:10694000FF29F6D0594503D226FA00F2D207EBD53B
:10695000022070E00920FBF74EFDC9F880500823A3
:106960002422002117A8F9F75DFE8DF874A017AA5C
:10697000012109F1D400F9F759FE0024DFF818A32A
:106980000BE05046FFF715FF4FF0FF31E0B2FFF785
:1069900075FF0020CBF80400641CD9F80000844285
:1069A00013D226FA04F0C00709EB840B48BF042079
:1069B000F0D428FA04F0C00747BF385D55F820101E
:1069C00004F0FF0040F4C041DBE70823302200213F
:1069D0000BA8F9F72FFEDFF8C452DFF8C42228789D
:1069E00013900BAB00200090102109F18400F9F7FF
:1069F00025FE08232822002101A8F9F723FE686854
:106A0000DFF8A012079000230020089001AA09F1E6
:106A1000A000F9F71BFEDFF89002016821F47C5119
:106A200041F4005101600120DFF880120860DFF8B6
:106A300080120860002021B0BDE8F08F2DE9F04100
:106A40008B4E04460D4606F1D40800F05EF8002097
:106A500035B9002020606060A06085B125E0401C51
:106A600015F82010FE29F4D0FF29F8D032689142A1
:106A700004D206EB810149680029F0D00024404689
:106A8000F9F7BCFD2046BDE8F08106EB8102012349
:106A9000546003FA01F162681143616055F82020E7
:106AA0007D49204600F0A3F8384615F82010FE294D
:106AB000E5D0471CFF29E8D1F6E72DE9F0410500B4
:106AC0000E46F7B203D06A4C2068874201D30220F9
:106AD00019E004F1D40800F018F804EB87004168CD
:106AE00009B101250BE0456001216868B940084300
:106AF000686032466849284600F079F8002540462B
:106B0000F9F77CFD2846BDE8F0814FF0FF314046A3
:106B1000F9F778BD10B50C46F0B1416821FA04F2DE
:106B2000D20719D50122A24091434160002050496B
:106B300001EB840250605748025D5748FF2A0EBFA0
:106B400044F02041D1F8801051F82210FFF731FEB7
:106B50004FF0FF31204686E0022010BD10B50446FC
:106B600006E090FAA0F0B0FA80F12046FFF7D2FFDD
:106B700060680028F5D110BD10B53D4B1C68A142DE
:106B800004D203EB81035B68834201D0022010BD75
:106B900001F18041100001F5083118BF0120087093
:106BA000002010BD10B5324B1C6801F0FF02A2425C
:106BB00004D203EB82025268824201D0022010BD4F
:106BC0000A464FF4E02100F012F8002010BD10B189
:106BD0000160002070470220704780B500F01CF86B
:106BE00080F0005080F4C04040F0004002BD38B555
:106BF0001F4C25680B46114601F0FF02AA4204D241
:106C000004EB82025268824201D0022032BD184653
:106C1000FFF7CFFD002032BD810001F1804101F579
:106C20000121174A09681140224A13680143C340F1
:106C3000DB07126D48BF41F48001C240D00748BF56
:106C400041F40001084670470B4610B51146084A4A
:106C50001468A34204D202EB83025268824201D03C
:106C6000022010BD1846FFF709FE002010BD0000ED
:106C700088200020E0200240E0200260282100203F
:106C8000007F077FD020024044130050A83F0050EF
:106C9000A326002078210020007FC767EC88000031
:106CA0009F67000069670000003009400C40094000
:106CB0000800094080200240DFF800F013C10110F5
:106CC00000B583B00821ADF8001001900321ADF8A4
:106CD00002106846DFF874160968884707BD00B5DA
:106CE0008FB008233C2200216846FDF7A1F8DFF8A9
:106CF000600600F15001079100234FF421710891C3
:106D00006A46012106910FF24521FDF7E3FD0FB020
:106D100000BD10B586B000F007FA0120DFF82C1690
:106D2000DFF830460968ADF80200684688479DF8EC
:106D3000040020700298A06004F13800FEF7FBFF09
:106D4000E06000230420019041F28832002000908E
:106D500004F114000FF2B551FEF7A2FF00214FF02D
:106D6000004000F079FB606006211F20FEF728FD3F
:106D700001208DF801000DF101020020ADF80A009C
:106D8000012101208DF800005020ADF808004FF4DB
:106D90004870ADF806000020ADF804004FF47A709A
:106DA000ADF8020040F20530FDF798FD0DF10A0242
:106DB000022140F20630FDF791FD04F144021E214C
:106DC0004FF44270FDF78AFD04F16402072140F29E
:106DD0000730FDF783FD6A4601214FF44470FDF74B
:106DE0007DFD02AA022140F21130FDF777FD0DF181
:106DF0000602022140F21230FDF770FD01AA0221C5
:106E000040F21330FDF76AFD0DF1020202214FF44A
:106E10004570FDF763FD04F16C0215210020FEF7BB
:106E2000C8FBA0210620FEF7CBFCA0210720FEF71F
:106E3000C7FCA0210820FEF7C3FCA0210920FEF713
:106E4000BFFC0020019001AA01208DF803008DF8FD
:106E50000200042100208DF8010001208DF80000BF
:106E60004FF48160FEF728FD0DF1030201214FF47C
:106E70008060FEF721FD0DF10202012140F2024087
:106E8000FEF71AFD0DF10102012140F20340FEF769
:106E900013FD6A46012140F20640FEF70DFD4FF05A
:106EA000FF30FEF783FB4FF0FF30FEF73BFB00F0B7
:106EB00013FB4FF0FF3000F019FC01208DF80300A8
:106EC00002208DF8020003208DF8010004200FF24B
:106ED00088418DF80000D1E9002301A80121C0E913
:106EE000002300200DF1030200F032FC0DF102023C
:106EF0000121012000F02CFC0DF1010201210220F2
:106F000000F026FC00F00BF901AA0521042000F096
:106F10001FFC04F1900000F014FC04F18400FDF764
:106F2000B1FE04F18800FEF7D0FA2078FEF7CAFA25
:106F30002078FEF715FBFEF7CCFD00F0DAF90FF232
:106F40002043002100F0B3FA06B010BD2DE9F04F48
:106F500087B0FFF7DEFE0FF2E8480FF2F0490FF2BC
:106F6000304ADFF8F053DFF8E46311E06888410746
:106F70000ED54FF6FB710840688005F11400FEF74E
:106F8000B3FE6946022000F01FFC08B900F0C7F804
:106F900000F0CAF80A20ADF802004FF0FF3001906F
:106FA00000F0B4F80028E1D100F0BEF8092000F0AC
:106FB000ABF89DF80620029F00287BD1BDF80400A5
:106FC0000124102804BF29788A4264D138884FF6FA
:106FD000FF72904228D1B87800075CD52869002854
:106FE00059D06978491C697000F10802017940881C
:106FF000FEF7CAFA162818BF0428834609D0286964
:10700000297840880022FEF7C6FD584600F090F827
:1070100041E000F0B2F853466878009000226868BA
:10702000052100F044FA36E03878912802D0B028E3
:1070300008D030E0787810282DD10021082000F009
:107040007BFC28E0787816280AD178880822FEF799
:10705000A2FDD8B9012000F06BF82F6100241AE0DE
:10706000397968687E2905D100F053F80FF20033B2
:10707000397A06E07F2909D100F04BF80FF200338E
:10708000398900910022052100F011FA397907F1C0
:107090000800FEF75FFC6FB164B13846FFF710FEE1
:1070A00008E0A07800F072F800F03EF801940520A6
:1070B00000F02AF8E868FFF7FFFD00287FF456AFDC
:1070C000E868FEF763FE0400F4D020880128E8D0C9
:1070D0000228E9D1A07880B10228E5D105A900F005
:1070E00073FB00F04AF84B469DF814000090002214
:1070F0006868042100F0DBF9D6E705A900F064FB1D
:1071000000F03BF84346EFE7ADF80200684631680F
:1071100008470021049103910291019170476A464A
:107120000121032000F014BB0820ADF800007047D7
:1071300010B5884C226986B0EAB130B9049003904A
:10714000029001900FF25C2308E0117902F108002F
:10715000FEF700FC00F011F80FF25C23607800905D
:1071600000226068052100F0A2F92069FFF7A8FD60
:1071700000202061607006B010BD002004900390D4
:1071800002900190704701460120C6E030B5714C75
:107190000146491E606807298DB000F29380DFE840
:1071A00001F00430916E7A35698807A94FF4417077
:1071B000FDF7D8FC9DF81C008DF8140007A905A860
:1071C0004A7842708A78827000220271C2704A79CD
:1071D0008DF81B200A79C9788DF81A20417105AA0B
:1071E0000821002000F080F907A8FEF7DCFD00F080
:1071F00076F8012100F05BF900F07BF80FF2D01374
:107200005CE000F065F80FF2D41356E004F11400CE
:10721000FEF76AFDFEF71EFB0546401E07A980B279
:10722000FEF72EFB98B90490039002900190009510
:10723000002260680FF2B013022100F038F90DF15E
:107240001E00FEF7B0FD034600F053F810E005A95C
:1072500040F21530FDF786FC00F04BF80FF2981362
:10726000022100F024F905A8FEF79DFD00F037F893
:10727000032124E000F02CF80FF288131DE004F144
:107280001400FEF74FFD1420FFF752FF00F031F815
:107290000FF2881306E01420FFF74AFF00F029F8E8
:1072A0000FF28813022100F002F960680522032121
:1072B0000AE000F00DF80FF280130022022100F026
:1072C000F6F803E00022022100F0ECF80DB030BD2A
:1072D00000210491039102910191009170470021D6
:1072E000049103910291019100910346606800228C
:1072F00070470020049003900290019000900022BB
:10730000606870470146022007E0000011494A8882
:10731000104348808868F9F771B93EB50446FFF715
:1073200003FF0D4604200949ADF8020001906846AC
:107330000968884740B9029A32B1148095700548AF
:107340008168C068FEF7FEFC37BD0000B40700206E
:10735000BC220020940A0020010203040500000062
:10736000424C45205065726970686572616C00001E
:1073700046432056696F6C617465643A2025640049
:107380004D54552053697A653A202464000000006A
:107390005273702073656E642072657472793A203E
:1073A000256400005273702073656E7420726574DA
:1073B00072793A20256400005273702072657472ED
:1073C00079206661696C65643A20256400000000DC
:1073D000496E697469616C697A65640041647665B7
:1073E00072746973696E67004E756D20436F6E6EBF
:1073F000733A202564000000436F6E6E6563746508
:1074000064000000436F6E6E6563746564204164C0
:10741000766572746973696E67000000446973630E
:107420006F6E6E65637465640000000054696D657D
:1074300064204F75740000004572726F7200000086
:107440004368617220313A2025640000436861720C
:1074500020333A20256400002DE9F8430D0008BFD1
:107460000FF2700504460027DFF8349000E07F1C1F
:107470000C2000FB07F859F8086076B1BC4203D035
:10748000B06980472042F2D0C8443268294640465D
:1074900090470028EBD0404600E00020BDE8F28392
:1074A000A889000010B103689B681847704700B9AD
:1074B000704710B586B00C9C04940B9C03940A9CF6
:1074C0000294099C0194089C00940468E468A04715
:1074D00006B010BD030000000FF204237D48102207
:1074E0001321FEF722B800002DE9F04300240828FC
:1074F00085B00E469146784F00F28A80DFE800F0B2
:10750000050C1824303C48537D00082E76D13246B5
:10751000494607F1080076E0152E77DA152107F1C4
:107520001000FBF7DDFA3246494607F110006AE029
:10753000152E6BDA152107F12800FBF7D1FA324638
:10754000494607F128005EE0152E5FDA152107F1A4
:107550004000FBF7C5FA3246494607F1400052E0C9
:10756000152E53DA152107F15800FBF7B9FA324608
:10757000494607F1580046E0152E47DA152107F174
:107580007000FBF7ADFA3246494607F170003AE069
:10759000152E3BDA883715213846FBF7A1FA32461B
:1075A000494638462FE00820ADF808000420ADF821
:1075B0000A00039602A8DFF82481D8F80010884753
:1075C000C8B9049DBDB1786807F1A00188420AD00E
:1075D0000821ADF8001001900521ADF802106846B1
:1075E000D8F800108847324649462846FAF77AFD0F
:1075F0007D603E700DE013240BE0072E06D132466D
:10760000494607F1B000FAF76DFD02E0182400E0EA
:107610000224204605B0BDE8F08300002DE9FE49B4
:1076200090464A680A9C107852780B9D00EB022025
:107630001F46002680B242F62322274B801A03EB16
:10764000040C07D0401E052810D9801F1ED02638F4
:1076500029D03AE0092C28D2C4F10800854228BF7D
:10766000C4F108053D800CF1080129E0D1F80CB007
:107670005846FBF75DFB80B2A04216DB011B8D4232
:10768000A8BF051B3D800BEB040119E018780146EB
:10769000A1420AD3001B8542A8BF0D1B3D8058683C
:1076A0003A8801190DE0082C01D307260FE0C4F138
:1076B0000700854228BFC4F107053D800CF1B001E9
:1076C0003A884046FAF70EFD01E03E800A26304631
:1076D000BDE8FE897C060020C4050020B407002018
:1076E0001D76000000000000000000003EB50446CA
:1076F0000820ADF800000420ADF802007549764876
:1077000000780968754D8000019068468847002818
:1077100014BF002002980100A86001D113203EBDD3
:107720004FF6FF7000F0C8F9E00708D50FF2B0136C
:107730001022112105F11400FDF7F7FE3EBD0020D7
:107740003EBD18B165494860002070471120704760
:107750003EB5002404281346604D31D8DFE800F020
:1077600003080D122500012928D11878287028E077
:10777000012923D11878687023E001291ED11878D7
:10778000A8701EE0012919D11878E87005F11403DA
:107790000FF2710002900022FF200190E91C1120DD
:1077A0000090A86800F0A2F90BE0052906D1052297
:1077B000194605F10C00FAF795FC02E0182400E0E8
:1077C000022420463EBD000010B5024600240846B3
:1077D000042A424912D8DFE802F0030507090C0029
:1077E000097804E0497802E0897800E0C9780170FE
:1077F00005E005220C31FAF775FC00E00224204672
:1078000010BD000038B51046049A00240AB10B20C0
:1078100032BD0A78022A1ED14A681578527805EBE3
:10782000022292B24FF6F175521B012A04D9D21EE0
:1078300002D0521E06D00BE001221A80C9680978D6
:1078400001700AE005221A80C968FAF74BFC04E0CF
:107850001C800A2401E01C800124204632BDF0B5C2
:1078600083B00C780025022C18BF012526D14E6864
:1078700037787678089C07EB0626B6B242F60217F0
:10788000F61B1DD04DF2EF67F61B01D0B61E1ED1C0
:107890001CB9012B03D00D2510E00B250EE010784C
:1078A000CA681070C8680D4A5168904214BF02201F
:1078B000002019B109680A0018BF88472846FEBD94
:1078C00001250195009400F074F90546F6E70A25B4
:1078D000F4E70000B4070020F00700200C090020A6
:1078E000057800005F78000000000000DFF800F07D
:1078F00055C0011038B50FF24100394C394D00F038
:10790000EDF93948FEF7DBFF23681B6801220121EE
:107910002846984722685268012128469047FCF77C
:10792000CDFBFCF7E9FBFDF7D3F9FFF7D8F9FFF73B
:10793000DDFF002032BD000070B52C4E04463068DB
:1079400086B00D4628B900214FF00040FFF784FDB6
:10795000306000F05CF80FF2DC030021FFF7A7FDB8
:1079600030680FF2E003022C0BD0042C02D0052C5F
:107970001CD027E000F054F800F042F80FF2D003DA
:107980000EE0012D06D100F04BF800F039F80FF2AF
:10799000D40305E000F044F800F032F80FF2DC0305
:1079A000306800220221FFF782FD16E000F038F86F
:1079B00000F02DF80FF2D8030221FFF778FD00F058
:1079C00017F80AE000F02CF800F021F80FF2D003CD
:1079D0000221FFF76CFD00F00BF806B070BD00004F
:1079E000D801001000400340A0880000980A002041
:1079F00001208DF800009DF800000028FBD17047A1
:107A000000200490039002900190009070470020A5
:107A1000049003900290019000900022306870471B
:107A20000021049103910291019100910022FFF73E
:107A30003EBD00003E3E3E535441434B2041535314
:107A4000455254002A2A2A4552524F522A2A2A00C5
:107A50003E3E204F5554204F46204D454D4F5259E4
:107A6000210000003E3E20494E5445524E414C20DC
:107A70004657204552524F52210000003E3E2049B9
:107A80004E5445524E414C204552524F5221000017
:107A90003E3E204943414C4C2041424F525421002C
:107AA0003E3E2044454641554C54205350494E4C8F
:107AB0004F434B210000000038B54FF6FF74A04241
:107AC0000DD10020654A137898420EDA21F8204043
:107AD00001EB80050023401CAB70C0B2F3E700F05F
:107AE000A9F810B104800021817031BD2DE9FE4F4D
:107AF00080460026B8F1000F82B006D0080004D0FE
:107B0000180002D0109F380001D1022035E00F9CF0
:107B100000252CE0EDB2A94638F829004FF6FF7198
:107B200088421EBF08EB890A9AF8020000281DD07F
:107B3000029ABDF83810049800F02AF85FEA000BAA
:107B400014D09AF80200C00705D500F019F80121F9
:107B500000F086F806439AF80200800706D500F088
:107B60000FF8022100F07CF80643F6B26D1C3B4989
:107B70000978E8B28842CDD3F0B205B0BDE8F08F05
:107B8000019700949DF80C2038F829005B46704757
:107B900030B5002400E0641CA3B28B4207D2A4B22B
:107BA00000EB0413DD689542F5D1184630BD002086
:107BB00030BDF8B5044606980D460026F0B9022BF4
:107BC0001AD11078517800EB01270798C043B9B259
:107BD00001420FD1E8680168204600F012F8B9B2FE
:107BE00088420CD0E8680168BAB2204600F00FF86D
:107BF000064604E0802602E00D2600E00B26304613
:107C0000F2BD80B500F016F800B1807802BD70B505
:107C100004460D46164600F00DF840B929464FF6C9
:107C2000FF7000F007F808B9112070BD048086705D
:107C3000002070BD10B5002200E0521C074C2478D3
:107C4000D3B2A34207D2D2B231F822308342F4D168
:107C500001EB820010BD002010BD0000F0070020E5
:107C60002DE9F04186B00D4690461F46044603AB11
:107C70004FF6FF721B21FDF75EFE059040B3FF211A
:107C800002910246BDF80C10DDF834C001910DF1EF
:107C900012030021009120463946E047064688B984
:107CA0007889ADF81000E80705D5424604A92046BA
:107CB000FDF7EFFC05E00C9B424604A92046FDF7CA
:107CC000F7FC06462EB11B2104A8FDF743FE00E099
:107CD0001526304606B0BDE8F08100000149086075
:107CE00070470000C005002081B001208DF8000021
:107CF0009DF800000028FBD101B0704770470000DC
:107D0000DFF800F06DA9011070B50568AE6A0024B7
:107D100006E0242000FB04600830FEF7B3F8641C82
:107D200095F82C00E4B28442F3D3686800F0E8FAD6
:107D3000DFF868020068FEF711FF0020288070BDA0
:107D40004FF0FF310160DFF85C12416000210172E9
:107D500070472DE9F043DFF8489299B0D9F8005008
:107D6000D9F80470044688461646F8F73FFC29887F
:107D7000012902D1F8F73EFC0DE001212980F8F736
:107D800039FC1EB904A8FFF7DBFF04AE002C18BFB6
:107D9000B8F1000F01D100205BE010A800F0C8FA94
:107DA0007068149010A9307A8DF85800F87900F0B6
:107DB000AAFA00284DD0686008233068A860AC6239
:107DC00085F82C802422002107A8F8F72BFC002638
:107DD00008E0242000FB064007AA01210830F8F73C
:107DE00025FC761CF6B24645F3D301208DF834000D
:107DF00007AA012105F10C00F8F718FC3979DFF822
:107E0000A801DFF89841014300916946BA7910430F
:107E10004860DFF89821787910438860FE20C860B8
:107E2000201DFEF70BFE206098B1DFF88411DFF80B
:107E300084010968B0FBF1F0FFF762FF79792068EF
:107E40000122FEF799FE39681122484600F078F8C1
:107E5000484619B0BDE8F083026892F82C209142A0
:107E60003CBF012200F0DBB87047006890F82C207E
:107E7000914200D3704770B508302423026A5943F9
:107E80008B188D5801685C6803F108063046F8F7D6
:107E9000B9FB48B11CB121462846FDF7B7FF304673
:107EA000BDE87040F8F7AABB70BD2DE9F843006843
:107EB000154690F82C20914228D200F10802242483
:107EC000106A614351F80080089C081800F1080905
:107ED000099811685E1B071B00F01DF9F6B2FFB28E
:107EE000A0B10020844607E05A185B1C02F808C0C5
:107EF000DBB29E42F8DA401CC0B2874205DB0119B2
:107F000005EBC11189B20023F2E714E0BDE8F1836B
:107F10001CB500F00BF803D200F003F800F0B2F843
:107F200013BD01240194049C00947047046894F8E4
:107F30002C40A14270474846BDE8F243F8F75EBBCB
:107F40002DE9F04100F022F800F01DF800F019F8DA
:107F500000F013F800B12FE0BDE8F0812DE9F04109
:107F600000F014F80122FEF707FE00F00AF800F016
:107F700004F800B120E0BDE8F081424629462046E1
:107F80003DE0B97930680022FEF7F6BD0446034EA5
:107F9000676830680D469046397970477026002032
:107FA0009489000040420F000000C08000008080E3
:107FB0009C8F0000A0860100B9793068BDE8F041CF
:107FC0000122FEF7D9BD38B50FF258142568009587
:107FD00001F00F049DF80030D2189DF802308DF8A2
:107FE0000020E3188DF8023003229DF8013003EBE6
:107FF00011118DF801106946FFF7A2FF31BD00B5E0
:1080000085B00023039300920293019169460068B2
:10801000406800F092F900B1012005B000BD2DE9E3
:10802000F84381461500D9F800600F4605D0B168C5
:1080300006F10C00F8F7E6FA10B3B06A2421794390
:108040000F58081800F1080825B1B1684046F8F744
:10805000D9FA90B10024224600214846FFF7B3FF29
:10806000802207EBC4114846FFF778FF641C082CF8
:10807000F1DB2DB14046F8F7C1FA06F10C005BE7E1
:10808000BDE8F1832DE9F84F064615460C461F461C
:10809000284600F065F980460A9807EBC0101FFAE1
:1080A00080FA3068826A242161438E580B9C8918BB
:1080B00001F108091CB1816800F02DF830B30027E8
:1080C0000FF2640B12E0213A02EB820292B200231B
:1080D00003EB020C03EB010E1CF80BC00EF806C0FC
:1080E0005B1C052BF4DB002141717F1C47450ADA3C
:1080F000062000FB07A17A5D8819202AE3D106211A
:10810000FDF784FEF1E70CB1484607E0BDE8F18FCA
:1081100001F1080901684846F8F774BABDE8F24F62
:10812000F8F76CBAB010000000005F000000070014
:108130000700147F147F14242A7F2A122313086453
:108140006236495522500005030000001C22410000
:108150000041221C00082A1C2A0808083E080800C2
:108160005030000008080808080060600000201077
:108170000804023E5149453E00427F4000426151A1
:1081800049462141454B311814127F10274545457A
:10819000393C4A4949300171090503364949493694
:1081A000064949291E0036360000005636000000F8
:1081B000081422411414141414412214080002015A
:1081C000510906324979413E7E1111117E7F49499C
:1081D00049363E414141227F4141221C7F49494964
:1081E000417F090901013E414151327F0808087F62
:1081F00000417F41002040413F017F081422417F20
:10820000404040407F0204027F7F0408107F3E41CF
:1082100041413E7F090909063E4151215E7F09190E
:108220002946464949493101017F01013F4040400B
:108230003F1F2040201F7F2018207F6314081463F5
:108240000304780403615149454300007F41410222
:108250000408102041417F00000402010204404054
:10826000404040000102040020545454787F4844A8
:1082700044383844444420384444487F38545454A3
:1082800018087E090102081454543C7F080404783D
:1082900000447D40002040443D00007F1028440001
:1082A000417F40007C041804787C0804047838443A
:1082B0004444387C14141408081414187C7C0804F2
:1082C00004084854545420043F4440203C4040207B
:1082D0007C1C2040201C3C4030403C44281028445A
:1082E0000C5050503C4464544C440008364100004B
:1082F000007F00000041360800003E1C080000001E
:10830000016809680847084A1268904201D30020B2
:10831000704709B90FF228010C224243034B981809
:108320009A58D26810470000280B0020548900009A
:108330000FF20C012022F9F7E5BE0268126910471E
:1083400000000000FFFFFFFF000000000000000031
:1083500040420F0008000000000000000000000084
:10836000002100E0491CC9B20A5C002AFAD1084683
:10837000704701680A680A4482604B681A44C26008
:108380000831016070478168C268914208D1016874
:108390000A680A4482604B681A44C260083101606E
:1083A0008168491C816011F8010D704738B5044699
:1083B0000D46A068E168884212D120686168884251
:1083C00008BFFCF783FA2068227C016802B14944A7
:1083D000A16042680A44E260083091422060ECD01B
:1083E000A068401CA06000F8015D31BD2DE9F0419E
:1083F0008AB000F1080105910268520801EBC20140
:1084000006910021079108910168490800EBC1011C
:1084100008310091017901F001018DF810104068D8
:108420000099400801EBC0000190002002900390E9
:1084300006E005A8FFF79DFF07980899884207D135
:10844000059806998842F4D101980AB0BDE8F081F8
:1084500005A8FFF798FF044614F0030603D105A80A
:10846000FFF791FFC61C25090F2D14D105A8FFF7B2
:108470008AFF00F10F050EE007980899884204BFB3
:1084800005A8FFF776FF0798401C079010F8011D1C
:108490006846FFF78BFF761EEED1002DCCD005A8E5
:1084A000FFF771FF0646A00800F00300032804BF91
:1084B00005A8FFF768FFDDF800800299039F06EB2F
:1084C000002008E0A8F10808A8F10801801A0A684D
:1084D00049685718394658F8082C8A1A8242F1D34D
:1084E00040420C18AE1CA7D0BC4206D158F8044B31
:1084F00058F8040B2718BC42F8D00298039914F8D6
:10850000015B884217D100980199884208BFFCF7A7
:10851000DDF9009800689DF81010029009B14844F8
:108520000290009902984968009A014408328842F2
:1085300003910092E7D00298401C0290761E00F84A
:10854000015D3FF479AFCFE780B501280CD0022858
:108550000CD0042802D008280AD00BE000201146D5
:1085600012689047002002BD0220F8E70420F6E7D9
:108570000520F4E7FCF7AAF900BF10B5044601E0B6
:10858000F9F724FFB4FA84F0202800D110BD00F0E0
:1085900016F8F5DB401FF9F72EFFF3E710B5044698
:1085A00001E0F9F7A9FEB4FA84F0202800D110BD4B
:1085B00000F005F8F5DB401FF9F7B2FEF3E7C0F174
:1085C0001F00C0B2012181404C400528704738B5DA
:1085D0000546012068713D4C2879A8B1FBF762FC83
:1085E00005462078FF2805D12846FBF766FC6FF08A
:1085F000060032BD401C2070C0B2012804BF606874
:10860000FFF7BBFF284615E0FBF74CFC21780A007A
:1086100004D1FBF752FC6FF0070032BD491E2170F8
:10862000C9B239B9FBF749FC6068FFF7B7FF002012
:10863000687101E0FBF741FC002032BD70B50446D3
:10864000606810F07F4F02D06FF0020070BDFBF742
:1086500029FC1E4E0546307828B17068FFF79EFF52
:108660006068FFF78AFF606870602846FBF725FCAA
:10867000002070BD80B5406810F07F4F00D00DE045
:10868000FFF77BFF002002BD80B5406810F07F4FF0
:1086900000D003E0FFF782FF002002BD6FF0020070
:1086A00002BD10B5044682B0A1686068086014205D
:1086B000FBF7AEFD009010B96FF0030016BDA36884
:1086C000034A0F21F9F708FE002016BDB807002065
:1086D0004985000010B50446FAF705F8207100201E
:1086E00010BD80B5FAF710F8002002BD10B50446A1
:1086F000F9F773FD6060002010BD10B50446606896
:10870000F9F7EFFFA060002010BD0000F0B50446AF
:1087100085B0A068656800790E460021FE2803D068
:108720001C49084300900421FE204DF801006946D1
:108730002846FEF783F905F10C07386038B3307826
:10874000387205F2344605F13400306005F1180145
:108750004FF4806070601C2205F23C40F9F7D2FCB7
:1087600002A8FFF7EDFA02AA01213046FFF7F1FA5D
:10877000786040B10021FFF778FB78680021FFF7AF
:108780006BFB204603E03868FEF7E8F9002005B0EF
:10879000F0BD00000008C08010B54468206930B109
:1087A0000021FFF762FB2069BDE8104012E010BD18
:1087B0001CB54468206913468B4238BF0B4630B164
:1087C000019300917F2300220021FFF76EFB2069B7
:1087D000BDE81C400021FFF73FBBF0B58BB04768F8
:1087E0000D4614461E4604A81821FAF779F906200A
:1087F0004443387D234601281A4605D005D3032873
:108800002AD038BF7F2300E00022D0B2D9B28842FC
:1088100007D001950095DBB23869D2B20021FFF78D
:1088200044FB1498109B0390324613980290162133
:10883000129801901198009004A800F024F8009577
:10884000E3B2386904AA0021FFF762FB386900210E
:10885000FFF702FB0BB0F0BD00227F23D9E710B574
:108860004468E06840B1FEF779F90020E0602069D3
:10887000FFF74AFA0020206110BD6FF00100704739
:108880004FF0004070470CB480B502AF3A6827F053
:1088900003031B1DF9F70DF9BDE8804002B07047D6
:1088A000190880801B088080070880800608808067
:1088B0000B2000C0132000C00C2000C00F2000C0FF
:1088C000122000C00D0080800400C0800500C08020
:1088D0000E00C0801A008080140080801800C080C4
:1088E0001E00C0800300C080FE000000FF000000EA
:1088F0000000000000000000158B00008D26000025
:1089000001010100000002400A29FF009817002021
:10891000048900000000000000000000000000408A
:1089200017FF000000000000040000000800000025
:108930001000000009080AFF0080004018FF000036
:10894000000000000500000000000100000002001F
:1089500017181EFFE88E0000B81700201C890000C1
:10896000E88E000094180020388900000000000004
:10897000000000000000000040A1C0A6A22FF800E7
:10898000278116AC00AFB01000000000788900000D
:1089900004050E00701900208C890000FFFF0505FA
:1089A000948900000D000000CC8E0000A01900206A
:1089B000A08900000000000000000000000000008E
:1089C000080000009E260020C08900000000000072
:1089D0000000000080B5F7F709FE36490A7822B991
:1089E000354B1B681A7001220A7080B2BDE8024044
:1089F000F7F700BE38B5F7F7F9FD04462E4D2846C7
:108A000000F064F8A0B2F7F7F5FD284632BD70B566
:108A10000E461446F7F7EAFD85B227480168097843
:108A200009B900F053F826B94FF4807101220846C5
:108A300012E0304600F027F858B114B14FF0FF3083
:108A400020700820F9F76CFC2846F7F7D3FD0020CA
:108A500070BDB2687168306800F042F817490120B3
:108A6000086017480068C007FBD50220154909684F
:108A70004968884706460CB1002020702846F7F761
:108A8000B9FD304670BD4FF0FF3180B102681AB1B8
:108A9000403AB2F57F5F0AD2426822B1A2F58072F5
:108AA000094B9A4203D28068102838BF002108463B
:108AB00070470000A2260020C4890000A80250428E
:108AC00008800240CC01001000FFFF0001680A7816
:108AD0002AB901220A7040680068F9F78CBC704717
:108AE00010B50A4B1C6824F480641C600902120251
:108AF000090CA4B202F4706244EA014442EA014162
:108B0000C0F387101C600843586010BD14800240F9
:108B100030BF704738B5FAF759FCFAF709FCF9F796
:108B200044FB044604F00C000C2849D0600721D413
:108B3000F8F71EFE054601210120F9F740FB234905
:108B4000096801FB05F2904214D28220B0FBF1F0DB
:108B50001F4C291A04F10C00F7F75CFD04F10C001E
:108B6000F7F75CFD0120F9F79EFC04F10C00F8F723
:108B70005CFE27E0200723D41648FAF7D3FA04282E
:108B8000FAD0E206144900D418B9086840F0010090
:108B900002E00868400840000860104C1048114D81
:108BA000016841F00301016020202168896988473C
:108BB00028682068806B804701202860286801E0D1
:108BC000FFF7A6FFBDE83140FAF704BC9C8F000018
:108BD000EC0C0020004003408C210840B80100103C
:108BE000242208402C200940EBC70CEEC90CF1CB25
:108BF0000CF44B14F74E19FA521DFD582500613143
:108C000001144202184E031C5A04249305309300A9
:108C1000E88B00000D070000C7100000E97C000091
:108C2000E1110000E97C0000DB13000029140000C2
:108C30002B140000E97C0000E97C0000BF15000057
:108C4000D5150000E97C0000E97C0000E97C00000B
:108C5000E97C00008D110000E915000033160000CA
:108C600071160000D5890000F58900000F8A000008
:108C70007B756E6B6E6F776E2D696E7374616E634C
:108C8000652D6E616D657D007B656D7074792D69F4
:108C90006E7374616E63652D6E616D657D0000009D
:108CA0007B7374617469632D696E7374616E63653F
:108CB0002D6E616D657D000019E050F8041BCB0737
:108CC00044BFA9F101035918121F0023042A41F8D7
:108CD000043BF9D25FEA827C0B4604D54FF0000CCE
:108CE000A1F800C09B1CD10744BF0021197050F8A7
:108CF000042B002AE1D1704710B507497944183197
:108D0000064C7C44163404E00A68081D1144884768
:108D10000146A142F8D110BD2C0000006C010000FA
:108D20007FC80110C9BC011051B2011037C2011037
:108D3000BDAD0110C1B1011071BA011069BB0110C4
:108D400021C0011075FFFFFF8C180000180E0020D5
:108D50000000000099F6FFFF020000000200000082
:108D6000E40500001A000000780100202C0000003B
:108D70007DF6FFFF02000000020000001706000061
:108D800003000000EC0100200400000061F6FFFF7A
:108D90000200000002000000F505000003000000D2
:108DA000F00100200800000045F6FFFF020000006F
:108DB00002000000AA0500001A000000A401002023
:108DC0002400000029F6FFFF02000000020000005E
:108DD000A80500000C000000C80100201C000000D5
:108DE0000DF6FFFF02000000020000001B0500005E
:108DF0001B0000000001002044000000F1F5FFFF0F
:108E000002000000020000008E05000006000000C5
:108E10000002002004000000D5F5FFFF0200000062
:108E2000020000006C05000003000000F8010020B3
:108E300008000000B9F5FFFF02000000020000007A
:108E4000E204000022000000440100203400000081
:108E50009DF5FFFF02000000020000002805000051
:108E600009000000E40100200800000081F5FFFF78
:108E70000200000002000000400100004F0300005B
:108E800020050020F4080000DFF800F059C50110AB
:108E90000548012808BFF9F7DFBF704703480128DC
:108EA00008BFFFF7F1BF704701000000010000009C
:108EB0000A18232A242A252A262A272A282A292A60
:108EC0002A2A502A02000000B08E00000D87000000
:108ED00099870000B1870000DB8700005F880000F1
:108EE0007B88000081880000035F00005B5F00005A
:108EF000E3610000EF61000021630000D163000026
:108F0000AF61000000F00BF8002803D0FFF7F4FE7B
:108F1000FFF7C4FF0020FEF7EDFCF9F741FF012049
:108F2000704700B581B0FFF7B3FFAFF3008001B029
:108F30005DF804EBFFF7E6BF44F22830C2F2000010
:108F4000854648F62370C0F200008047FEE7000027
:108F5000010000000000000000000000000001000F
:108F600000000000F0FFF1FFF2FFF3FFF4FFF5FF58
:108F700002000000648F000045B50110C52F0000FD
:108F800099A6011019B8011000280000032800005C
:108F90000129000002290000200000000A00000052
:108FA000C40B0020E5210000FF1D0000F71D00009C
:108FB000892E0000452F00001200018301000143AB
:108FC000C5A70D63AD2F15B0070100340B0020C5F8
:108FD000A7000161106108100F071000003840352C
:108FE000002D400140028460005D08101700F80168
:108FF00018A384070083057EA40306E0EA23060184
:109000000003040102351C102308047F17630400C9
:109010003888604500C3003801AC526003A302AD3C
:109020000163026801438AFF0043022804FF011024
:1090300003FD7C00000E6360026406002082A00A2B
:109040004D6F64656C204E756D62657296F003021B
:10905000536572696119500F4669726D7761726567
:10906000205265766973696F6E1CF0020348617265
:109070006418F00203536F667418500F4D616E75DB
:109080006661637475726572204E616D65181003B8
:10909000FE006578707C14046D656E74616C32122C
:1090A0000D191002100100020747888F603001C4BB
:1090B0008E0010528C102002060E00201043B28E3B
:1090C0001043CC0510612052072052B420D2D42086
:1090D00052082052B620D2EC2052092052B820C3A8
:1090E000040620520A2052BA20D21C20520B2052D1
:1090F000BC20D23420520C2052BE20D24C20520D23
:109100002052C020D26420520E2052C2201274205D
:109110001003A53E0000BB04300187400001120689
:1091200007100301051B0068DC7005108C00001897
:109130008C000112640C12C01810070303000078A1
:109140001E00207C04432C0120196682000130059A
:109150000600800C0000E813F003983075FFFF0054
:1091600001F00150020106AD8B0200A4CB708FA468
:10917000560FA4126610253F430C0910529020C7C9
:10918000300AD45210306A6804D130D244305211BF
:1091900030526A78D20E30D2583052123030016CD0
:1091A0008F0001520F305294A0D21440D26C405222
:1091B0001340126E10120408D218301280301C02B4
:1091C00043686172E3031DCE032004737469632056
:1091D000316AD114F2023214F2023314F20234145E
:1091E000F336350001100A140953696D706C65423D
:1091F0004C45505D1C0770686572616C0512501219
:109200000313020A65193C40030302F0FF00261213
:10921000202782202811208387718A2C0205730061
:10922000006C051E2CE8052104611A47E519583029
:1092300001FF001413124C1C2104525404834002F9
:10924000444D7B03100101007018F206701C128C53
:10925000182104529404529C0412CC211208244375
:10926000180F7C4380061012BC1C2104439C01048F
:109270006301004C4101434B180D12E424210452B8
:10928000EC0452F40452FC0443040C04939717F4C6
:10929000830000E95101435C0C131234082104528D
:1092A0003C04524404524C04525404525C04526430
:1092B00004526C04830000A86204641510439815DE
:1092C0001CD0030BC201100001D2011112B84821B9
:1092D0000452C00452C80452D00452D80452E004CC
:1092E0006178F1C7016520F3090101E68008DB27F9
:1092F0000000492800009B27242BFF7FDC6202012D
:1093000000030A0208100283010001A10CD003B877
:109310000C0020000152E814200234010020045205
:109320003C0412000110039C2600206804126C0407
:10933000211043283F08110170052001010000A001
:1093400025103101520001100720050020040C00F7
:10935000200111C30100012002C40B0020042200DF
:109360000150026CDC0200015003780B0020030D59
:1093700010034D2F00009504F30101000120023479
:109380000C002017120001000220050020520001ED
:0C93900052000112000100020800000061
:10FDC00038B504460D460DF08BFF084821680160E8
:10FDD00061684160A16881600CF0C5FB0CF0B5FB67
:10FDE0002846BDE8324007F0A4B800BFD84700203D
:10FDF0004F7D0100AFAA0100D7910100CBAC0100FB
:10FE0000B564010031AF01004743010063130100F5
:10FE1000813B0100A9FF00000A006E1902000000EA
:10FE200094CC01000200000090CC01000061310080
:10FE30002CFE0000010000000000D0020A050000B6
:10FE4000000000000201000000000000100000009F
:10FE500000000000EC000021000000000000000095
:10FE600054FE000038FE0000000000003CFE0000D0
:10FE700040FE000044FE000048FE00004CFE000072
:10FE800050FE0000B4460020DFF800F0419500105D
:10FE9000DFF800F071950010DFF800F0D195001048
:10FEA000DFF800F03D970010DFF800F065970010D4
:10FEB000DFF800F029980010DFF800F0F598001046
:10FEC000DFF800F0C9990010DFF800F0F999001090
:10FED000DFF800F0159A0010DFF800F0319A0010FA
:10FEE000DFF800F0A19A0010DFF800F0F59A00109A
:10FEF000DFF800F0159C0010DFF800F08D9C00107A
:10FF0000DFF800F0099D0010DFF800F0459D0010BB
:10FF1000DFF800F0D19D0010DFF800F02D9E0010FA
:10FF2000DFF800F04D9E0010DFF800F06D9E00102D
:10FF3000DFF800F08D9E0010DFF800F0AD9E00109D
:10FF4000DFF800F0CD9E0010DFF800F0ED9E00100D
:10FF5000DFF800F00D9F0010DFF800F0499F00105F
:10FF6000DFF800F0699F0010DFF800F0D19F00106B
:10FF7000DFF800F011A00010DFF800F031A0001051
:10FF8000DFF800F075A00010DFF800F0F1A000101D
:10FF9000DFF800F009A10010DFF800F0B5A10010B3
:10FFA000DFF84019087070472DE9FE430C46200425
:10FFB00054D5DFF83009007800F0A9FD05004AD0DB
:10FFC000DFF8247939680126002918BF11F1010FE3
:10FFD00007D0DFF81809007800F03BFD4FF0FF3044
:10FFE00038602878812802D082282CD02FE0002089
:10FFF0008DF808608DF80900AE88AF7995F8028019
:020000040001F9
:10000000B00A3F2807D1C6F3C21020B100F029F88A
:1000100000F02EF803E000F024F800F088F88146A4
:10002000284600F007FD9DF80800A0B1DFF8C008E1
:1000300001904B469DF8090000903A4631464046F3
:1000400000F0BAF907E0284600F064FB064616B156
:10005000284600F0EFFC84F4004000E00020BDE8FA
:10006000FE8302AB0DF109022946304670470000BD
:1000700038B500F07F04C00900F00700401E0428D6
:100080000D4652D8DFE800F0030C2C474C00122C30
:100090004BD12A7CE9682889BDE8384000F0E3BFED
:1000A0002889E968012C17D00B2C11D00D2C0BD00E
:1000B000132C05D0192C38D1BDE8324001F0D5B849
:1000C000BDE8324001F0BEB8BDE8344001F08CB864
:1000D000BDE8344001F07AB8BDE8344001F023B8FF
:1000E00028891B2C11D01D2C07D0432C1DD1AA8987
:1000F000698902F0C2F8002032BD6B7C2A7CE96875
:1001000001B0BDE8304002F0C5BA2A7CE968BDE81C
:10011000384002F0F5BA204601B0BDE8304013E2A5
:10012000204601B0BDE830408AE1012032BD0B46D7
:1001300040F21D41401A00F0978040F2E471401AED
:1001400000F09580801E00F098802A3800F097809B
:10015000363800F08F8040F29E31401A00F09480D3
:10016000401E00F09380401E00F09280801F00F03F
:1001700091804FF47F71401A00F08E8040F6FC3180
:10018000401A00F08C80801E00F08C80001F00F070
:100190008B80083800F08A80401E00F08980401E65
:1001A00000F08880401E00F08A80C01E00F08C8025
:1001B000401E00F08C80401E00F08C80401F00F03C
:1001C0008D80401E00F09180401E00F08980401E0E
:1001D00000F08F804DF6E231401A00F08C80401E16
:1001E00000F08D80C01E00F08E80401E00F08F80D9
:1001F000401E00F08F80401E00F09480401E00F0F2
:100200009780401E00F09680401E00F09780401EB0
:1002100000F09680401E00F09680401E00F0968010
:10022000C01E00F09580801E00F09680401E00F0F9
:100230009680401E00F09880801E00F09980401E3D
:1002400000F09B80801E69D0401E00F09C80401E04
:1002500000F09E80401E00F09E80801E00F09F8077
:10026000401E00F0A280A5E01889FFF70DBE986837
:10027000FFF70EBE986802F045BE02F09FBD598997
:100280001889C9B2FFF708BE02F09ABE02F0A7BDF6
:10029000FFF706BEFFF708BE188902F0BDBE9868DA
:1002A00002F073BEFFF704BEFFF706BEFFF708BEFD
:1002B000FFF70ABE1889D968C0B2FFF709BE1889CE
:1002C000D968C0B2FFF708BE1889FFF709BE1889C0
:1002D00002F0F1BDD9689868FFF706BEFFF708BEC7
:1002E0009A7A597A187A02F0FBBD1889C0B202F0E6
:1002F00000BEFFF701BE1889C0B2FFF701BE188922
:10030000C0B2FFF701BED9689868FFF701BE9868D0
:10031000FFF702BE1889C0B2FFF702BE1889C0B24B
:10032000FFF702BE59891889C9B2C0B2FFF700BEF3
:10033000FFF702BE1889C0B2FFF702BEFFF704BE86
:100340009868FFF705BE1889FFF706BEFFF708BEDD
:100350001889C0B2FFF708BE1889FFF709BE59898E
:100360001889C9B2FFF708BED9681889FFF708BE17
:1003700018895989C0B2FFF707BE59899A89188927
:10038000C9B202F000BE18895989C0B2FFF700BE99
:10039000188902F0E6BD1889C0B202F0CFBD5989B4
:1003A0001889C9B2C0B2FFF7F7BD1A69D968986851
:1003B00002F01FBD012070472DE9F843089C8046DC
:1003C00004F10C000F461546994680B200F020FB60
:1003D000060016D08020307086F8019040F27F60D1
:1003E0007080B780B57106F10C00F471B0602246E0
:1003F000099900F0BEFA31464046BDE8F44300F0EA
:1004000028BBBDE8F18310B502460020941E012CE4
:1004100002D9A41E02D004E0102900E004290ED065
:100420000CE0A2F12004402C04D2BDE8104010469C
:1004300003F03CBCA2F18001102900D3022010BDC2
:1004400070B5401E052882B00C461546DFF8A4643E
:100450004FD8DFE800F0030C15182A3D00F04BF8E8
:1004600008BBE2683146284603F006FF76BD00F07F
:1004700042F8C0B9E2683146284603F00DFF76BD68
:1004800003F031FF0FE0A06868B1DFF86C14016081
:10049000DFF868140988818091218171032101812D
:1004A0001421418123E0022076BDDFF854341B681B
:1004B000083300221B68002100209847B071010A10
:1004C000F171010C000E70723172042028700EE080
:1004D0004FF6FF70ADF8000002F00CFCADF8000024
:1004E0000222022028706946B01D00F042FA002066
:1004F00076BD012076BD257A667A3146284682E7A8
:1005000038B5012815461C4602D0022809D00DE056
:10051000049B0A462146284601B0BDE8304004F05D
:1005200017B80846BDE8324004F036BB0846BDE8BF
:10053000324004F03FBB0B4601281146184608BF65
:1005400004F042B804F04DBB2DE9FC410F461546BE
:100550000024DFF8A06380B3032849D0062837D0F1
:1005600007283AD008283FD00A2846D00B2852D076
:100570000C2869D00D2800F08D800E285ED00F2841
:1005800053D010284CD011283DD012283FD030280D
:1005900064D031286BD032285BD0332800F07F80C4
:1005A000342800F08080352800F08C80362800F058
:1005B0008C80372800F09180A7E078690190386935
:1005C0000090FB68BA7A797A387A04F059FB82E0B5
:1005D000F968387A04F07EFB7DE0FB68BA7A797AB4
:1005E000387A04F0C0FB76E0387A04F0F0FB72E071
:1005F000F968387A04F0C9FE6DE03A7B7989387A77
:1006000005F020F867E0B86805F059F863E0B868CD
:1006100005F089F85FE0F968B86805F0F1F85AE08C
:10062000B97A388905F03AF955E0387C0090FB68D2
:10063000FA7AB97A388905F080F94CE0FA68B97A23
:10064000388905F0B9F846E03989F86805F035F9D8
:1006500041E0F968B86805F0B5FC3CE03889798973
:1006600026282DD028282BDA04F044FE33E04FF65C
:10067000FF78ADF800803889FF2821DA26281FD0BE
:1006800028281DDA04F043FE4045ADF8000017D0DD
:1006900002200EE0B97A388905F0ECFC1BE0B8685E
:1006A00004F0BBFB17E0387A04F00CFC009038B182
:1006B0000420287002466946B01D00F05AF925E072
:1006C000022423E004F023FC05E07989FA683889E4
:1006D000C9B202F0D9FC044618E03F89B11D384682
:1006E00002F09AFD044640F201403F1A04D03F1F39
:1006F00004D0FF1E04D005E0022004E0102002E038
:10070000042000E00120287000E001242046BDE81C
:10071000F68100002DE9F04184B0044600208DF8F8
:10072000090001208DF80800A588A079A778042D7C
:10073000804669D8DFE805F068030A28440002AA69
:100740000DF10901204600F07BF85BE0002610283F
:1007500014D013280DD0142807D0152854D1E268DE
:10076000A17A208901F03CFF4CE0A06803F0C8FDAD
:1007700007E0A17A208903F0BDFD02E0207A03F0B2
:10078000B6FD8DF8086040E00026A8B1042804D02A
:10079000052806D006280AD036E0A06805F059FDE5
:1007A00033E02089E168C0B205F02CFD2AE000F0BA
:1007B00041F805F0E7FC25E0A06805F03EFD21E0EA
:1007C000062821D8DFE800F01B20140F20040A00BF
:1007D0002089E168C0B200F05FFE13E000F02AF863
:1007E00000F02BFE0EE0E168208900F004FE09E035
:1007F0002369A27BA189A06800F0D2FD02E0A06875
:1008000000F0A7FE064600E00126204600F012F99F
:100810009DF8080050B13648019033469DF8090014
:100820000090424629463846FFF7C6FD002004B036
:10083000BDE8F08161892089E268C9B2C0B2704721
:10084000F8B50D4681792B4F00240429164626D091
:10085000102910D0112912D0122915D0132922D015
:10086000142926D015292CD017292FD018290ED0BD
:1008700019290FD033E0007A05F00EFE24E0817ACA
:10088000008906F062F826E006F08AF823E006F018
:1008900073F820E0C168008906F009F80FE080686D
:1008A00002F05DFE10E0C268817A008902F064FE09
:1008B00005E0837C028AC168007A02F001FD0446EB
:1008C0000EE0008902F099FD347009E00269C16808
:1008D000007A02F0BAFDB8710120287000E001240E
:1008E0002046F2BDDA48002044430020E1480020C1
:1008F0001647002010470020020202001AFE0000E6
:100900004043002000B583B00821ADF800100190ED
:100910000B21ADF802106846DFF8741609688847A5
:100920000EBD1FB58DF806100824ADF800408DF8F7
:1009300004000624DFF858168DF808200393ADF85C
:10094000024068460968884704B010BD80B505209C
:1009500006F07FF800F0EDF90C2000F001F802BD80
:10096000DFF82C160968ADF802006846084706F063
:100970007FB803E011F8013B00F8013B13465A1E13
:10098000002BF7D170471144491E03E011F80139DB
:1009900000F8013B13465A1E002BF7D1704770B583
:1009A00004460D46A8B206F07FF8060003D02A469A
:1009B0002146FFF7DEFF304670BD10B513465A1EC4
:1009C0003BB110F8013B11F8014BA342F6D00020D7
:1009D00010BD012010BD10B5044610460A46014660
:1009E000204606F081F8204610BD03F073BCDFF806
:1009F000A425DFF8A435126A11541B7805E0DFF84E
:100A00009835DFF890251B78126AC018115470478A
:100A100010B5040001D1002010BD04F10C0080B21B
:100A200006F042F828B1002101600481FF218172A3
:100A30000C3010BD80B508B9052002BD10F8021CAD
:100A4000FF2901D0042002BD0C3806F03AF800203E
:100A500002BD38B50C46010622D5DFF838150A78F4
:100A6000FF2A08BF4D7805D0DFF82C351B78096ABE
:100A70009A188D5CFF2D02D1FFF768FF0EE000F0A1
:100A80009BF90146FF2004F8020C23460022284669
:100A9000FFF747FF48B12046FFF7CCFF012032BDEA
:100AA0002146BDE83840002200E032BD70B50D009F
:100AB0000446164618D0200648BFFFF747FFDFF868
:100AC000D81409788C4204D32846FFF7B3FF0320DB
:100AD00070BDA5F10C000168002904BF817AFF29CF
:100AE00004D02846FFF7A6FF052070BD8472012EB2
:100AF000DFF8A004294603D1001D00F055F802E0FC
:100B0000001D00F039F800F033F8002070BD2DE929
:100B1000F0410446DFF88404DFF878740068804709
:100B2000804678680026002503E005B9064650F89F
:100B30000C0C50B110F8021CA142F6D1002D08BFD8
:100B40000546F4D000F014F805E04FF400412046CB
:100B500000F0A4F825B132462946381D00F031F8DE
:100B6000DFF83C140968404688472846BDE8F08114
:100B70004FF40041204642E038B500F00FF8002164
:100B800045F80C1C216811B9256006E0114651F8A2
:100B90000C2C002AFAD141F80C5C27E10446DFF85E
:100BA000FC0300680D46004738B5FFF7F7FF2168E2
:100BB00045F80C1C2560DFF8E8130968BDE83440EF
:100BC000084770B5044600F014F8A5F10C0123683D
:100BD0000A689D420CBF226046F80C2C00220A6075
:100BE000FF228A72BDE8704002E1DFF8B4130968A1
:100BF0000847DFF8A80300680D46164600472DE9B0
:100C0000F0410446DFF89003DFF8885390F8008045
:100C100020060E462CD50420FFF7FAFE070008BF79
:100C2000042039D04FF6FF7038807E80A7F10C0683
:100C30002878FF280FBF6D78296A40440D5CFF2D8E
:100C400005D13846FFF7F6FEFFF780FE0EE020469E
:100C500000F0B2F8FF21B1723B460146002228465F
:100C6000FFF75FFEC0B13846FFF7E4FE012013E056
:100C7000444510D200F028F8DFF82813096831F84D
:100C80001420324321F81420FFF7AFFFE868FFF784
:100C900039FE002000E00320BDE8F08138B50C46A5
:100CA000BD490978884205460CD200F00DF8BD49CF
:100CB000096831F81520A24321F81520FFF795FFA8
:100CC000002032BD032032BDB4480068004730B573
:100CD000B04C0020606083B005F048FF06F095F846
:100CE000AD480578680005F0DFFE20626A00FF214C
:100CF000FFF771FE0222FF21A01CFFF76CFE06F039
:100D0000DBF800F016F81420A14D2968ADF80200B8
:100D1000684688470198206100F00BF81520ADF86F
:100D200002006846296888470198801E606100209B
:100D30003EBD0820ADF80000704730B587B00820F0
:100D4000ADF808001B20ADF80A0001200390914D7A
:100D50000FF27D008E4C21680590E8690690A86925
:100D6000049002A888470499A96108B1FFF7EEFD35
:100D700000F053F8FFF7DDFF0A20ADF802004FF056
:100D8000FF300190684621688847F1E780B500216F
:100D9000804A0A449378FF2B01D1907001E083428E
:100DA00003D141F08000C0B202BD491C0229EFD33B
:100DB000FFF7CCFDFF2002BD10B580F08004022CAF
:100DC000A8BFFFF7C3FD73482044807810BD000022
:100DD00038B50446FFF778FF05466E48C1698C4276
:100DE00004BFC068FFF78EFD4FEA0500BDE8344040
:100DF0006B490968084710B50446608850B9A07966
:100E0000FFF7C4FFFF28E07102D16FF0030010BDAF
:100E1000002010BD6FF0010010BD2DE9F04F8BB028
:100E200005F0C7FF00245FEA000B03D005F0D3FEF6
:100E30004FF0FF3B574DA868010003D0804701E009
:100E4000FFF784FD0820ADF808000720504E3168F8
:100E5000ADF80A0002A888474F499DF80E20049F6C
:100E60000978E8B9002600E0761C8E42E8D2286AAC
:100E7000805D9042F8D1F6B2FF2EE1D017F8080C51
:100E8000FFF784FF17F8061C012908BF387002D04D
:100E9000022908BFB87039463046FFF7DAFDD1E7BE
:100EA000404F3868E4B230F8140018B9641CE0B25E
:100EB0008842F5D3E0B28842DFF8E480DFF8DC90C6
:100EC0001DD2D9F8000080473968E4B231F814A087
:100ED000002200F047F8344A2C70514652F8242082
:100EE000204690478246FF202870D9F800008047AE
:100EF000396831F814204AEA020200F033F805F0AC
:100F000058FF07465F452AD007B9284F6869B8429D
:100F100038BF0746D9F8000080470446FFF709FFAD
:100F20001C20ADF80200A869316801906846884726
:100F30000821E869ADF81410401C1321E861ADF8F0
:100F40001610099006971A49A8690891079005A8F4
:100F5000316888470798A861204600F005F80BB073
:100F6000BDE8F08F21F81420D8F80010084710B51C
:100F700048B1002300E05B1CDCB2944205D2DBB236
:100F8000C45C8C42F7D0002010BD012010BD0000D1
:100F9000D8470020A444002018FE0000DC470020B1
:100FA000E0470020F0470020F0FD00008EC2F52849
:100FB000D10D0100DFF800F0F5950010DFF800F02A
:100FC00031960010DFF800F05D9600100A4610B56B
:100FD000052A18BF042A03D0062A18BF072A08D1F9
:100FE0000C24484B62431A4422F8301D90700020B4
:100FF00010BD022010BD38B50D46044628880528CE
:1010000018BF042803D0062818BF072801D1686834
:1010100008B9022032BD0121204605F096FC08B92E
:10102000142032BD4FF6FE70844207D0204605F0F2
:10103000C8FC2989884201D21B2032BD3248007881
:1010400000282946204603D0BDE8344003F08CBB7D
:10105000BDE8344003F03EBB80B52C4B00931346F3
:101060000A4601211AE070B50D4684B004461646C2
:10107000EB88AA886988288801F082FE58B1002090
:1010800002900196042000902A46214B122120460E
:1010900003F0B6FA00E0182004B070BD03F0E2FAE5
:1010A00002BD38B504461B480129017011D11A4808
:1010B0000088051DADB20120FFF77CFF94FBF5F021
:1010C00082B2284601B0BDE8304000230021FFF77E
:1010D00075BFBDE832400020FFF76CBF03B50D4877
:1010E0000078012881B003D102AA01A9FFF76AFFA5
:1010F00007BD094A001F1080034801707047064869
:10110000008870478C480020E646002069480100AE
:10111000E7480100DF480020FC460020704700003F
:101120006E490860704780B5002200920B4601228C
:101130006B4900F0BAF802BD80B50A88172A05DBB2
:10114000002200920B4603226649F2E7022002BD0C
:1011500038B50D460446A878012818BF02280DD1DD
:10116000288800281CBF6868002807D0022103F0E7
:101170005DFD00902B4605225B4931E0022032BD27
:1011800038B500F01EF81CBF6868002806D000F0D3
:1011900036F800902B460722544921E0022032BD48
:1011A00038B500F00EF81CBF6868002807D002218F
:1011B00003F03CFD00902B4609224D4910E002202F
:1011C00032BD0D46044628880028704738B500F027
:1011D00024F808B100F013F800902B460B22454983
:1011E000204600F062F832BD38B500F016F808B1BC
:1011F00000F005F800902B460D223F49F0E7012151
:1012000003F014BD38B500F008F808B1FFF7F7FF98
:1012100000902B460F223949E2E70D4604466868E4
:10122000704738B5FFF7CDFF1CBF6868002807D0AE
:10123000022103F0FBFC00902B4611223049CFE73E
:10124000022032BD80B5002100910023132270E7F7
:1012500038B50D460446A86810B1052103F0E6FC38
:1012600000902B4617222749BAE780B5002100914C
:10127000002319225DE738B5FFF7CFFF10B1032136
:1012800003F0D4FC00902B461B2209E038B5FFF791
:10129000C4FF10B1032103F0C9FC00902B461D22AE
:1012A0001949204605F0A7FF32BDF8B50446069857
:1012B000009015461E46204605F09DFF07000AD106
:1012C00006480268100006D0012D04BF3078451C86
:1012D000E9B2204690473846F2BD00000848002099
:1012E000FB6F010017700100317001008B7001006D
:1012F000CF700100EB7001004371010067710100C4
:101300006B710100A5710100D5710100DFF8581C57
:101310000870704738B5DFF8544CDFF8545C20761D
:101320002878C00005F0C0FBE061C8B1002108E0EA
:101330004FF6FF7220F8312000EBC10300225A6003
:10134000491C2A789142F3DB052000F0AFF8207E9B
:1013500001F058F8BDE83240DFF8180C05F037BA54
:1013600031BD38B50C46200418D5DFF8000C007EDE
:10137000FFF7CDFB05000ED02878B02808D128460D
:1013800000F0FDF820B1297905F1080003F01CF9FF
:101390002846FFF74FFB84F4004032BD002032BDE9
:1013A0007CB506001C460DD0ADF800108DF802206B
:1013B0000196684600F0B8FF05001AD1CCB17689D5
:1013C000300001D1022514E00C2005F06DFB08B9B6
:1013D00013250EE00021016086808460DFF8981BF1
:1013E0000A6812B9086004E00A4611680029FBD1B6
:1013F0001060284676BD30B50C46DFF87C1B0546EC
:10140000086883B0002201E00246006898B1838832
:10141000AB42F9D10368002A0CBF0B60136005F0E2
:1014200050FB6946284600F0CDFF010002D10CB107
:10143000019921603EBD01203EBD70B550BB012920
:1014400026D1DFF8280BC169002300E05B1CDFF820
:10145000204B2478A34217DA31F833404FF6FF755A
:10146000AC42F3D0002400E0641C467EE5B2B542F5
:10147000ECD201EBC305E4B26D680C266643AD5BAC
:10148000002DF1D0012070BD1078BDE870400DE056
:10149000182070BD022070BD0022002803BFDFF8B5
:1014A000CC0A407E08700222104670472DE9F843AE
:1014B000DFF8B87A0446002078760C25F869DFF862
:1014C000B06A406805FB04F870B105F0FAFA002034
:1014D00006E0F969C0B201EBC00100224A60401C7D
:1014E0003278C1B29142F4D3307808FB00F080B278
:1014F00005F0DAFA5FEA000928D0307808FB00F23C
:1015000000214846FFF767FA00200FE0516805FB0D
:101510000CF34FF0000E21F803E019440CF1010C1C
:10152000C1F808E0A445F1DBC144401C3278C1B2E7
:10153000914208D2F969C0B201EBC0024FF0000C31
:10154000C2F80490EEE77C76002000E01320BDE8AE
:10155000F28301460020C90705D50023102201218E
:10156000DFF8180C1CE77047DFF80C1A096821B186
:101570008A888242FAD188687047002070472DE936
:10158000F04186B004460020ADF8100001208DF82F
:101590001200DFF8D859286A38B9FFF7B0FD05F016
:1015A00083FA0028286200F0E280182200212846F1
:1015B000FFF711FA2079461C02284FF6FF7817D062
:1015C00006282CD008282FD00A2833D00C2857D032
:1015D0000E2800F08B80102800F08D80122800F07B
:1015E0008F80162800F09380182800F09780BBE0C9
:1015F000FFF785FD288029466088FFF79DFD0028BC
:101600002189288804D0814228BF01462980A0E092
:10161000814228BF0146608802F045FFA4E004A98A
:10162000204600F0AEF87DE004AA0021204600F03C
:101630002CF977E000F0A0F8070052D0608805ABE5
:1016400042460B2102F084FF03006B6024D0207916
:10165000BDF81620039000953946BDF8140002909D
:101660000020019000F026FA070004D16088294686
:10167000FFF7ACFD29E0162F686808BF00272BE0B4
:1016800000F07AF807002CD0608805AB42460D21A7
:1016900002F05EFF686020B92089ADF810001127C4
:1016A00045E02179BDF8162003910346BDF81410DA
:1016B0000291618901910095394600F0FBF907001C
:1016C00006D160882946FFF78FFD002841D12AE026
:1016D000162F686808BF002703F083FA380001D18D
:1016E00021E001272089ADF810001CE004A9204664
:1016F00000F06EF916E004A9204600F0E9F911E0C7
:101700000DF1120204A9204600F086FA0AE00DF15C
:10171000120204A9204600F0C0FA03E004A9204602
:1017200000F029FB0746380011D0162F11D0607841
:1017300014280CD0207928702F712946BDF810008C
:1017400068806088FFF7EFFC08B1012601E0162FE2
:101750000AD160882B46F2B2162102F09AFE18B127
:10176000F1B2284602F030FF204602F0C9FD9DF894
:10177000120006B0BDE8F08120890DF1160100F0DD
:10178000B9BE2DE9FA47044686B06088DFF8DC5719
:1017900005F0C5FD80460DF1120000F0D4F80027D9
:1017A00081464FF0FF0AB9F1000F5BD009E0BDF8A8
:1017B00010304354BDF81000696892B2000A885492
:1017C000571CBFB2A8F1050087424BDA207903907D
:1017D0000026A8F1070080B20290019605F11A00D8
:1017E00000902B6ABDF812206088494600F0CCFBBF
:1017F000002802BF6A8B208A904214D1296A60694E
:10180000FFF7DBF878B1686858B900F055F907219F
:1018100002F09EFE686020B9069920890880112098
:1018200030E0B9F80A60BDF81220618904AB48467F
:1018300000F086FE002E8146B5D06868C655781C3B
:101840006A6880B231121154411C4A1C6868B9F1AF
:10185000000F89B2ABD100F801A092B2686800F81D
:1018600002A0571CB8B248B13F04B80C28802946E2
:101870006088FFF785FC28B1162003E006992089CF
:1018800008800A2008B0BDE8F0872DE9F04304463F
:1018900085B060888846914605F041FD851EADB251
:1018A000DFF8C87601E0401C2081A81E39898842F3
:1018B0002FDB5FEA08002CD104A800F044F80600F2
:1018C00027D070892081BDF81020317A608800F01F
:1018D0009DFD5FEA00081CD120793B6ABDF810200D
:1018E00003903146A81E80B200F0EBF800F0E2F859
:1018F0005FEA00080DD173897A8B396A608800F03D
:101900002AF85FEA000804D120894FF6FF71884267
:10191000C9D1388901000AD0798890FBF1F038806C
:1019200039466088FFF73CFC50B1162008E05FEABA
:1019300008002089A9F8000008BF4FF00A084046B7
:1019400005B0BDE8F0830090237B6189208904F114
:101950000D0200F0A0BD2DE9F846824689461546E5
:101960001E4605F0DCFCDFF804460746208990B9E6
:1019700000F0A3F80921504602F0EAFD606008B9C2
:10198000112023E0A81C60803A1F208901466B18B3
:101990009A4206D203E06088A91C8842F4D0012054
:1019A00014E0401C2081606846542089411C21813C
:1019B000310A62681154606823892A4649461844EE
:1019C000FEF7D7FF2089281820810020BDE8F28685
:1019D0002DE9F047044686B06088DFF890750D4623
:1019E00005F09DFC0026A0F10109A0F1010814E01A
:1019F0003888798B0346C9188845BCBFA9EB00001D
:101A0000788378687A8B396A1844FEF7B2FF388891
:101A1000798B0818761C3880B6B2A0898642BCBF84
:101A20003888404534DAA06810F8162000EB4600EC
:101A300004A9407802EB002080B200F05BFD0100B9
:101A400009D14FF0010A00F02BF8786808B103F0D3
:101A5000C8F85046DDE02079BDF8102003901FFA49
:101A600089F000F02EF83B6A00F024F80028824646
:101A7000E9D178680028BBD100F01EF80F2102F0F0
:101A800067FD00287860B3D100F00AF81120E1E783
:101A900060883946FFF7B6FB0028DBD01620D9E76F
:101AA000A06810F8161000EB4600407801EB00200B
:101AB00028807047608867E2608800234FF6FF72D5
:101AC000704702900020019007F11A0000907047C3
:101AD0002DE9F047044686B06088DFF890548946C7
:101AE00005F01DFC059004F10D0204A80090237B75
:101AF0006189208900F0CFFC0026B24607464FF0EE
:101B0000FF0810E0696801F8068080B2696801F892
:101B10000080461C68686A8B296AB6B28019FEF795
:101B200028FF688B8619B6B2FFB1BDF81020397A4C
:101B3000608800F06BFC5FEA000A13D12079BDF8E1
:101B40001020039039460598801F80B20290002033
:101B5000019005F11A0000902B6AFFF7ABFF5FEAD6
:101B6000000A10D07889A9F80000002E48D06888B3
:101B700096FBF0F0288029466088FFF752FB00288A
:101B800047D0162045E07EB9FFF796FF112102F0FD
:101B9000DFFC686020B97889A9F80000112038E0DE
:101BA000688B001D688009E0688B6988021D91427E
:101BB000DDD10599891F80198142D8DB6968788950
:101BC000885579896A68701C80B2090A1154461CCC
:101BD000BDF8102061890DF11203384600F0B0FC09
:101BE0000746701C002FB6B28CD06A68BDF8121080
:101BF000915580B2BDF812106A68090A115488E73D
:101C00005FEA0A002089A9F8000008BF4FF00A0A1D
:101C1000504606B0BDE8F087FEB504460D46208963
:101C2000164602A900F066FC07002ED0387A80061E
:101C30000BD5BDF8080000F0A1F903000BD06088B7
:101C4000122239469847070020D1607C002814BF33
:101C50005220207901E00E2718E00190002000902A
:101C60006389E2682189608800F08AFA070007D159
:101C7000607C68B96088FFF7E5FA48B11620FEBDC0
:101C8000162F03D10027377002E001272089288012
:101C9000607C00B100273846FEBD2DE9F0410446C6
:101CA00082B00D4660889046012104F04EFE002768
:101CB00018B9142060700E205BE02089694600F09E
:101CC00019FC060051D0307A80060BD5BDF8000013
:101CD00000F054F9030013D060881222314698476F
:101CE000070043D16688304600F008F928B94FF65E
:101CF000FF7000F003F9A0B3068000219B4E02E0C4
:101D00000E2733E0491C737ECAB29A4229D2426838
:101D1000C9B20C234B4313441A88002AF2D10C2277
:101D200004F108011846FEF724FE002088F80000A0
:101D30000C2204F108013046FEF71BFEA2896088E0
:101D40000023172102F004FCB06060B1A289216970
:101D5000FEF70FFE60883146FFF77AFA40B1162091
:101D600007E0092702E0112700E0012720892880E9
:101D70003846BDE8F6812DE9F043044683B060881B
:101D8000894600F0BBF800265FEA00084CD0207AB4
:101D9000012845D1414604F1080000F051F8A0B1F6
:101DA000D8F804701820019078880090BB88BA6831
:101DB0003988608800F0E4F90646162E02D100202A
:101DC000B8602DE060B3388828E000270EE001906D
:101DD00068880090AB88AA68608800F0D1F9064650
:101DE000162E18D10020A8607F1CFFB25F48407EED
:101DF000874215DAD8F804100C227A430A441546B3
:101E000029880B000CD07B1C83421DBF90890028C1
:101E100016201820DBE7002EE6D02888A9F800005D
:101E2000404600F080F82EB96088FFF71EFA20B116
:101E3000162003E0162E08BF00263046BDE8FE83BC
:101E40002DE9F84F0C460020002700264FF00C0B20
:101E500046490DE0984202BFBCF8025093B2AB4233
:101E600024D1BCF80430DF19BFB29A1892B2761CA4
:101E70004B7E9E420FDA63680BFB06FC9C44BCF869
:101E8000003043B10028E5D1BCF80470BCF8022052
:101E90001846BA18EAE7022E2DDB38004FF0000989
:101EA00004D002F087FE5FEA000801D1002023E0A1
:101EB000CA461AE00BFB0AF14518A96859B1AA886D
:101EC00008EB0900FEF755FDA88848441FFA80F981
:101ED000A86802F086FEBAF1000F04D00C2200219F
:101EE0002846FEF778FD0AF1010AB2456068E1DB99
:101EF000C0F8088087800120BDE8F28F10B51B4A2A
:101F0000D269002100E0491C194C2478CBB2A342CD
:101F100007D2C9B232F831308342F4D102EBC100AA
:101F200010BD002010BD70B5044600250BE0B06860
:101F300008B102F056FE0C2200213046FEF74BFDA0
:101F4000002030806D1C0949497EE8B2884207D2E2
:101F50006068EDB20C216943461830880028E6D14C
:101F60004FF6FF70208070BDFE4600201C48002008
:101F700054480020272201004048002080B5FFF788
:101F8000F3FA00B1806802BD2DE9FE4F0D46804690
:101F9000287AC00693461E464FF0000A0CD55846D4
:101FA000FFF7ECFF030000F0E4800A2229464046D8
:101FB00098470028824649D128780C9F0D9CDDF86F
:101FC0003890022816D100F018F94FF42051401A29
:101FD000012810D9801E3AD0401E14D0FD3876D08A
:101FE000401E00F07D80401E6AD0401E6FD0401E13
:101FF00000F09180A7E0002C2AD1E86801783980B0
:102000000278416883E0002C22D101203880002131
:10201000E868007830706889401C80B200F06AFA85
:10202000398860B10278921C5118398041897170E9
:102030004189090AB17002784168F01C68E0081D06
:10204000388004220021701CFEF7C5FC93E0002CB0
:1020500062D1E8680488042038803470200A7070E7
:102060000DF10201204600F045FA05001ED0EC6893
:10207000BDF802204FF6FF786B46414600F060FA4B
:1020800040B92B786A688B48022105F0F7F808B947
:10209000ADF80080207802280AD161680222301D44
:1020A000FEF767FC3888801C388001E0ADF80040FE
:1020B000BDF80000B070BDF80000000AF0705AE0F2
:1020C00054BBE8680168404605F05CF902E01CBBBF
:1020D000E8680088022139803070000A70704AE098
:1020E000E868FEF744FC82B2A242B8BF4FF0070A8C
:1020F00041DB944208BF002206D009EB0401914263
:10210000B2BF4A46121B92B23A80E9682144304677
:10211000FEF72FFC2FE014B14FF00B0A2BE0E8681C
:102120000721398001783170417871704188B17030
:102130004188090AF17001793171C1887171C088D3
:10214000000AB07117E05846FFF70EFA00281CBFCE
:10215000D0F800C0BCF1000F0BD00F980290CDF862
:10216000049000943B46324629464046E04782466A
:1021700001E04FF00E0A5046BDE8FE8F08460020F1
:102180002DE9FE438046894617461E4602A9484669
:1021900000F0B0F905002CD0BDF80800FFF7E4F915
:1021A00000281CBFD0F804C0BCF1000F1FD00A9853
:1021B0000B9C0090019433463A4629464046E0473E
:1021C0000646B8B9FE2C15D02878022812D100F0A6
:1021D00014F842F6021188420CD13878797800EB75
:1021E000012082B24946404600F047F802E00E2640
:1021F00000E001263046BDE8FE836868017840783B
:1022000001EB002080B27047E0B58DF80820022372
:10221000120A8DF80920FE2201920022009202AAE1
:10222000FFF7AEFF0EBD7CB50129044605D002299B
:1022300022D1012104F089FBF0B92046FFF75EFEB0
:1022400008B1FFF770FE01A800904FF6FF7502235A
:10225000194A2946012000F01EF90BE0F0680168D8
:10226000204605F075F8BDF80420002329463046C5
:1022700000F066F90600F1D173BDF8B50F4F0446C2
:102280003878FF280D46164611D00A20FEF7C0FB0D
:1022900068B1B12101704480002141700171C58095
:1022A000068101463878BDE8F440FEF7D2BBF1BDA7
:1022B000000000009CCC0100A4CC0100FE460020E0
:1022C00070B5DFF8385A28780624604304F0ECFB38
:1022D000DFF82C1A086008B9132070BD0020FF2217
:1022E00006E03380401C0023F270B2703371C0B23C
:1022F0002B7898420ADA0B6804FB00F61E4400288B
:102300000CBF4FF6FE734FF6FF73EAE70FF2514032
:1023100001F0EAFF0FF61510FEF702FF0FF6551059
:1023200004F055FA002070BD70B50446208868B1ED
:1023300060680378426800F040F948B96068037843
:102340004268DFF8C00900F03AF908B9022070BD10
:10235000A078C01F0A2801D3182070BDDFF8A85943
:102360002888010004D02188C0F58030884201DA35
:10237000012070BD0C2004F097FB060001D1132052
:1023800070BD002008E06268298880B202EB00126C
:10239000401C5181491C298081B222889142F2D38C
:1023A0000020306008222146301DFEF7E2FA6868FE
:1023B00010B96E6004E0084601680029FBD1066090
:1023C000002070BD38B502460846DFF83C194C685D
:1023D000002301E02346246894B1A5686D899542E5
:1023E000F8D12268002B0CBF4A601A6018B108228D
:1023F000211DFEF7BEFA204604F063FB002032BD2B
:10240000012032BDDFF804190870704710B504468A
:1024100010461422114203D000F0DAF8012204E041
:102420004A0608D500F0D4F8002201462046BDE84F
:10243000104004F0CCBAC80701D4022010BD00201F
:1024400010BD70B505460E46B0061C4609D51046AF
:1024500000F0BEF801462846BDE87040012204F0B5
:10246000B6BA8820064210D0104600F0B1F80146F6
:1024700006F00802284604F0AAFA010009D0617AA1
:1024800041B1217A012904D070BDB00701D40320E5
:1024900070BD002070BD2DE9F0478146DFF8680867
:1024A00044688A4690461E4600E02468FCB1002736
:1024B00000E07F1CA188B8B28842F6D2A068BFB203
:1024C00000EB07156889484528BF8245F1D33EB126
:1024D000297868683346424604F0D0FE0028E8D0E8
:1024E000089810B1A16849890180284600E00020C1
:1024F000BDE8F087F0B5DFF81028546800E02468E4
:10250000E4B1A5686E89B042F9DBA788BA19904298
:10251000F5DA4FF0000C01E003F1010C1FFA8CF228
:10252000BA42ECD21FFA8CF305EB0312B2F80AE0C0
:102530008645F1D101B10E801046F0BD0020F0BDFE
:102540002DE9FC4104460027ADF804704FF6FF78F2
:102550006089404515461E4608D001AA0092401CDD
:102560002378626880B2FFF796FF07462378626897
:1025700000F023F830B923786268DFF8880700F0AC
:102580001EF808B160890CE023786268DFF88007E4
:1025900000F015F858B11FB1BDF80400A84203D0EF
:1025A000284600F0D2F803E07889404400E06089D2
:1025B00006B130803846BDE8F681DFF858070221C1
:1025C00004F05CBE80B500F0F3FA00B1008802BDF3
:1025D00080B500F0EDFA08B1807802BD102002BD90
:1025E00070B5012982B00446154616D0032918D0CB
:1025F000052925D0072927D0092929D00B292BD037
:102600000D292DD00F292FD0112931D0132933D0E6
:10261000172934D0192936D039E02946FEF783FD31
:1026200033E0FEF76CFDADF8000069462046FEF78A
:1026300083FD06002CD12988204601F034FF27E0D5
:102640002946FEF785FD20E02946FEF799FD1CE0AE
:102650002946FEF7A5FD18E02946FEF7B7FD14E070
:102660002946FEF7C1FD10E02946FEF7CBFD0CE040
:102670002946FEF7D6FD08E0FEF7E4FD05E0294611
:10268000FEF7E6FD01E0FEF7F0FD064600E002265B
:10269000304676BD2DE9FC410E46054617461C46E0
:1026A00001A900F092FA804638BB380014D000200F
:1026B000ADF8000069463088FFF71CFF012FBDF818
:1026C000000018BF0027FFF783FF01463A4628465F
:1026D00004F07DF9804680B931462846FEF7D6FDE4
:1026E000804650B9019DFF2C07D0AB1C1E22294605
:1026F0000FF2555001F0B9FEEC704046BDE8F6818E
:102700007CB50D460446164601A900F05EFA17286E
:102710001AD0300014D00020ADF800006946288897
:10272000FFF7E8FE012EBDF8000018BF0026FFF7F6
:102730004FFF01463246204604F049F9010003D11B
:1027400029462046FEF797FD76BD10B50446FFF7F3
:1027500039FF01001CBF611E0C18A0B210BD0000A3
:102760002DE9F0430D4689B08146A87800261E2841
:10277000174614D1484600F03CFA06001EBFB07858
:10278000FE28FF2822D0002000900022AB78F078AD
:10279000494601F03FFE304600F040FA16E01228AC
:1027A00004BF6878012813D0484600F022FA0600DA
:1027B0000ED0327910000BD0100607D4A978484605
:1027C00001F084FE307940F080003071002069E033
:1027D000DFF838452078FF2812D0A878811E172905
:1027E0000ED200F08AF958B1A87800F0B3F938B1E8
:1027F000287810B96878012804D1A878122801D067
:1028000006204FE0A87800F078F9844602A80090EE
:10281000AB88AA6869782878E0470028804640D1CC
:10282000A87800F097F9024602A9484690478046EA
:10283000D8B9AB78042B34D002A8009000222078BD
:10284000494601F0E7FD804658BBA97802A801F08F
:1028500055FE08B100203870A878122804BF6978A6
:1028600001291ED0EEB130711BE06878C8B9A87894
:102870008DF800008DF804806946A878042818BFF8
:102880000628BDF80800ADF802004846FEF74BFCEC
:1028900028B16B4601221621484601F0FAFD4FF09F
:1028A0000008404609B0BDE8F083002070472DE9DC
:1028B000FE430D46804628886988814201D3010085
:1028C00001D101206DE00021ADF8041002914FF616
:1028D000FF7900E0401C002100910023698800225C
:1028E00080B2FFF7D8FD070037D0BDF804000028FC
:1028F00038D16B464A460521404601F029FE0400C6
:1029000001D111204DE002943878022806D101202F
:102910008DF80600BDF80000860827E002208DF83B
:1029200006001221BDF8000090FBF1F6387810285F
:1029300013D1788904F8010B102200F034F8103418
:10294000BDF80400401CADF80400B1B2BDF80400AD
:10295000884202D278894845BCD1BDF8040080B9CC
:102960000A201EE09DF806000128DFD138780228F1
:10297000F3D1788904F8010B022200F014F8A41CAA
:10298000DEE701A94046FEF7E3FB48B101AB0522B3
:102990001621404601F07DFD10B1029802F021F9A8
:1029A0000020BDE8FE837889000A04F8010B204668
:1029B0007968FDF7DEBF10B582B04C880888844284
:1029C00001D3020001D1012016BD00F016F808B9AC
:1029D0000A2016BD002016BD10B582B04C880888AC
:1029E000844201D3020001D1012016BD00F005F898
:1029F00008B90A2016BD002016BD002200924A1D0B
:102A00000B79214647E510B5044682B00846694671
:102A10000088FFF76FFD08B9012016BD017ABDF8E7
:102A200000202046FFF7F2FC16BD70B582B00646C6
:102A30000D46002401E0641CA4B2A888844229DA6F
:102A4000286810F8142000EB44006946407802EB37
:102A5000002080B2FFF74EFD50B9286810F814101E
:102A60000170286800EB440149784170012076BD6F
:102A7000017ABDF800203046FFF7C8FC0100DAD02B
:102A8000296811F814200A70296801EB4402527871
:102A90004A7076BD002076BD10B50C4682B0208805
:102AA0006188814200D308B9012016BD2379994875
:102AB000621DFFF784FD08B9102016BD00200090AC
:102AC000237961882088621DFFF7E5FC08B90A2098
:102AD00016BD002016BD38B504460D466946288847
:102AE000FFF708FD08B9012032BD017ABDF80020CA
:102AF0002B462046FFF7A5FC32BD022814D004283F
:102B000014D0062814D008281AD00A2812D00C286D
:102B100012D00E2812D0102812D0122812D0162847
:102B200012D0182812D013E07B4870477B487047BA
:102B30007B4870477B4870477B4870477B487047AD
:102B40007B4870477B4870477B4870477B4870479D
:102B500000207047022814D0042814D0062814D06E
:102B6000082814D00A2818BF0C2812D00E2812D01A
:102B7000102812D0122818BF162810D0182810D0EC
:102B800012E06F4870476F4870476F4870476F4852
:102B900070476F4870476F4870476F4870476F487D
:102BA00070470FF2090070470020704700207047FF
:102BB0005549496800E0096829B18A68528982420A
:102BC000F9D1081D70470020704710B50C4600F081
:102BD00010F860B104B120608078FE2801D1172080
:102BE00010BDFF2801D1002010BD162010BD02200D
:102BF00010BD10B5424A1268002100E0491C3F4C4C
:102C00002478CBB2A34207D2C9B206234B43D45A8D
:102C10008442F3D1D01810BD002010BD10B5044679
:102C2000A01C01F02AFCFF20E07010BD10B50C467E
:102C3000FFF7DFFF30B101794A1C944204BF01F075
:102C40008001017110BD000010B582B004001EBFEC
:102C5000A078FF28FE280BD0002000901E2321889A
:102C6000E078172201F0D6FBFE20A070FF20E07074
:102C700013BD000070B504464FF6FE70844282B06A
:102C800037D008004FF6FF760AD12046FFF7B1FF94
:102C900078BB3046FFF7ADFF05002AD0048073BD36
:102CA000012906D12046FFF7A4FF050021D02E8080
:102CB0000BE002291DD10121204603F046FEC0B9D8
:102CC0002046FFF796FF050013D0A878FF280ED006
:102CD000FE2807D0002000901E23E8781422214609
:102CE00001F098FB2846FFF799FFFF20A87000200D
:102CF000287173BD0448008870470000DD4800203B
:102D00004C4800209CCC01001846002000470020C1
:102D1000A0CC010098CC01000D70010027700100CB
:102D200049700100D17001001F710100477101005D
:102D300093700100EF7001007D710100C37101000B
:102D4000AB280100AF280100B7290100D9290100F3
:102D5000072A01002B2A0100992A0100D72A010025
:102D6000DFF800F0DD8A0010DFF800F0A18B001022
:102D7000DFF800F0D5700010DFF800F09D5800106B
:102D800030B540F67B44851FA5423CBF8D1FA54250
:102D900012D2814210D3B2F5FA7F0DDAA3F10A0004
:102DA00040F67744A04207D2501C49004843B0EB9C
:102DB000C30F8041C00F30BD002030BD80B505F08D
:102DC0005AF88DF8000005F0ABFE77490020087036
:102DD0006A4676490880012140F6034063E080B5E9
:102DE0000FF26022412141F20200FFF7B9FF0020FB
:102DF00002BD7CB5002808BF00294FF620442DD124
:102E000062BB01A805F0C7FD9DF8040000EBC000FF
:102E1000451DEDB2284603F047FE060018D02020DD
:102E20003070042070700020B0709DF804000028FD
:102E30000CBF0022721D311DF01C05F099F83246BE
:102E40002946204606F08AF8304603F03AFE15E09F
:102E500004218DF801102020072106E005F088F8F4
:102E600004218DF80110202000218DF800008DF83C
:102E700002106A460321204606F070F8002076BD55
:102E800080B500208DF800006A46494800788DF82A
:102E90000100042100208DF80200464800788DF8DA
:102EA000030042F20200FFF75BFF002002BD012099
:102EB00070470120704738B5044642F2160529468E
:102EC0000020FFF751FF204605F0E9F88DF80000DB
:102ED00020B16A4601212846FFF742FF002032BD9B
:102EE00080B5012305F0B5FA00F01BF842F21E0090
:102EF000D9E780B5012105F069FB00F012F842F234
:102F00001D00D0E780B530B1014608222A48FDF700
:102F100030FD002000E0122000F003F840F663408E
:102F2000C1E78DF800006A460121704780B542F282
:102F300013010C20FFF718FF002002BD80B51D21F2
:102F40008DF8001004218DF8011010B9FFF710FF63
:102F500000E011208DF802006A4603214FF61D4063
:102F60000DE080B51C208DF800006A4604208DF825
:102F7000010003210C208DF802004FF61C4005F0E3
:102F8000EDFF002002BD05F03FBD80B530B10B491B
:102F900002780A7040784870002000E01220FFF7A5
:102FA000C0FF42F201007EE7244F0020264F0020A0
:102FB000284300202A430020C4480020BC480020A9
:102FC00000B585B06A460DF1020101A8FFF7D4FEF5
:102FD0008DF80800222107208DF8090002AA02A816
:102FE000817002218DF80B109DF804108DF80C10E3
:102FF000BDF802108DF80D10090A8DF80E10BDF8FD
:103000000010C171090A017241F201000921FFF7A4
:10301000A7FE002005B000BD10B582B004460DF13A
:10302000030105F0BEFC8DF800008DF80140200A78
:103030008DF802006A46042141F20540FFF790FE38
:10304000002016BD000000800000C000000000E469
:103050000000002822000000000000040000F7C368
:10306000B37E00000000000000000000000000002F
:103070000000000000000000000000000000000050
:1030800000000000000000007CB5164600244FF44C
:103090008063C21ADFF8105C21D0521E26D0521E67
:1030A00029D0521E2ED0521E33D0521E38D0521E5E
:1030B0003FD0521E44D0521E47D0521E4ED0521EF8
:1030C00074D0521E79D0521E00F07E80521E00F045
:1030D0008380D21E4DD0083A00F08A8090E001290A
:1030E00011D1307803280ADA687393E002290AD1F3
:1030F000308828858EE0012905D1307802287DDAD4
:10310000A87387E0012979D13078052876DAE87349
:1031100080E0012972D1307802286FDA287479E0D2
:1031200010296BD11022314605F13C00FDF721FC3E
:1031300070E0012962D1307802285FDA687469E0B2
:1031400001295BD13078287564E0042956D13068B4
:10315000DFF8B01C884251D2E8625BE000294DD113
:1031600003F00CFA10B900F076FC17E00120E875C6
:1031700050E0072942D10622711C6846FDF703FC86
:1031800030780022694600F060F906460A2E40DADF
:1031900003F0F4F930B9304600F069FC502001F03A
:1031A00089F822E0A9190120087733E0012925D107
:1031B0003078022822DAA8742CE001291ED1307858
:1031C0000A281BDAE87425E0012917D13078C11FDD
:1031D0000A2913D268751DE001290FD1A97D307825
:1031E000A875002908BF012814D100F0D8FB11E010
:1031F000012903D116B1307868760BE0182409E074
:10320000282806DA022904D1318802F073F804462E
:1032100000E00224204676BD38B500244FF48063D8
:103220000D46C21ADFF8801A1CD0521E1CD0521E46
:103230001CD0521E1CD0521E1CD0521E1CD0521E1E
:1032400020D0521E20D0521E20D0921E21D0521EBD
:1032500021D0521E21D0521E21D0521E21D00A3A16
:1032600022D024E0487B20E0088D24E0887B1CE00D
:10327000C87B1AE0087C18E010223C312846FDF794
:1032800078FB1BE0487C10E0087D0EE0C86A2860EF
:1032900014E0887C09E0C87C07E0487D05E0887D73
:1032A00003E000F0C5FB00E0487E287006E0282817
:1032B00003DA02F02CF8288000E00224204632BD18
:1032C0002DE9F04F93B0914698460AAA0023C2E92F
:1032D0000033DFF8D47900F0B8F88246BAF10A0F6B
:1032E00071DA4FF0060B0BFB0AF404F1200000F03A
:1032F0007FF80028787B0CBF9DF80D500025022830
:103300000CBF01260026B8F1080F0BFB0AF004D110
:10331000290758BF00F1220B01D500F1210B1C2217
:1033200000210CA8FDF757FB0CAA1C215FFA8BF0BB
:1033300000F0A2FF05F0010558B99DF84A00C01F32
:103340000A2806D200960CAB00222946484602F015
:10335000F4FA1422002101A8FDF73DFB04F124003A
:1033600001AA00F0D1F880B91022FF2101A8FDF7D1
:10337000FEFD50B904F1250005AA042100F0C5F8AE
:1033800001AA2946484602F017FA0AF1700006AA77
:1033900000F0BAF8A0B906A800F040FA002406AD83
:1033A000204635F8201041B106A901EB80018A784A
:1033B00035F820104846FEF727FF641C042CEFDB8D
:1033C000504600F010FBB8F1040F04BF787B0228D0
:1033D0000AD1797C002001B10120B97B01B104211F
:1033E0000143484602F046FE002013B0BDE8F08FCE
:1033F0006A460E21C0B200F03FBF70B503F0BEF8C0
:1034000010BBDFF8A448E07D01280AD100F023FBBF
:103410000020E0750A22002104F11C00FDF7DBFA10
:103420000CE000256619307F012804D1284600F001
:103430001EFB002030776D1C0A2DF3DB502000F0BE
:1034400039FFBDE87040AAE270BD2DE9FF41164684
:103450000D460A246A79022102F0C002C02A08BF80
:10346000002102D0402A08BF0121020018BF022813
:1034700003D0032818BF00290DD1284600F07AFA9E
:1034800004460A2C3CDA002E3AD006222946304661
:10349000FDF76FFA34E0022910D10027DFF88089A8
:1034A0000E207843404406222946C01DFDF785FAC8
:1034B000F0B97F1CFFB20A2FF2DB21E001291FD1F6
:1034C00000270620784323306A4600F01DF850B9E3
:1034D0001022FF216846FDF74AFD20B929466846BB
:1034E00002F070FD20B17F1CFFB20A2FE9DB07E07C
:1034F0000A2F3C4604DA1EB13146204600F023FA7A
:10350000204604B0BDE8F0811021C0B200F0B4BE86
:10351000F8B50C4615264FF6FF71884215460BD1BB
:1035200000272A462146384600F021F900B100263E
:103530007F1C0A2FF5DB10E003F0D9F960B1811D83
:1035400040790022FFF781FF0A2806DA2A46214641
:1035500000F00DF9002600E014263046F2BD10B54B
:10356000DFF84447217B2063262001F0C3FE207B47
:10357000BDE81040FDF7CABE38B504460025080076
:103580000DD1DFF88008DFF87C38B2FBF0F021467F
:1035900003FB102002F0ABF9050003D00121204607
:1035A00002F07CF9284632BDF0B585B0DFF8F85658
:1035B0000446A178286B062900F0CB80092900F089
:1035C00088800A2920D00B2905D00E2979D00F290F
:1035D00000F08E80C0E050B10668300007D020694E
:1035E0000090637B227B6189E01CB047B4E02069D6
:1035F0006189002814BF0120E86A02F078F90028E8
:10360000F4D06089012191E060780026002846D13D
:10361000A079C00743D5686B002840D10E2200F086
:10362000A2F8A08803F063F90600DFD06769CFB184
:10363000387C8DF80600062207F111016846FDF777
:1036400098F90622B11D06F10C00FDF792F9062249
:1036500007F11101B01DFDF78CF9387C40F0020034
:10366000707107E070798DF806000622B11D68467A
:10367000FDF77FF9A1799DF80D00890801F001019E
:1036800008438DF80D002146684600F0D6F828B9A9
:10369000287B0221FDF7B3FA00205EE01526286B97
:1036A000002859D04368180056D06278A0880121BC
:1036B0009847300050D02B6BA0885B6832460321BE
:1036C00045E0002848D04368180045D062780221C0
:1036D0003CE0E0780022211DFFF7B7FE0A283BDA24
:1036E00006235843253004F10C0200F038F833E08B
:1036F000A088A97C09B1E97C18E0697B09B905219A
:1037000014E003F0F4F8060026D0A07AC00710D524
:10371000707901000DD0E168C1F3402149B96A46D2
:10372000B11DFFF792FE20B9A088032102F0B6F880
:1037300012E07179A08804F1080200F0E1FA286B28
:1037400050B14368180007D000220021A088984794
:1037500002E0A088FFF751FE012005B0F0BD042172
:10376000C0B200F099BD00216846FDF734B970B5CC
:1037700006460620704388B00C461546203004AA41
:10378000FFF737FE002838D10622FF2104A8FDF7F5
:10379000EEFB90BB70366A461021F0B200F06CFD73
:1037A00048BB684600F03AF8200009D110220021F9
:1037B0006846FDF7DCFBF0B91022FFF7D4FF12E0FA
:1037C000694600F01DF838B9280016D06946002077
:1037D00000F016F888B104808178A9420BD085707A
:1037E0000DB900210180684600F018F86A461021E2
:1037F000F0B200F051FD012000E0002008B070BDE3
:10380000002231F82230834202D101EB820070475E
:10381000521CD2B2042AF4DB00207047002130F899
:103820002120D24320F8212000EB8102491C93780B
:10383000DB4304299370F2DB70472DE9F043DFF896
:103840006844DFF8DC958046606B85B00F460E2635
:10385000E8B9B8F1000F18BF002F70D0404600F053
:1038600089F80A28207612DB002506FB05F00622DF
:10387000FF214844FDF77BFB40B96D1CEDB20A2DDA
:10388000F3DB607E002814BF25780A252576207E8C
:103890000A2854DA0625616B6843C9B920304246CC
:1038A0000E21FFF75DFF207E00F09DF81022FF2122
:1038B000FFF75AFF207E703000F046F9207E7043FB
:1038C0000E2241464844FDF754F86763002037E074
:1038D0008A683AB121301C21FFF742FF616B00205A
:1038E0008860F3E70A693AB122301C21FFF738FFFC
:1038F000616B00200861E9E74A693AB12330102181
:10390000FFF72EFF616B00204861DFE7CA6882B1D4
:1039100024301021FFF724FF606BC06800F1100213
:10392000207E68432530FFF71AFF616B0020C860D6
:10393000CCE7A07D08B100F04CFA00F0D2F90120EC
:1039400005B0BDE8F08330B50A2885B00C4600DA32
:103950000CB902200CE0062358432030FFF748FD45
:10396000050004D1062269462046FDF702F82846E4
:1039700005B030BD70B504460025DFF8A4640E2004
:103980006843062221463044FDF717F808B128465F
:1039900070BD6D1CEDB20A2DF1DB0A2070BD38B58B
:1039A000002400F029FA0620604320302A460E2128
:1039B000C0B200F061FC58B10622FF212846FDF795
:1039C0000AF80622FF21E81DFDF705F800206873BC
:1039D000641C0A2CE5DBB448807D08B100F0F9F9DD
:1039E000BDE831407DE138B50A210A23AE4A5C1EAC
:1039F000DBB2134413F8013C834201D1214603E0BA
:103A00002346E4B2002CF2D1C9B2084605E01418EE
:103A1000135C657815546370401C0928F7DB09298D
:103A200005DABDE838400A21052000F035BC31BD7B
:103A300070B500240025DFF8E8630E2068430622F5
:103A4000FF213044FDF793FA00B9641C6D1C0A2D68
:103A5000F3DBE0B270BD10B50024204600F007F89B
:103A6000641CE4B20A2C01DA0100F6D010BD2DE985
:103A7000F0478D4D297E884290B0814609D1287B40
:103A80000121FDF70BF9287B0221FDF707F900F072
:103A9000BBF9062000FB09F505F1200607AA0E2157
:103AA000F0B200F0E9FB002845D10622FF2107A86B
:103AB000FDF75DFA00283ED11C22FF21FFF754FEDE
:103AC0001022FF210BA8FCF786FF0E22FF2107A87A
:103AD000FCF781FF07AA0E21F0B200F0DDFB0646DD
:103AE00005F1210000F02BF8824605F1220000F0DC
:103AF00026F8804605F1230000F026F8044605F17B
:103B0000240000F021F8074605F125006A4604214B
:103B1000C0B200F0C1FB48EA0A012143394340EA40
:103B2000010509F170000BAA1021C0B200F0B4FB2E
:103B30002843304300E0002010B0BDE8F0876A461B
:103B40001C21C0B200F0A8BB6A461021C0B200F030
:103B5000A3BB10B5B34C207304F14C0002F0FBFD85
:103B6000FFF71DFF22460A21052000F085FB30B13A
:103B70000020C0F109012154401C0A28F9DB10BDC6
:103B8000F0B50D46280485B0474C25D5207BFCF7C1
:103B9000BEFF04001DD021780120B0290FD0B1292B
:103BA00005D0D02904BF2046FFF7FEFC0DE02079A8
:103BB00060B92289E1886088FFF7AAFC06E02179D4
:103BC00004F1080000F000FD00E010B12046FCF711
:103BD00031FF85F4004065E0A80709D500210020E9
:103BE000FFF72BFE002885F0020550D102214FE09F
:103BF000E80752D5606B8688A06B4FF6FF7748B90F
:103C000004F12A0000900223874A39460120FEF77A
:103C100042FCA06385F00105A16B21B3FF20039056
:103C200002200290002001900DF11200009004ABE0
:103C3000628D3046FEF7A8F968B99DF810009DF82E
:103C4000111000EB012290B228B1A06B418992B211
:103C50003046FFF75DFC628DA06B00233946FEF70E
:103C60006FFCA06398B9206B70B1436818000BD04B
:103C7000606B8088002201219847606B236B8088ED
:103C80005B6800220321984700F0BEF803E00121A1
:103C9000207BFCF7B4FF284604E068074CBF85F0A2
:103CA0000400002005B0F0BD4844002010B52038C5
:103CB000062390FBF3F30624012204FB13000528DE
:103CC0000DD8DFE800F00305050707090E2904E019
:103CD0001C2902E0102900E0042908BF0022104638
:103CE00010BD80B5FFF7A4FE0228ACBF02200A2059
:103CF0008DF800006A460121052002F043FA01BD5B
:103D000070B5AAB006460C46154602F0F0FD08B99B
:103D100014205CE0A422FFF726FDADF80060414EC0
:103D2000F07B317D8DF8040001F00102707D8DF88B
:103D3000A0002798400842EA400020F0020248080C
:103D400000F0010042EA400020F48072080900F00F
:103D5000010042EA002020F40072480900F001004E
:103D600042EA402020F48062880900F0010042EA23
:103D70008020890820F0040001F0010140EA810060
:103D8000279001A9307C020008D04870102206F16B
:103D90003C010DF10600FCF7ECFD01E0002048704D
:103DA000707C28B11CB1279840F0020027900120B8
:103DB0009DF899100843B17B8DF8990001B1042159
:103DC00008438DF899002946684601F019FD2AB08C
:103DD00070BD38B5FCF778F8002400F00DF8062225
:103DE000FF212846FDF7C3F810B92946FCF770F803
:103DF000641C0A2CF1DB31BD0E21094861434518D2
:103E00007047000040420F0010B5064C606B18B1BF
:103E1000FCF710FE002060630A20207610BD000031
:103E20004847002048440020A4CC0100002010B5E1
:103E3000DFF828446070207082B000F004F900219F
:103E400000F0FEF80098B0F5801F02D100F0E3F812
:103E50000BE020B900F0DFF800F01DF905E000F0FC
:103E6000BDF800F0ABF804206080607816BD38B56E
:103E7000DFF8E8432578290001D0012032BD6188B0
:103E8000C1F5805189B2814200D350B900F09EF84B
:103E90000020607000F0FFF818B96578280008BFAE
:103EA0000125284632BD13B5DFF8B003BDF8021076
:103EB00040881C46C9B200F0CBF8010009D0DFF8F9
:103EC000A003049A0003A3B2000E05F0C1F800207D
:103ED00016BD012016BD2DE9FB43DFF8806382B0DB
:103EE000002070701746BDF80A90708898465FFAF7
:103EF00089F100F0ADF80446B8B1002501E0641C7A
:103F00006D1CEDB2B9B28D420CD2D548000301232D
:103F100001AAA1B200F094F89DF8040018F8051069
:103F20008842ECD0B8B285423ED0BFB2F81C4110F6
:103F300000EB9170801087007088BFB23818001DA8
:103F4000B0F5805F03DD00F041F800F0A4F874885C
:103F50004FF6FF70ADF800003D1947F4004000F047
:103F600027F8BDF80200C0F30E0000F021F8BA05F2
:103F7000120E4146204600F016F95FFA89F141F42D
:103F80000040ADF8000000F015F8BDF80000C0F3E7
:103F90000E00ADF8000000F00DF87078010004D1BB
:103FA0007088391D08187080002005B0BDE8F083C6
:103FB000ADF8020001226946A8B2F4E080B54FF4E2
:103FC0008010009001226946002004E080B50020A6
:103FD00000900122694600F0E6F801BD70B5A148E5
:103FE00000688047044600F023F905469C4800031A
:103FF0000021000E05F04DF805F056F8064628465B
:1040000000F00EF90EB100F006F92046BDE8704050
:1040100095490968084710B582B040F6FC7400F075
:1040200012F8214600F00CF8009810F1010F03D1AE
:10403000241FA4B2042CF2DA8849201D488013BD45
:10404000000E05F005B88648000304236A46704751
:1040500038B50C46051F00E02D1FADB2042D18DB4E
:10406000FFF7F1FF2946FFF7EBFFBDF80010BDF8A1
:104070000200A14203D1C0B2281A80B232BD0104AD
:10408000EAD4011D8D42A8BF281AE3DA002002F00D
:10409000E0FC002032BD2DE9F04F83B000F0C8F8FD
:1040A0006E4FDFF8BC9183467888041F4FF0FF08FD
:1040B0000025A4B24FEA193A2DE04FF0885081193B
:1040C000042201A805F006F8BDF804005FFA88F1A3
:1040D00088421BD0BDF80600301A061FB6B2301F4A
:1040E00040F6FC718842E8D3BDF802004FF08851D9
:1040F0004A19031D211A9BB289B25FFA8AF004F0B3
:10410000A7FFBDF802004019051DADB2BDF80200C1
:10411000201A041FA4B2042C2ADB04236A46214679
:104120005FFA8AF004F094FFBDF800004FF6FF71CB
:10413000884218BF002810D1BDF80200010448BF12
:10414000241FE7D4001D8442E0DA002002F081FC45
:10415000584600F065F8002023E00004D6D4BDF8EE
:1041600000005FFA88F18842D0D080462E1FB5E764
:10417000FFF734FF45B12A464FF0885109F104009A
:1041800004F082FFFFF71AFF584600F049F87878EC
:1041900028B9281D7880C5F5805080B201E0002044
:1041A0007880BDE8FE8F2DE9F04705462C480E4685
:1041B000040B82B017462946E0B204F06AFF81463C
:1041C000284800688047804600F032F88246BA00EE
:1041D0003146484604F058FF504600F021F801E00F
:1041E0002D1D361D3846471EC0B270B104236A46E5
:1041F000A9B2E0B204F02CFF04223146684604F074
:10420000A5FF0028ECD000F006F8404616490968E2
:104210008847BDE8F387114801214170017070475C
:1042200028B1124A1248126852680121104770479B
:1042300038B50F4C204604F0BBFF0546C0B250B164
:104240000A4A12685268002120469047204604F02E
:10425000AFFF0028FAD1E8B232BD0000F8460020D6
:1042600000E00100DC470020E0470020D8010010FA
:10427000004003400020D9E5E0B5ADF806000B464C
:104280000020ADF808008DF804000092DDE901017E
:104290000022FFF708FE0EBD82B01346ADF8020003
:1042A0000A460020ADF804008DF80000DDE90001A9
:1042B00002B010E6652807DA0003642190FBF1F0F4
:1042C000C0F5805080B2D2E504207047DFF800F0DE
:1042D0000158001080B502216846FFF7F7FFBDF8CE
:1042E000000002BD704770478149086070478149EE
:1042F00008707047032290FBF2F080B2FCF7D1BE49
:104300000178B02904BF417800290CD10179122924
:1043100003D1417C012906D101E01B2903D140884A
:104320000121FCF7DBBE704710B5734C607002F0E2
:1043300037FB401C207004216078FCF747FEBDE885
:104340001040FDF7BDBF38B50C46200411D56A48B2
:104350004078FCF7DCFB050008D02878A02804BFD3
:10436000284600F008F82846FCF764FB84F4004077
:1043700032BD002032BD30B587B0044601208DF833
:10438000000001A9204602F00BFE05002AD19DF88D
:1043900006105748C9070AD54368180005D0608839
:1043A0006A4601A9984705461CE006251AE00368FD
:1043B000180006D060886A4601A99847050001D117
:1043C00010E006259DF8050060B99DF806008DF8FF
:1043D00010008DF814500020ADF8120004A9608878
:1043E000FCF7A1FE9DF8000000281EBFA068002871
:1043F00000F0F7FB45B99DF80600122806BF9DF8AE
:10440000051001291B2803D060880121FCF766FEF6
:1044100007B030BD2DE9F0410446FF2C0D4616468D
:1044200098461FD02020FCF7F3FA070018D0B020E0
:1044300038707E707D8087F80480069929B1182233
:1044400007F10800FCF795FA04E0182207F10800CC
:10445000FCF7C1FA39462046FCF7FBFA002002E0DF
:10446000132000E00220BDE8F08110B54FF47A740B
:104470006243BDE8104004F0EABE10B504001EBF60
:104480002078FF28FE2803D004F0E9FEFF202070EA
:1044900010BD80B5009313460A46014615480078C2
:1044A000FFF7B8FF02BD30B583B004460D4602F0F9
:1044B00021FF50B901A80090ADF804507F230D48AA
:1044C000007800222146FFF7A5FF37BD00B583B075
:1044D0007E238DF804108DF8052001A9009100229B
:1044E000014604480078FFF795FF07BD0000000073
:1044F00044480020FF460020DD480020052923D045
:1045000006291BD0072918BF09291DD00B2918BF60
:104510000D2919D00E2913D00F291CBF11291229DA
:1045200012D0162918BF17290CD01B2918BF1D2916
:104530000AD0522918BFD22906D007E0C0687047B8
:104540000068704780687047406870470020704777
:1045500070B5052914461D4616D0062912D0092922
:1045600018BF112910D0122912D0162918BF1729E7
:104570000CD01B2918BF1D290AD0522918BFD229D7
:1045800006D007E0072606E0022604E0052602E042
:10459000032600E001264FF6FF72944203D102F099
:1045A000BEFE841B02E0D22908BF0C34301980B251
:1045B00000F0F2FA38B105B12C807142BDE87040CC
:1045C00009B200F033BB70BD80B5FFF797FF18B19B
:1045D000BDE8024000F005BB01BD0000DFF800F0BF
:1045E000E9940010DFF800F0A19400100A7802703E
:1045F0004A7842708A78C97802EB0121418070477D
:104600002DE9FC410D4616461F460A9A09990446B3
:1046100001AB00F0F0F9804608BB019908980870DA
:104620003346DFF858050178491CCAB2002A06BF94
:10463000012101220A460170294601980271009762
:1046400001980279204600F00DF8804620B90198C3
:104650001E2100F015FA02E0019800F0F5F940463D
:10466000BDE8F6812DE9F041044684B00E461746B8
:104670009846172000F090FA050026D00A9A1000FC
:1046800003D04146281D904700E00020010A2E700B
:10469000E9706F70A8700521001DADF80800ADF835
:1046A000001001956946DFF8D804007800282046FC
:1046B00002D000F059F801E000F00CF804462000A8
:1046C00004D0284600F08DFA00E01324204604B000
:1046D000BDE8F08110B50B88DFF8A8240C246343F3
:1046E0001A44303A536833B94B6853600989508192
:1046F0001181002010BD162010BD80B5052000F0EE
:104700000FF858B9062000F00BF838B9042000F073
:1047100007F818B9072000F003F800B1012002BD26
:104720000C2210B5DFF85C1442431144A1F13004AF
:1047300084B06168A9B1DFF8482412787AB1ADF885
:104740000000019169462089ADF80800608900F0F9
:104750000BF810B1606800F044FA0020606001209E
:1047600000E0002004B010BD70B50D460446288955
:10477000010004D0DFF810140988814201D21B2007
:1047800070BD6868042100F051FA0646288930702F
:104790002889000A70702888B0702888000AF07094
:1047A0002889051D4FF6FE70844213D10C20FCF7BA
:1047B0002FF901000CD0902008704C800220087165
:1047C000CD808E60DFF8C4030078FCF742F918E072
:1047D000132070BD3346AAB200212046FFF7FEFE2B
:1047E000010007D002280ED0072810D012280CD0C4
:1047F0001F280DD1DFF8880301780A001CBF491E6D
:104800000170002070BD142070BD022070BD042016
:1048100070BD38B50446002060600879022821D1B7
:10482000CA88042A1EDB886801784378C57801EBC2
:104830000321837889B203EB05230D1D95429BB2BA
:1048400010D1052B18BF042B03D0062B18BF072B44
:1048500008D1218123806FF0030100F0E7F9606047
:10486000002032BD012032BD0B88037002220B886C
:104870001B0A43700B88012B06D14A8882700422E0
:104880004988090AC1700CE0022B0AD14A8882705B
:104890004A88120AC2708A88027106228988090A27
:1048A000417110467047022A1BDB0A784B7802EBF5
:1048B000032202800288012A05D18A78C97802EB96
:1048C000012141800BE0022A09D18A78CB7802EBE2
:1048D000032242800A79497902EB0121818000207C
:1048E0007047012070470A8802700A88120A4270D5
:1048F0004A8882704A88120AC2708A8802718A883D
:10490000120A4271CA888271C988090AC1710820D5
:104910007047082A18D10A784B7802EB03220280EC
:1049200011F8022F4B7802EB0322428011F8022F7C
:104930004B7802EB0322828011F8022F497802EBB8
:104940000121C1800020704701207047022A00D158
:1049500001E0012070470A78497802EB01210180CB
:1049600000207047F8B504460D4616461020FCF7A7
:104970004FF8070016D0A02038707D800020787096
:104980002EB10C223146381DFBF7F3FF04E00C2258
:104990000021381DFCF71FF839462046FCF759F86E
:1049A0000020F2BD0120F2BD2DE9F04180460D4608
:1049B00016461F462020FCF72BF8040019D0A22031
:1049C000207066706580069820716771079929B11B
:1049D000182204F10800FBF7CCFF04E0182204F1D0
:1049E0000800FBF7F8FF21464046BDE8F041FCF720
:1049F00030B8BDE8F08170B51E0004460D4621D0E8
:104A0000012101F0A2FFD8B161480078002100E047
:104A1000491CC9B2814211DA5E4B1B6803EB0112DB
:104A20005388002BF4D10020107001F14000508019
:104A300022B1D48015723260002070BD152070BD87
:104A4000142070BD012070BD10B504461022002155
:104A5000FBF7C1FF23E0002200E0521C4C4909781B
:104A60008A420BDA4B49096801EB02114B88002B93
:104A7000F3D00B798342F0D108467047002070478D
:104A80004FF47A724A4300F1090301460FF219000C
:104A900004F0DDBB10B50446607A04F0E0FBFF20B3
:104AA000607210BD0000000010B504001CBF6088DB
:104AB000002807D01721204600F005F82046BDE861
:104AC0001040C1E710BD1CB50446207804280FD162
:104AD0000020019000900A46E188207A1323FFF716
:104AE00063FFE18802B0BDE81040122205202EE0ED
:104AF00013BD072170B50446002539BB18E02548D1
:104B00000068EDB200EB0516307800281CBF707A03
:104B1000FF280CD0F088A04209D13046FFF7BAFF39
:104B200014213046FFF7CFFF3046FFF78DFF6D1C95
:104B300017490978E8B28842E1D30425FF222146CB
:104B4000284600F004F86D1C082DF7DB70BD10B589
:104B50000C240C4B60431844A0F130046089884257
:104B60000AD1606840B1FF2A1CBF0178914203D18D
:104B700000F037F80020606010BD0000E048002021
:104B8000E64600208C480020FC460020E446002039
:104B9000E5460020E846002080B5001D80B2FFF702
:104BA00021FD28B1BDE804406FF0030100F03EB8DC
:104BB00002BD000070B500F035F8054604F10800AC
:104BC00080B201F071FF060005D02A48B480016868
:104BD000316006600836284909682846884730460B
:104BE00070BD38B500F01EF8224A05461068002155
:104BF00001E00146006878B100F108039C4221BF42
:104C00008388C3180833A342F3D3036800290CBF79
:104C100013600B6001F055FF2846BDE8344016498B
:104C200009680847044615480068004738B5044637
:104C30000D4600F00FF801000AD06842204401F14F
:104C40000803984221BF8B88C9180831814200D2DD
:104C5000204632BD0749096841B101F1080290427E
:104C600021BF8A888A1808328242F4D308467047E6
:104C700000000000E4470020E0470020DC4700205F
:104C800038B50225012918BF04291C4610D100F0AF
:104C900047FB05000CD10599049800F055FB204610
:104CA00000F05FFB00F03DF901F001FA04F05AFB5F
:104CB000284632BDDFF800F0A1980010DFF800F0C0
:104CC000BD980010DFF800F0D9980010DFF800F070
:104CD0006D98001070B5DFF8F065054630680C4639
:104CE00008B1112070BD00F0E7F801D1122070BDAD
:104CF000DFF8D805806800281CBF0078002801D1A3
:104D0000102070BD0C2001F0CFFE306040B30120B8
:104D100001F095F9306805700021306841700A2271
:104D20002146801CFBF725FE00F0C4F9040002D0E8
:104D300000F0A9FA15E0DFF898050078032810D1F3
:104D40001D2000F0E4FADFF88C15088048B1DFF888
:104D5000880500784EF66022042101F07BFF00E018
:104D60001324204670BDF8B50C46DFF8701509789D
:104D70001546052211421E4627D0012CDFF84C159E
:104D800002D18F680FB301E0CF68F7B1202D02DAAE
:104D90002A0002D00EB90220F2BD08701F220021A5
:104DA000781CFBF718FE2A463146781CFBF7E1FD1C
:104DB0003D70284624B1791CBDE8F440FFF77ABF66
:104DC000791CBDE8F440FFF779BF1220F2BD38B579
:104DD000DFF8F444216809B9122032BD0978814214
:104DE00001D0032032BDDFF8F0542878022101F011
:104DF0004BFFDFF8D814002048800421287801F008
:104E000043FFDFF8D0140020088003202168487099
:104E10000020BDE83240FFF755BFF8B5044600F06A
:104E20004BF801D11220F2BD1CB1207801F0D3F86B
:104E300008B90220F2BD6078801C202823DA20788F
:104E400000F0A3F908B11820F2BDDFF880546B68B8
:104E50000021002202E0B61C71181B685BB15E687D
:104E6000767828B9C9B27718BF1C202FF3DB012050
:104E7000B61CB218F1E7D0B238B16078D2B280185F
:104E8000801C202801DB0B20F2BD082001F00CFE65
:104E900006000FD0082200F07CF8686830B100E00E
:104EA000084601680029FBD1066000E06E6074606E
:104EB0000020F2BD1320F2BDDFF8200400780521A8
:104EC0000842704710B500F01CF801D1002010BD59
:104ED000DFF8F8335968002201E00A46096869B131
:104EE0004C6824788442F8D14C680868002A14BFC2
:104EF00010605860084601F0E4FD00E00024204600
:104F000010BDDFF8D8130978052211427047DFF889
:104F1000CC0300780521084218BF00F043B91220E5
:104F2000704770B5DFF8A443A06818B101F0C9FD5F
:104F30000020A060E06818B101F0C3FD0020E0602F
:104F40000521DFF89853287808421CD004F110009E
:104F500001F0FEFB287800260521084211D000F060
:104F600077F9A06060B100F013F800F071F9E0602B
:104F700010B100F00DF804E0A06801F0A2FDA660F9
:104F80001326304670BD002001F0E2FB002070BD0A
:104F900020220021FBF71FBD2DE9F0478288DFF8B2
:104FA0002863DFF82853316842F20607D31B4FF01D
:104FB000010805D09B1E012B60D99B1E0FD00BE072
:104FC0008068007841B1020003D101204870FFF7EA
:104FD00079FE01006BD038E04FF0000867E0806890
:104FE00007780029F8D04878BD4C012833D100F06B
:104FF00058F9DFF8E492B0B1012000F088F9824658
:10500000BAF1420F0AD399F800004EF6602202214D
:1050100001F020FEAAF13C00688010E04FF47A70A5
:1050200000FB0AFA02E000F072F98246BAF1000FC2
:1050300005D099F800005246022101F0F3FD3168D5
:1050400002204870207818B9384600F004F92EE0A4
:10505000002020702BE0207848BB0320FBF7D8FC11
:1050600048B1D02101704770042181700146306839
:105070000078FBF7EEFC00F006F918E0806807788E
:10508000287842F208018A420CBF01260026FF2838
:105090000DD00420FBF7BCFC010008D0D020087024
:1050A0004F7002208870CE702878FBF7D2FC404603
:1050B000BDE8F087F0B5844F386885B070B3847868
:1050C00001F05CFA28B10A2000F021F905460B2016
:1050D0000DE000F0E6F828B1062000F018F90546CA
:1050E000072004E0082000F012F90546092000F02E
:1050F0000EF906467648007800F01BFA3968CA7A3D
:10510000039203468A7A029228460A1D0192224699
:10511000C97800913146FFF7D9FD00E0012005B0C4
:10512000F0BD38B5014668486B4D02682878674C79
:1051300001291ED161880B0002D0694B1B7823B175
:1051400012B31078BDE8324041E63C29A8BFA1F176
:105150003C000CDA022101F097FD60884FF47A716F
:1051600001FB00F22878022101F05CFD0020608044
:1051700031BD4AB159490978490705D5022101F0E5
:1051800083FD002060807CE031BD5049496800E02B
:10519000096829B14A6812788242F9D108467047F5
:1051A00000207047F8B54D480078002405210842DA
:1051B00001D11220F2BD454DA86810B900F048F8A1
:1051C000A860E86810B900F043F8E860A868002813
:1051D0001CBFE968002901D11320F2BDFFF7D8FEFA
:1051E000E868FFF7D5FE6E6812E09B1C501859184E
:1051F000401C117071684978491C01707168097808
:105200004170801C71684A784968FBF7B2FB3668C8
:10521000AA6896B13CB97068117843785F18BF1CD2
:10522000202FE2DB01247368E9685B780A789B1C15
:1052300088189A18401C0A70DCE71078511CFFF798
:1052400039FDE868411C0078FFF738FD0020F2BD09
:10525000202001F029BC38B51B4D0446286878B1E0
:105260000320FBF7D5FB48B1D02101704470032126
:105270008170014628680078FBF7EBFB04B100E081
:1052800031BDBDE8314010B50F4C206840B101F090
:1052900018FC002020600120BDE8104000F0D4BEC2
:1052A00010BD80B50948806858B10278431C694632
:1052B000012000F09AFE20B10078C00701D501203E
:1052C00002BD002002BD000018480020DC4500207F
:1052D0007E45002080450020F84500207D450020C7
:1052E0007F450020DFF800F049980010DFF800F05B
:1052F000C9560010282808DA4FF6FF72914204D0F0
:10530000CA4A22F81010002070470220704728284F
:1053100003DAC64931F8100070474FF6FF70704746
:1053200070B504460D46C24E1C2200213046FBF7E4
:1053300052FB34777577FAF7B7FD01000EBF0121F4
:1053400000211220317070BD10B5B94CE160A06031
:1053500010220021FBF70BFE012801D1A0680CE010
:1053600010BD10B5B24C606010220021FBF7FFFDAC
:10537000012801D1606800E010BDBDE81040102197
:1053800004F0B3BBAA48406870472DE9FC41A84D22
:105390000446002695F81E80042C0F4624DA28784F
:1053A000032818BF102054D101F0E8F828B900F004
:1053B0000BFE10B900F00AFE08B1122049E0012CE2
:1053C00018BF022C1DD1BFB1062200216846FBF791
:1053D00002FB00F040F838B90622FF216846FBF7CF
:1053E000FAFA00F038F808B1022032E00622394615
:1053F0006846FBF7BEFA0BE00621684604F075FB31
:1054000006E0032C04D16868694604F067FA064692
:10541000884FAC770421387801F036FC00202884CE
:105420009EB9ACB1684600F05BF8064668B9032C3B
:105430000ED11D20FFF76BFF288448B138784EF657
:105440006022042101F006FC02E00EB185F81E8006
:105450003046BDE8F681062269463846FBF7ADBA0C
:1054600070B5044600252000714E05D121B10622F9
:1054700006F11000FBF77DFA307801280CD10125E8
:10548000200004D102203070FDF7FAFC04E0002077
:105490003070204600F0A8F8284670BD38B50024CA
:1054A000E0B10578624A290006D14178837801EBA2
:1054B0000321D182C0781076107802280ED1012401
:1054C000280006D103201070117ED08AFBF711FE50
:1054D00001E000201070284600F086F8204632BD1A
:1054E00010B5534CA17F81B10146062204F124007E
:1054F000FBF73FFAA07F04F1240100F008F804F163
:105500002400BDE81040FFF7EDBE002010BD79B1CA
:1055100002000DD04A79012808BF42F0C00006D031
:1055200002F03F0203284A7102D142F04000487164
:105530007047010018BF01210846704770B53C4D07
:105540000446287FFF2815D00A20FBF761FA0600E1
:1055500010D0D020307074700820B0700622A87F60
:10556000F07005F12401301DFBF703FA287F314666
:10557000FBF76FFAE87F01280FD12F48006818B1B8
:105580008068010018BF8047BDE870402948007856
:105590004EF66022042101F05DBB70BD2448806896
:1055A00070472348C068006870472148C1680A688E
:1055B000521C0A60007FFF281CBF4FF48041FBF79C
:1055C0001EBB70471A48807F704738B50446184D97
:1055D00005F11000FFF78AFE05F110001CB9A97F44
:1055E00009B105F1240032BD70B5114D0446287F84
:1055F000FF2819D00E20FBF70BFA060014D0D0209C
:10560000307074700020B070062205F11001F01C9B
:10561000FBF7AFF9E88A70813146287E3073287F26
:10562000BDE87040FBF715BA70BD00008C45002046
:1056300060450020F8450020FC450020DFF800F020
:10564000259500102DE9F041044688461227404672
:105650004FF6FE7188421646DFF84C5908D1A8690A
:1056600050B30268100027D041462046904720E002
:105670004FF6FF71884212D1A86938B10268100054
:1056800004D0414620469047070005D031462046C9
:1056900000F0BDFA07000FD12C706E700CE001F025
:1056A00026F948B10078A04205D131464046FFF7BF
:1056B000C5FF074600E003273846BDE8F08110B576
:1056C000044684B000F072F808B9022029E020886E
:1056D000012101F03AF908B9142022E0208801F0F4
:1056E00045F9042812D1DFF8C00881894FF6FF720E
:1056F000914218BF112014D1218881816188818055
:10570000A188C180E1880181218941810020029026
:10571000019020890090E388A28861882088FDF7A5
:1057200005FC04B010BD30B5044685B0208840218A
:1057300001F00BF9002836D02088ADF8040000F005
:1057400035F8002500281CBFA07A002807D10021C9
:10575000684600F0B1F9A07AF0B102251CE0912072
:105760008DF800008DF803503E208DF801000121D6
:1057700006208DF80200A088ADF808006088ADF81A
:105780000600E088ADF80A002089ADF80C008DF81D
:105790000350684600F090F920880022402101F073
:1057A00072F8284600E0122005B030BD2389E28857
:1057B000A1886088FDF7E4BA70B50C46DFF8EC17F5
:1057C0000978022918BF0129154601D1122070BDA0
:1057D0000DB9022070BD01F08AF8060001D1142035
:1057E00070BD1CB1307940F00200307110222946A2
:1057F00006F11800FBF7BDF82869B062002070BD03
:10580000F8B506000C4601D10220F2BD308801F047
:105810006EF8050001D11420F2BDDFF89007007882
:10582000022818BF012803D0A87C082802D10CB197
:105830001220F2BDDFF87077786908B11120F2BD4F
:10584000B02001F031F9786108B91320F2BDB0221F
:1058500000F0A5FA786931884180A022311D001D31
:10586000FBF787F8796902200870A87C796932888B
:1058700008280CBF012000200B1DDFF83417097821
:1058800004F040FB06461CB12146284604F00FFDFB
:10589000300018BF00F038FA3046F2BD38B5044683
:1058A0000D4601F024F808B9142032BD8DF80050DF
:1058B0006946204604F02EFC32BD38B50022A0B166
:1058C00001230624E4B2051915F8015C303D0A2DC8
:1058D0000BD203FB05220A256B43641EE5B2002DA3
:1058E000F0D11046BDE8344001E0022032BD30B5B1
:1058F00005460C4685B0204600F0F9FF08B9122095
:1059000019E0DFF8B006854228BF022013D210222A
:1059100000216846FBF75FF8280A8DF801008DF832
:105920000050280C8DF802002146280E8DF8030047
:10593000684604F02EFB05B030BDF8B50546DFF82B
:105940006C060078022818BF01280C461F4601D1BA
:105950001220F2BD0FB90220F2BD284600F0C7FFA9
:10596000060001D11420F2BDF06A08B101F0A9F8D7
:105970001C213846FBF713F80100F16201D1132016
:10598000F2BDB07C08280AD1069840B1887E00900C
:1059900001F112030A8A284604F0B4FC00E000205A
:1059A000317941F004010CB141F002013171F2BDD5
:1059B0002DE9F0410D4600F09AFF04001FD0A562CA
:1059C00000F0EAF90546C0B200B92578A66A94F855
:1059D00005801020FBF71CF8070010D0D02038708D
:1059E000062200207870A11D0920B87087F8038076
:1059F000381DFAF7BEFFFE603946E8B201E0BDE8A7
:105A0000F081BDE8F041FBF724B8F0B50C0087B099
:105A100050D0A079DFF89065002830690CBF0825C8
:105A2000042508B9DFF890050778042D08D1DFF8C0
:105A30008C05006820B1416808001CBF0020884721
:105A4000207D059004F10803608A04903946208A7D
:105A50000390E08902900195A0880090E279E078B7
:105A600000F071F8E07880B9172004900122E089F5
:105A7000039002950020019004F108000090E37962
:105A8000A188384600F0B2FEE070306908B100F03D
:105A900056F9307801000DD0717800F0B8F848B1AF
:105AA000E378312B04D0A2883178184600F079F8D9
:105AB0000020307007B0F0BD10B5044684B0A08857
:105AC00051B1002102910191A1890091638922893C
:105AD000E188FDF7ECF91FBD04B0BDE810403B21A3
:105AE000FDF7E7B970B504460026A08800F0FFFE78
:105AF00018B10678A08800F0ACFEDFF8AC54287826
:105B0000010007D0864205D1697800F080F848B1DD
:105B100000202870300005D0A379A288A0783146F3
:105B200000F03FF8686908B100F0EEF8A08800F0D6
:105B30001DFF042802BFA088A989884204BF4FF630
:105B4000FF70A88170BD2DE9F041064688461746D2
:105B50001C461620FAF75CFF050020D0D0202870E4
:105B60006E700520A870EF702CB106222146281D0A
:105B7000FAF7FFFE04E006220021281DFAF72BFFAA
:105B8000069868812946079828730898E88109983B
:105B900028820A9868820B982875404631E7BDE84C
:105BA000F081F8B504460D4616461F460820FAF760
:105BB0002FFF48B1D021017044700621817086808A
:105BC000877101462846EDE0F1BD2DE9F04105461B
:105BD0000E46174698460C20FAF71AFF040014D018
:105BE000304600F084FE08B9DFF8CC030078D021FD
:105BF000217065700721A170E570A680E780A4F888
:105C00000880069961812146FBE6BDE8F08110B568
:105C10000C4600F081FE28B140882146BDE81040C6
:105C2000FFF70CBD122010BD2DE9F84F074689463D
:105C300092461C46484600F05AFE5FEA000B1EBF23
:105C4000DFF86453696900295CD051F8A42F18204B
:105C500002B134208A6802B1143004B11C304968A2
:105C600001B1173080B2FAF7D3FE06004AD01822ED
:105C700000F095F800F090F85FEA000808BF9BF884
:105C80000080D020307077700A20B070A6F80490A1
:105C900086F806A006F118076969D1F8A40040B19A
:105CA000B7603846D1F8A41000F11C071C22FAF79F
:105CB00060FE6969D1F8AC0040B1F7603846D1F8B0
:105CC000AC1000F114071422FAF753FE3CB137610F
:105CD000384600F11C071C222146FAF74AFE686983
:105CE000D0F8A81031B177611722D0F8A810384643
:105CF000FAF73FFE31465FFA88F0FAF7AAFEBDE8F0
:105D0000F14F01E0BDE8F18F10B5A74C6069A8B173
:105D1000D0F8A40008B100F0D4FE6069D0F8A80063
:105D200008B100F0CEFE6069D0F8AC0008B100F018
:105D3000C8FE606900F0C5FE0020606110BD10B5AE
:105D4000994C206940B100F0BCFE00202061042085
:105D5000BDE8104000F078B910BDF8B504460D4616
:105D6000284600F0C4FD060015D000F015F8070025
:105D700008BF37780620FAF74BFE06000BD0062244
:105D800000F00DF8D020307074700E20B070B58027
:105D90003146F8B206E0F1BD2620FFF7B8BA00217F
:105DA000FAF719BEBDE8F440FAF753BE2DE9F843FF
:105DB00005460E4617469846304600F098FD5FEAC5
:105DC00000091ED01020FAF723FE040019D010227B
:105DD000FFF7E5FFFFF7E0FF08B999F80000D021D1
:105DE000217065700F21A170A680277284F8098048
:105DF000C0B20899A1720999E1720A99E16021463D
:105E000031E0BDE8F1832DE9F84304468846914628
:105E100000F06DFD070024D01420FAF7F9FD05000D
:105E20001FD0FFF7B9FF060008BF3E78D0202870CA
:105E3000062200206870B91D0B20A870E81CFAF734
:105E400098FD6C8118F00101C5F8109018BF012170
:105E50002973F0B218F0020118BF012169732946B5
:105E600001E0BDE8F183BDE8F443FAF7F2BD2DE9A6
:105E7000F14F90460D469946404600F038FD070028
:105E80000A9EDDF82CA0DDF830B00D9C3ED09DF8C8
:105E9000000000283AD1387940F010005FEA4971DB
:105EA0004CBF40F0020000F0FD00002E08BFBAF128
:105EB000000F08D1BBF1000F08BF002C03D100F088
:105EC000FB00387122E040F0040038713CB12069D9
:105ED000B8621022214607F11800FAF74AFD3EB1D8
:105EE00035B9F86A08B100F0ECFD1C2130460AE033
:105EF000BAF1000F0AD0012D08D1F86A08B100F0FC
:105F0000E0FD1C215046FAF74AFDF862264D68690B
:105F1000002842D086B1D0F8A40028B91C2000F097
:105F2000C3FD6969C1F8A4006869D0F8A40018B17C
:105F30001C223146FAF71DFDBBF1000F11D0686934
:105F4000D0F8A80028B9172000F0AEFD6969C1F8A3
:105F5000A8006869D0F8A80018B117225946FAF7C6
:105F600008FD8CB16869D0F8AC0028B9142000F0A5
:105F70009BFD6969C1F8AC006869D0F8AC0018B144
:105F800014222146FAF7F5FC9DF8000053464A46D4
:105F9000414601B0BDE8F04F46E6BDE8F18F084943
:105FA0000860704700000000444500207D45002047
:105FB000F845002040420F007C450020FC450020B1
:105FC0000C48002003F0A6BC264800E026480068E4
:105FD00000B101207047010001D0172801DBFF2824
:105FE00001D101207047002070472DE9F04D0D468A
:105FF00093460024BBF1200F80461F462C7003DB24
:106000000020BDE8F08D0419E0B25845F8D2E4B2A2
:106010003E5D641C002EF3D0E4B231198B45EFDBFA
:1060200017F804A05046FFF7D6FF641C0028E7D0FD
:10603000701EC2452870E6D1E4B23819E1E70B4979
:106040000A7810430870704708490A7832EA00005D
:10605000087006D10648006818B14068010018BFF2
:10606000004770471848002014480020DC480020F2
:106070001048002038B504460D4600F038FCA0B1A9
:10608000807C042801D0122032BD3748006808B156
:1060900090F899502946684603F053FD334B6A4601
:1060A0000221204604F0C5FC32BD142032BD80B56B
:1060B0002F480078400707D52E48FFF770FF2E497C
:1060C0004FF6FF70088001BDBDE802400020FFF7D9
:1060D00066BF7CB5012403280D4610D042F213019F
:1060E000884204D04FF6FF7188421ED02AE0A8787B
:1060F0000C2818BF112826D100F027F823E0E878F3
:10610000A9881D4E1A2804BF33889942F4D06A89A1
:1061100000922B89EA88FFF758FDA88831888842C9
:1061200011D14FF6FF7030800DE0687900241228FD
:1061300009D1ADF80040297968886A46FAF78CFFE2
:10614000012400E00024204676BD38B50A4C2088A2
:106150004FF6FF75A84205D008490A780849FAF7B2
:1061600082FF258031BD000058450020FBA90100B9
:106170007D4500200446002050450020F8450020C1
:1061800048450020F8B5144600250E46BC4FBD4BCF
:1061900040B1012815D0042818D006281ED00728A1
:1061A00022D02CE0162928DA1622002107F10C0053
:1061B000FAF711FC3246214607F10C00FAF7D9FB39
:1061C0001EE0022E19D12088388119E0082E14D142
:1061D00038462146082202F07DFF11E0012E0CD145
:1061E000DA6903F1280104E0012E06D1DA6B03F12C
:1061F0004801207800F030F802E0182500E0022580
:106200002846F2BD10B50B4600249D4920B1012857
:1062100008D0042809D00DE015220C311846FAF7F1
:10622000A8FB08E00889188005E01846082202F05B
:1062300051FF00E00224204610BD01460020C9079E
:1062400006D50FF248238F4810220721FBF7A8B884
:1062500070478D490860704710B50B7884074CBFB4
:1062600043F0020303F0FD0304064CBF43F0800338
:1062700003F07F0304074CBF43F0080303F0F70368
:1062800084064CBF43F0200303F0DF030B70AA2108
:10629000084203D0107840F00C0003E018B91078E1
:1062A00000F0F300107010BD2DE9F0410F461546C7
:1062B000387802281E464FF000085ED178680178D1
:1062C0004078069C01EB002080B221001CBFB0F595
:1062D000285F0B2056D14FF42851401A08D0401E99
:1062E0001AD0401E28D0401E1ED0401E2AD044E0A6
:1062F000F868FAF73CFB079A80B2031B9342B8BFD9
:10630000021B92B21019162803DA3280F8680119BC
:106310000EE04FF00D0834E0F8680088022131806B
:106320002870000A68702CE0062030800622F96888
:106330002846FAF71EFB24E001203080F868007838
:1063400028701EE0F868B0B10821318001882970FA
:106350000188090A69704188A9704188090AE970B1
:10636000818829718188090A6971C188A971C088E9
:10637000000AE87105E0308003E0A6F800804FF0E5
:1063800001084046BDE8F0812DE9FC4B0E468046F1
:1063900030780027022891461D466BD1706801783D
:1063A00040780A9CDFF8E0B001EB002080B24FF4A7
:1063B0002851401A06D0401E29D0401E4CD0401E05
:1063C00038D057E0F068FAF7D2FA80B2A04204D38E
:1063D0002919162903DB0D274DE007274BE0F36849
:1063E0002A4649461819FAF7C4FA2C19F068A4B2DB
:1063F000C4F1160200212044FAF7EDFADBF80000A0
:10640000002838D00268100035D0002121E07CBB84
:10641000022DE0D199F8000099F8011000EB01205D
:10642000F1680880DBF8000028B30268100022D071
:1064300001210EE0E4B9062DCDD1F06806224946CF
:10644000FAF797FADBF80000A8B10268100012D042
:106450000321404690470EE054B9012DBBD199F875
:106460000000010013BF0128F1680870802702E0D6
:106470000B2700E001273846BDE8F68B000000003E
:10648000204600204446002050480020A962010018
:106490008963010000000000B1494870704710B5E1
:1064A000AF4C207004F021FB2078BDE8104005219E
:1064B000FAF78CBD7CB5AA4D28780C46210419D575
:1064C000FAF725FB060084F4004411D000F058F8D8
:1064D00058B93078A22806BFA24800786878FF280B
:1064E00003D03146FAF7B5FA02E03046FAF7A2FADD
:1064F000204676BDE10709D5A86820B141680800AB
:106500001CBF0020884784F0010076BDA10709D593
:10651000686820B1416808001CBF0120884784F0EA
:10652000020076BD610727D58F4E31880A001DD045
:10653000481E308080B2E0B9FFF746FD48B18B4974
:1065400001200870686820B1416808001CBF012064
:106550008847FEF717FF694603F0C0F96846FEF763
:10656000BFFF1D20FEF7D3FE308002E0042100F0C3
:106570008BFB84F0040076BD002076BD00F0FCB9F2
:1065800038B502780124912A4FF6FF7102D0A22A71
:1065900076D07BE04278052A49D00E2A04D00F2A13
:1065A00048D03E2A69D071E082886D4941F20905E0
:1065B000531B2DD040F6F9755B1B2FD0DB1E31D05D
:1065C0005B1E08D09B1E022B05D9DB1E012B15D9A3
:1065D000DB1E08D05AE04968002958D009680A0033
:1065E00055D0884750E06249096800294FD04B6870
:1065F00019004CD0014642F20E003CE089680029A7
:1066000045D00B68190042D00146104698473BE040
:106610008068411C0078FEF723FF35E08068FEF7B4
:106620003DFF31E080680078FEF788FF2FE0FFF73C
:1066300059FA2CE0828842F20D05531B13D09B1FA0
:1066400002D09B1F0FD021E04A4B1B888B420AD0FF
:1066500049490968D9B10A68110018D0014642F2C7
:106660001300904710E04249096881B14B68190056
:106670000DD001461046984706E000F00AF803E006
:106680000246408800F04BF8044600E00024204613
:1066900032BD70B505460124A8780128014611D005
:1066A000022806D0032811D0062815D00A2809D0C0
:1066B00032E02B48806880B3416808002DD028461E
:1066C00088472AE02946FFF7A0F926E0A8882A464D
:1066D00000F025F8044620E00E20FAF799F90600AC
:1066E0001BD0A8880122402100F0CDF8D0203070C6
:1066F0003146E87870701120B070A888B080E888C2
:10670000F0802889308168897081A889B081154816
:106710000078FAF79EF900E00024204670BD70B5BD
:106720000C46154600F022F90126042804D112482F
:10673000006858B1026803E00D48006830B1426853
:10674000100003D02946204690470646304670BDCB
:10675000034948607047094908607047000000001D
:10676000F84500207C450020804500207F45002022
:106770005C450020504500200C48002010480020B7
:1067800038B5AE4C00220021204601F0F1FB207804
:106790003025684300F088F96060B8B100210AE054
:1067A00005FB01F202444FF6FF735380491C00239E
:1067B0001371D362C9B222789142F1DB002000212B
:1067C00004EB8002401C0C289160F9DB31BD0021F4
:1067D0009A4A02EB8102936813B9906000207047D7
:1067E000491CC9B20C29F3DB132070472DE9F04195
:1067F00006460C4617469846204600F078F808B141
:10680000112024E04FF6FF7000F071F805001DD054
:1068100085F8058006220699A81DFAF7AAF806222F
:10682000002105F10C00FAF7D6F86C802F712E705C
:106830000020E86200210898A8740998A8820A98A4
:10684000E882204600F0E9F8002000E01520BDE8CD
:10685000F08110B500F04BF8040012D060880121DF
:1068600000F0DBF8E06A08B100F02BF930220021DB
:106870002046FAF7B0F84FF6FF70608000202071D4
:1068800010BD022010BD38B50C46154600F02FF89B
:1068900058B10179002D14BF2143A1430171022198
:1068A000408800F0BAF8002032BD152032BD38B55E
:1068B0000C4600F01CF8050017D02879207006223D
:1068C00068796070A91DA01CFAF753F8062205F13B
:1068D0000C0104F10800FAF74CF8A87CA073A88A10
:1068E0002082E88A6082002032BD012032BD10B5CE
:1068F0000022524B00E0521C1C78D1B2A14209D2B6
:106900005968D2B23024544321444C888442F2D195
:10691000084610BD002010BDF0B5484B5C68002251
:106920004FF6FF7700E0521C19788A420BDA3021CB
:1069300001FB02F561194E88BE42F4D0655D8542C7
:10694000F1D10846F0BD0020F0BD10B50C464FF661
:10695000FE71884206D0FFF7CAFF00281CBF0079ED
:10696000204201D0012010BD002010BD80B5FFF7EE
:10697000BEFF00B1807C02BD10B5002000212F4A6F
:1069800008E05368C9B230244C4323441B7903B157
:10699000401C491C1478CBB2A342F2D3C0B210BD44
:1069A00026480078704710B50C46FFF7A0FF002876
:1069B0001CBFC18AA14202D0C482002010BD0120A8
:1069C00010BD80B5FFF793FF00B1C08A02BD70B55E
:1069D00005460C461646FFF78AFF28B94FF6FE70AB
:1069E000854218D0142070BD0179C06A28B9CA0642
:1069F00009D5C90609D40F2070BD01F01202102A72
:106A0000F7D1002EF5D0052070BD20B1807EA042C8
:106A100001D20C2070BD002070BD70B504460D463B
:106A20000026064800EB86008268100002D0294646
:106A300020469047761C0C2EF3DB70BD5448002096
:106A400002000A4A08BF0FF22100506051707047DF
:106A50007047064A010004BF5178012902D011781D
:106A60005268104770470000704700009C440020A7
:106A700000F10103810704D010F8011B89B18107DF
:106A8000FAD10268B2F10131914311F0803F04BFA5
:106A900050F8042FF6E710F8011B11B110F8011B94
:106AA000FBE7C01A70470000E0B50821ADF8001000
:106AB0000190042100F00FF808B100200EBD0298EB
:106AC0000EBD00B583B00821ADF80010019005217E
:106AD00000F001F807BDADF80210684601490968E9
:106AE00008470000D847002062F30F2262F31F42DC
:106AF000401810F0030308D0C91A1FD3DB0748BFA2
:106B000000F8012D28BF20F8022D130030B41446E0
:106B10001546103928BF20E93C00FAD8490728BF9C
:106B200020E90C0048BF40F8042D890028BF20F858
:106B3000022D48BF00F8012D30BC7047C91818BF9E
:106B400000F8012DCB0728BF00F8012D7047000089
:106B500000B583B00820ADF8000012209C490968F8
:106B6000ADF802006846884701980EBD10B5994CF3
:106B70000020A060FFF7ECFF606010BD70B5044618
:106B80000D46164600F018F808B1466070BD10209A
:106B9000FFF78AFF78B184720581466000210160A9
:106BA000C1608C490A6812B9086070BD0A46116854
:106BB0000029FBD1106070BD864A12682AB1138982
:106BC0008B4204BF937A8342F7D11046704708B1D5
:106BD0000021018170472DE9F041FFF7B9FF7D4E9B
:106BE0007D4977680C68C51BB4F57A7F14D0A4FB87
:106BF00005014FF47A72002303F08EFF4FF47A7888
:106C0000A8FB0023054608FB01331046194622461F
:106C1000002303F081FFC01970602846BDE8F041F1
:106C200003F0F2BFF8B504466A4800680D46164600
:106C300008B9FFF7D0FF69480068804700F01FF8E7
:106C400000F048F80446384688470CB10020F2BDF1
:106C50000820F2BDF8B50446604800680D461646A7
:106C6000804700F00CF804005D4918BFE660096831
:106C7000384688470CB10020F2BD0820F2BD074617
:106C800032462946204679E770B500F026F80646D8
:106C900029462046FFF790FF040018BFFFF797FF33
:106CA00000F018F8304688470CB1002070BD06206F
:106CB00070BDF8B500F011F8074629462046FFF7E9
:106CC0007BFF002600B1466800F004F8384688478C
:106CD0003046F2BD42490968704704463F480068A3
:106CE0000D4600472DE9F147DFF8F080394DD8F81F
:106CF0000000DFF8ECA081B080470246A868019947
:106D00000818A8601046DAF8001088472E68002E90
:106D10004DD00027D8F8000080478146BDF8060016
:106D20000024002804BF9DF80500002807D1307911
:106D30009DF80420904202D3801A307106E07068FA
:106D4000019981423ABF401A70607460B08858B9A6
:106D5000F08858B9F06868B1318908000AD0B07A73
:106D6000F9F74DFFF0687060B08808B9F08808B195
:106D7000308930B93068002F0CBF28603860344645
:106D800000E037463668DAF800104846884764B1B4
:106D9000A088002804BFE088002803D12189A07AB8
:106DA000F9F72DFF2046FFF78CFE002EB2D1BDE88B
:106DB000F3870848016841B10A484A680968824275
:106DC00098BF10460029F8D1704700207047000096
:106DD000D8470020FC470020B4440020DC470020B6
:106DE000E04700208EC2F52800B583B00821ADF839
:106DF00000108DF804001721ADF8021068461D49F7
:106E0000096888479DF805000EBD1B480021818058
:106E10000121017070472DE9F0410D4617490978AD
:106E200001248842064602D2134F387808B901205F
:106E30001DE01348006880478046B88804FA06F6CB
:106E40004DB920EA0601B98060B159B90020FFF7B9
:106E5000CBFF044606E010B90120FFF7C5FFB88854
:106E60003043B88040460749096888472046BDE856
:106E7000F0810000D8470020F447002018FE0000F1
:106E8000DC470020E047002030B585B014460822DA
:106E90000291ADF8002000223A490968ADF80400DB
:106EA000ADF802201D46684688479DF80C102170F9
:106EB0000499296005B030BD1CB51420FFF7F4FD1E
:106EC0003149086014220021F9F785FD002000F007
:106ED0000BFE012003F0D2FD022002F071F9032025
:106EE00003F0C2FE0420FFF7DAFA052004F012F8DE
:106EF0000620FDF719FA0720FAF70CFA0820FCF72C
:106F000028FE0920F9F74CF801AB6A460021102051
:106F1000FFF7BAFF9DF800100920F9F768FD00247B
:106F20009DF800102046F9F76AFD641C092CF7DB78
:106F300013BD10B582B004F061F8144B144A154922
:106F40005020FFF7A1FF60B10520FFF782FD082068
:106F5000ADF800000C200B490968ADF80200684646
:106F600088470D48006880470446FDF783F9F9F724
:106F7000AEFE0A49096820468847F9F7DEFE002080
:106F800016BD0000D8470020F0470020B044002084
:106F9000DB480020F70D0100DC470020E04700201F
:106FA000F8B505460C46AF892FB3AA6816783006A7
:106FB0000FD50D2F1FDB0C3FBFB2D01900903B4601
:106FC0006888012102F02EFE002814BF0220012053
:106FD00000E000202070B00900F00100607006F0B1
:106FE0003F00A070781EA08080B208B1A868401C45
:106FF000A0600020F2BD0120F2BD0A7802704A882C
:1070000042704A88120A8270097985E0022B00D109
:1070100063E00420704700BF0A8802700988090AEB
:10702000417002207047042B00D17DE0042070479E
:107030008A7802708878098801280CBF0420122001
:107040004843401C80B2704770B51E46062E144659
:1070500019DB049D2078617800EB01202880022252
:10706000A078E17800EB01206880211D02202871C2
:10707000681DF9F77EFCB01F288180B200B1A01D09
:10708000E860002070BD042070BD08888004000CFA
:10709000704710B5029C062B104612D102212171B7
:1070A0004278017801EB02212180C278817801EBDE
:1070B00002216180011D2279601DF9F75AFC002030
:1070C00010BD142B08BF1021E9D0042010BD4DE0E5
:1070D000022B00D101E0042070471078517800EBBA
:1070E000012000990880002070470888704710B57B
:1070F000022B0FDB029C207261721078517800EB3A
:1071000001202080981E608080B200B1901C6060D9
:10711000002010BD042010BDC17004207047042B56
:1071200000D101E00420704700981178537801EBFA
:10713000032101809178D27801EB02214180002067
:1071400070470888704703EBD3704008B3EB4000EA
:1071500007D15908022904DB0098818002600020D1
:107160007047042070470888704700BF4A88098824
:107170000270514389B2481C80B2704710B5042B8D
:107180000EDB00F031F8D478917801EB04214180D6
:10719000191F818089B201B1111D8160002010BDCD
:1071A000042010BD00BF0A8802700A88120A4270CB
:1071B0004A8882704A88120AC2708888001D80B28C
:1071C0007047012B04D10099107808700020704797
:1071D0000420704700BF0A8802700A88120A4270B1
:1071E0004888801C80B2704702981178547801EB6F
:1071F0000421018070472DE9F04784B080460C9D42
:107200000C4691469A4655B91720FDF7C5FC012654
:10721000050005D11324204604B0BDE8F087002600
:107220002846012700F8019B14B15146A047471C8E
:107230005FEA09600DD510214046FFF786FBD8B9FB
:10724000BFB2EA193946284602F09FFC044668B9E5
:107250000C370420ADF800000195ADF808706946C0
:107260004046F9F7C8FE00280446D4D0002ED2D0FC
:107270002846FDF7B6FCCEE71924F7E730B502291A
:1072800018BF102985B00446154603D1022B18BF3C
:10729000102B01D0002017E00A469A4203D129465C
:1072A000F9F78BFB10E01029694606D1284600F05B
:1072B0000DF810226946204604E000F007F810227D
:1072C00069462846F9F779FB05B030BD38B50400AA
:1072D0000D4618BF002D0BD010220FF26401284676
:1072E000F9F747FB2078287360786873012032BD76
:1072F000002032BD38B504464FF6FE7084420D467C
:107300000BD0172D09DBF9F7FAFE2946884204D382
:107310002046BDE83440FFF746BB012032BD80B5B2
:107320004FF6FE71884205D0FFF74BFB010005D1F7
:10733000172002BDBDE80140F9F7E1BE02BD000023
:10734000FB349B5F80000080001000000000000004
:1073500038B54FF6FF74A0420DD10020164A1378BD
:1073600098420EDA21F8204001EB80050023401CF2
:10737000AB70C0B2F3E700F00BF810B1048000214D
:10738000817031BD80B500F003F800B1807802BD96
:1073900010B5002200E0521C074C2478D3B2A3425F
:1073A00007D2D2B231F822308342F4D101EB82000D
:1073B00010BD002010BD000054480020DFF800F090
:1073C0001DB50010DFF800F03DAC0010DFF800F054
:1073D00089D10010DFF800F0C9B40010DFF800F028
:1073E00019570010DFF800F061840010DFF800F09A
:1073F0008D670010DFF800F0BD800010DFF800F0AE
:107400002D8A0010DFF800F071940010DFF800F012
:10741000A9AC0010DFF800F0E5730010DFF800F011
:1074200035A30010DFF800F0E1AC0010DFF800F049
:10743000EDAB001080B54FF49E720FF23001DFF813
:10744000E00C01F057FEDFF8080D00210170012269
:10745000DFF8001D0A7302220A70DFF8FC1CC0F876
:107460000D10DFF8081EC0F82D1001BD9904002191
:107470001905002179040021F0B5174C402161184D
:10748000C878022805D009480021016008498847CA
:10749000F0BD256E074E35606007284320662768DB
:1074A00024600E48804727603560F0BD2C110440F1
:1074B000A56500002840044010B5074CA17D0029B7
:1074C00005D10121A175480204493E398847206849
:1074D000002800D0804710BD540200218B390000E5
:1074E00010B50549054A72B6C878012802DC0120AA
:1074F0004870121D62B61047940200216D470000CB
:10750000F8B51A4E0546316B1948CC09E401002D37
:1075100011D01849097802290FD0007B044372B6B4
:107520000120154F4002B847114820380088C10992
:10753000C90704D016E0C07AF0E7407BEEE70F49B8
:107540003463CC61400AC0070CD001208003F16A8B
:10755000002D01D0014300E081430846F162074954
:10756000403948630020B84762B6F8BD8002002168
:107570008800002196020021DF3C000040400440CA
:107580000749002800D00420064A72B60978C907C6
:1075900001D0105800E0802062B640B27047000071
:1075A0006B020021586004402DE9F0410FF24C00BD
:1075B000DFF8581D2722036844688568C668076994
:1075C000D0F814C0D0F818E0D0F81C800B604C60E4
:1075D0008D60CE600F61C1F814C0C1F818E0C1F829
:1075E0001C8020302031521EE5D14268836800683B
:1075F00008604A608B60BDE8F081000054610000C3
:107600007F140200060005000F0008004800520029
:1076100080FF3F00000000000000000000000000AC
:1076200000000000304000400140034007400F4090
:107630004F40CF40CF41CF43CF47CF4FCF3FCF2F4A
:10764000CF1FCF0F000000000000000000000F005F
:10765000080000003F00000040003F000000040060
:1076600068000E00DC00060043001A000500000060
:107670000000020000000000000000000400C00044
:1076800000000400C000000007000000000000002F
:1076900000000000000000000000000050C0009149
:1076A000007070C00091007082312100319110B1E2
:1076B0000070018101B100A18231329110B10191BC
:1076C0001110418141226340F106007051C00191C7
:1076D00030181039833108D01831416F31003191A1
:1076E00010B1831414166F680070251050C00091FB
:1076F000F4C340C12014036F311041045082F022C2
:107700008440512622C082312100319110B1633969
:107710003110410482C082312100319110B16339AE
:107720003110A2C082312100319110B150101531B9
:10773000051405920070536452C031103106613156
:10774000C102566412C13110213971065131E10272
:107750005664007051C0019101CCE2C0566453647C
:1077600011C1C2C0566454B0007154A064B0F0801E
:107770000022B54011C122C1566451C00191E2C03E
:10778000823160820200329110B100C3C868536434
:107790004012B09032B000C3CE6840C2D0688012B0
:1077A000B09032B00070536401C122C1566401C16F
:1077B000C2C0566453829D64C012B09032B0007053
:1077C000536472C281C0566422C111C1566402C0A2
:1077D00011C1566462C031C3566462C311C156649C
:1077E00002C311C15664538253399D64E2C35B6482
:1077F0001122F84042C281C8566452C211C1566477
:1078000072C2E1CE566402C281C8566402C201C887
:107810005664B0C00C690070536442C201C856641B
:1078200052C211C0566472C2E1C0566402C001C1A6
:10783000566462C001C3566422C101C1566462C36A
:1078400001C1566402C301C1566453829D64007035
:1078500002C1623101C0A080001E3241101A3461A1
:107860002010101A136F236E11161216346900704F
:10787000E092D08200223B45C0B2007000000000C0
:1078800000000000000000000000000000000000F8
:1078900000000000000000000000000000000000E8
:1078A00000000000067305720B720E7250B000717A
:1078B000818060B050A09280F0EFF19202933A651F
:1078C000412278458080F1C1100430160111011465
:1078D000016C8B618C618D618E618F6190619161B2
:1078E0009361956197619961706273629180F2C052
:1078F000210421318280422A1214321601112114EE
:10790000016CA661C761AC617362A661C761AC61BD
:1079100073629B619B619B619B619B619B61AC649A
:107920009B61D5649B61E2649B610E659B612A65E6
:107930009B618280E0DFF2923A65B0B0A261B1B0A3
:107940000673057230B05861D0CF3A6584C203C067
:10795000C0C36864907850916078103161781014D9
:1079600000925078403161781000403171781000F9
:107970001092B078609281782192307840314178CD
:107980001000309210C0F0919B6154A0F080502202
:10799000CF45408000226646C76100C8609159818A
:1079A00050B0918041222E46C0CF3A65128282317A
:1079B00082394239281077641282F11212042F1092
:1079C0001F312F1440C120140D6F6D39DE10F4C328
:1079D0004E0482C082312E006D39A2C082312D004A
:1079E0001A828A392082803180390BC00B18AC781A
:1079F00030824039021011C0013010C00118021845
:107A000082312100C126919103B013B063B053B00D
:107A100003823914418001226646B481C491D58124
:107A20009518B51C1C4EC51C544A6591F080102257
:107A30000C422C623D9110B13E9110B165910F92B4
:107A40005981F914AB18BC10F0805022C7411022A4
:107A50002C460C62B0CF3A6563B030820010F2C0A1
:107A60002004021011C0013010C001180218823128
:107A70002100C1269191919113B003B063B053B02E
:107A800064B054B0007141800122664663B064B0B6
:107A9000F0805022C741B181C191D181911861918B
:107AA00031B04462128282318239423928107764BF
:107AB00059810582591420820BC00B18AC7880C004
:107AC000007163B0626A0C62018262818231823D20
:107AD000A0EFF19202933A6503A09B61A2807764C4
:107AE0009B6150B000719B612DE9F04FDFF8D44AE3
:107AF000DFF8D45A207007210020E86183B0DFF856
:107B0000980B01700D21418040F222218180DFF825
:107B10008C0BDFF89C1B29628A7E0270FF2ACB7EC9
:107B2000437008BFFF2B0E7F86704F7FC77091F8A0
:107B30001EC080F804C0C97F417116D1FF2E08BF56
:107B4000FF2F12D1BCF1FF0F08BFFF290DD1DFF8C5
:107B5000641B0A7802704A7842708A788270CA7808
:107B6000C2700A79027149794171DFF84C1B0278C1
:107B7000DFF8488BDFF8487BDFF8483BDFF8486BDD
:107B80000A7042784A7082788A70C278CA70027924
:107B90000A714079DFF8342B4871FF21DFF8AC0B14
:107BA000017041708170C1700171417101202871B3
:107BB000101D017141718171C17101724172002109
:107BC00001708172A0218181032181730721C1731A
:107BD0000021017428214182012101750021817554
:107BE00002F15A0100224A7001220A7042750020F7
:107BF000DFF85C1B0880D8F82C104878A87008784B
:107C00003870801C8A782A708A681279521E1A701D
:107C1000CA786A70CA682A618969DFF8382BA96155
:107C20004FF4967111801821484380B2FEF73CFF53
:107C3000B060002855D03878010055D04FF49071CD
:107C4000484380B2FEF730FFDFF80C9BC9F8040010
:107C500008B9B06843E0387838214843FEF724FF7C
:107C6000686120B900F070F8D9F8040037E038787E
:107C7000DFF8E8AA0001FEF717FFCAF8000028B9EC
:107C800000F062F800F05CF8686928E03878DFF806
:107C9000D0BA0001FEF708FFCBF8000048B900F0A9
:107CA00053F800F04DF86869FEF70BFFDAF80000B2
:107CB00015E0387830214843FEF7F6FEDFF8A01BC8
:107CC000086088B900F040F800F03AF86869FEF7FB
:107CD000F8FEDAF80000FEF7F4FEDBF80000FEF72D
:107CE000F0FE4FF4804126E000F0BBFA0746082082
:107CF000ADF800001E20ADF802004FF40050DFF890
:107D0000641B096801906846884703F0B1F9D8F808
:107D10000C00697800880843DFF84C1B088038465F
:107D2000DFF8481B096888470C21DFF8300DFFF7A2
:107D300045FB4FF400512078F8F761FFBDE8F78F5D
:107D4000D9F80400FEF7BDBEB068FEF7BABE70B544
:107D50000C46E00788B00DD5FFF734FB38B10021A1
:107D60008160DFF80C0B0068010018BF804784F0C9
:107D7000010072E0A00707D500F071F83C2000F088
:107D8000E2FF84F0020068E06007DFF83C5827D586
:107D9000DFF8C409817840684FF490724A43024486
:107DA0006869382359430144901D12F82C3F06930B
:107DB00053891B090593838B0493D288520803923D
:107DC00000220292019201F12C020092012291F80C
:107DD00028300178002000F0B6FF84F004003CE079
:107DE000200607D500F03BF83B2000F0ACFF84F004
:107DF000800032E0A00508D5DFF8A00C016841F052
:107E00000041016084F4007027E0600504D5FCF7B0
:107E100069FA84F4806020E0600405D5812001F0D7
:107E2000CDF884F4804018E0A00415D54FF0FF3061
:107E3000E86103F0C4FC2E69366805F1340305F1EE
:107E4000480205F1240105F16000B047E86000F048
:107E500012F884F4005000E0002008B070BD00204B
:107E600006900590049003900290019000900023EA
:107E7000012200217047F8B5DFF84C47DFF8D858E9
:107E80002369E068DFF83868183300221B684FF078
:107E9000FF319847DFF82408DFF8641BC06A806868
:107EA00040790870002703F0AEFCDFF8580BFFF7AD
:107EB0008DFAFFF78FFAFFF791FADFF8780B0021C0
:107EC0000170017141718171C171017241720022B1
:107ED000DFF8F80700F10E010A70A0224A8007229D
:107EE0004A7103220A7100220A738A7200F8592F1C
:107EF0000122CA720021427081700BE068684FF461
:107F00009071794308444179012908BF03F03AFA96
:107F10007F1CFFB230788742F0DBFFF763FAA0786E
:107F2000DFF8641B087003F063FE03F098F9DFF8D4
:107F30005C1B00200870DFF8581B08700120DFF878
:107F4000541B08700020DFF8501B08700120DFF878
:107F5000501B08700020DFF84C1B0870DFF8481B2E
:107F60000870DFF8481B0880DFF8441B0870F2BD7A
:107F70002DE9F0411446DFF8485708B12A7802701D
:107F8000DFF8D48711B198F801000870002C3ED0BA
:107F9000002600271CE0C9B2DBB2605402F12800C1
:107FA0000179E154591C427900F034F8827900F0EB
:107FB00031F8C27900F02EF8027A00F02BF8427AFC
:107FC00000F028F80078C9B24E1C60547F1CFFB244
:107FD000287887421BDA3846FFF708FA0028F5D1DF
:107FE000D8F804004FF490717943F6B20844DFF8F2
:107FF000C41A4969A7553822006800787A430A44B0
:10800000711C4B1C80280CBF00200120C3E70020FE
:10801000BDE8F081C9B26254491C704738B50C0004
:10802000054601D1122032BDFFF7E0F9010017D15A
:1080300000F0DFFC01680978402901D00C2032BD36
:1080400000214B42625C0344491C102983F8E22062
:10805000F7DB012180F8E410052103F01EFA00206F
:1080600032BD10B50446FFF7C1F9010016D100F08A
:1080700036F801680978402901D00C2010BD00F1C4
:10808000F0010A78012A03D106220A77022102E0D0
:1080900006224A700D2103F000FA002010BD10B531
:1080A0000446FFF7A3F901000CD100F018F890F88E
:1080B000F810022907D1817900F1F902002000F0BF
:1080C0009DFD002010BD01680978802903D1082199
:1080D000FFF790F9F5E74029F3D1112010BDDFF843
:1080E000D80940684FF4907161430844704710B557
:1080F000040001D1122010BDDFF85C06407808B101
:108100000C2010BD03F0ABF8DFF8B00922784178FD
:10811000114041706278817811408170002010BD5B
:108120000404002138B50C00054606D0DFF88C1594
:10813000C96A89680979884201D3122032BD03F0E7
:1081400099FBDFF8BC08057001202070002032BDCB
:10815000A30300216C03002111040021DFF85C253A
:10816000D26A92681279904201D312207047DFF8E8
:10817000541508700020704710B5140019D011B1C3
:10818000012908D015E003F09AFB10F1800F207050
:108190000DD1302010BDDFF82405C06A8068016869
:1081A000007900EB4000084410F8030C2070002018
:1081B00010BD122010BD2DE9F8430C000546904675
:1081C000994605D05FEA090018BFB9F1010F01D047
:1081D000122044E0DFF8F0733878404504D28A205A
:1081E00000F0ECFE30203AE02846FFF7FFF80100EF
:1081F00035D1DFF86405DFF8906840684FF490717E
:1082000069434518307820B90120FFF7F7F80720B7
:1082100025E000F026F83178491E3170DFF84C1661
:1082200009688847B8F11C0FBCBF38781C280ADBE6
:1082300042462146284603F0A4F901000FD120460A
:10824000FCF7CFFC07E0102000904B464246214649
:10825000284603F0EEFB284603F05BFA0020BDE859
:10826000F283DFF85C080068004700005104002139
:1082700030B5DFF83C08017883B009B121203EBD5C
:10828000DFF84018DFF840480B7B496003F0E0035B
:1082900043F085030B7341F60A024B7B0A8003F01F
:1082A000F00343F002034B73002266238B734A8072
:1082B0008023CB7340F6C412DFF810388A600B615C
:1082C0004C615A6001251A7A1D8002F0FE021A7272
:1082D0002525DA7A9D7002F0F002002542F00102B5
:1082E000DD705D72DD60DA7225800D220270B64CA1
:1082F000DFF8DC27E068DFF8DC37CDE90025256909
:10830000083502222D68A84741E0000000C0002186
:1083100030B5282983B003DA050018BF012D01D03C
:1083200012203EBDDFF88847207808B121203EBDED
:10833000480000F6621081B2012003F0E2FBDFF892
:108340009817DFF89037496040F608000880002051
:1083500048808860012D087B00F06000087300F001
:1083600056F80CBF03200A2088730022DFF86C0740
:108370004861002008828861CDE90022C87C00F0B5
:1083800041F8C87402220B2000F048F8A847208169
:1083900000203EBD30B5282883B001DB12203EBD51
:1083A000DFF80C47217809B121203EBD400000F6DE
:1083B000621081B2002003F0A4FBDFF82417DFF87D
:1083C0001437496040F607000880002200204880EA
:1083D0008860CDE90022087B00F06000087302226B
:1083E00000F015F802208873DFF8F006086100201D
:1083F0004861C87B00F006F8C8730C2000F00EF846
:10840000A847C4E700F0F00040F001007047487B47
:1084100000F0F00040F00200487370472070DFF871
:1084200094462569E06808352D68704780B5DFF807
:10843000800600780B281CBF0C280D2801D02120B5
:1084400002BD40F2014003F04CFBFFF714FD002099
:1084500002BD2DE9F04F0D462828B8BF262D83B068
:10846000804616460FDA310018BF012E0DD0022EBD
:1084700018BF032E09D0042E18BF052E05D0062ED6
:1084800018BF072E01D0122099E0DFF8249699F842
:10849000001009B1212092E0DFF82846DFF82C76A1
:1084A000DFF824A641F60A01218040000021618006
:1084B0006460A1606630217B01F06001217340F6A9
:1084C000C41B617B01F0F00141F002016173A073F4
:1084D00029468020E0732761C4F814A0002038806A
:1084E000BD701846012818BF0228FE701BD100225B
:1084F00003F0DDFAB0F5BC7FD8BFC7F804B02EDDBD
:10850000B0F57A7FD8BF41F2883027DDB0F5CB6F68
:10851000D8BF41F64C5021DD40F6490188421EDAB1
:1085200042F210701AE003280CBF082002204143D9
:10853000C9001B2202FB001000F5BC7080B2F930AC
:1085400040F2712190FBF1F140F27122796002FB5F
:10855000110000B1012040180BFB00F07860387A60
:1085600000F0FE003872002100207872F860F87A7E
:10857000FFF748FFF8720020AAF80000DFF8640552
:108580008180C18080F800808021457086700172F2
:108590004C48DFF86C140078DFF818650870092083
:1085A00089F8000003F02FF900F07AF83569F068D7
:1085B000083502222D682146A84730810020BDE8F9
:1085C000FE8F0000844C00202843002030B528286E
:1085D00083B001DB12203EBDDFF8D4140B780BB161
:1085E00021203EBDDFF8DC4441F609032380420030
:1085F00000236380A3606632237BA27303F06003D1
:1086000023738022637BE27303F0F00343F00203E1
:1086100063736460DFF8D024DFF8D03422616361D3
:10862000002515600F25157101255571DFF8AC5433
:108630009560552515735573957300251561D57B88
:1086400005F0F00545F00105D57300221A805A8027
:108650009A8080229A7100229A60DFF85854DFF8DD
:108660008424107000205070FF20907000209080B3
:10867000D080802010720A20087003F0C4F800F047
:108680000FF8022221462C69E86808342468A047C4
:10869000288100203EBD00008C4C00206C4C002046
:1086A000DFF84C04DFF82C340021CDE900017047DD
:1086B000B63F0050E81200507C4C002058FE0000ED
:1086C000BC4C0020854C0020F44E0020EC490020DA
:1086D00070B5DFF8DC432078092818BF0A2801D0DC
:1086E000212070BD00F045F92078DFF8F813092843
